:020000040800F2
:1000000000060020E1010008E3010008E301000808
:10001000E3010008E3010008E3010008E301000830
:10002000E3010008E3010008E3010008652F000870
:10003000E3010008E3010008E3010008E301000810
:10004000E3010008E3010008E3010008E301000800
:10005000E3010008E30100080D3200083532000812
:100060005D32000885320008AD320008E301000867
:10007000E3010008E3010008E3010008E3010008D0
:10008000E3010008E3010008E3010008E3010008C0
:10009000E3010008E3010008E3010008D53200088D
:1000A000E3010008E3010008E3010008E3010008A0
:1000B000A9330008E3010008E3010008E301000898
:1000C000E3010008E3010008E3010008E301000880
:1000D000E3010008E3010008E3010008E301000870
:1000E00039330008E3010008E3010008E3010008D8
:1000F000E3010008E3010008E3010008E301000850
:10010000E3010008E3010008E3010008E30100083F
:10011000E3010008E3010008E3010008E30100082F
:10012000E3010008E3010008E3010008E30100081F
:10013000E3010008E3010008E3010008E30100080F
:10014000E3010008E3010008E301000819270008A3
:10015000E3010008E3010008E3010008E3010008EF
:10016000E3010008E3010008E3010008E3010008DF
:10017000E3010008E3010008E3010008E3010008CF
:10018000E3010008E3010008E3010008E3010008BF
:10019000E3010008E3010008E3010008E3010008AF
:1001A000E3010008E3010008E3010008E30100089F
:1001B000E3010008E3010008E3010008E30100088F
:1001C000E3010008E3010008E3010008E30100087F
:1001D000E3010008E3010008E3010008E30100086F
:1001E00002E000F000F8FEE772B6374880F30888B6
:1001F000364880F3098836483649086040F20000E6
:10020000CCF200004EF63471CEF200010860BFF36C
:100210004F8FBFF36F8F40F20000C0F2F0004EF638
:100220008851CEF200010860BFF34F8FBFF36F8F8C
:100230004FF00000E1EE100A4EF63C71CEF20001E4
:100240000860062080F31488BFF36F8F01F02CFF45
:1002500002F026FE4FF055301F491B4A91423CBF29
:1002600041F8040BFAE71D49184A91423CBF41F896
:10027000040BFAE71A491B4A1B4B9A423EBF51F83E
:10028000040B42F8040BF8E700201849184A914281
:100290003CBF41F8040BFAE701F00AFF02F054FEFC
:1002A000144C154DAC4203DA54F8041B8847F9E7A7
:1002B00000F042F8114C124DAC4203DA54F8041B22
:1002C0008847F9E701F0F2BE000600200022002076
:1002D0000000000808ED00E00000002000060020FB
:1002E0006837000800220020402200204022002021
:1002F000602E0020E0010008E0010008E001000895
:10030000E00100082DE9F04F2DED108AC1F80CD066
:10031000C3689D46BDEC108ABDE8F08F002383F3CF
:1003200011882846A047002001F072FAFEE701F08C
:1003300001FA00DFFEE7000038B500F0BBFB01F07A
:1003400083FE054601F0A6FE0446C8B90E4B9D4249
:1003500018D001339D4218BF044641F2883504BFCE
:1003600001240025002001F079FE0CB100F074F8A2
:1003700000F000FD284600F0BFF800F06DF8F9E746
:100380000025EFE70546EDE7010007B008B500F0EE
:1003900063FBA0F120035842584108BD07B541F264
:1003A0001203022101A8ADF8043000F073FB03B082
:1003B0005DF804FB38B5302383F3118817480368D0
:1003C0000BB101F0F1FA164A144800234FF47A7188
:1003D00001F0E0FA002383F31188124C236813B173
:1003E0002368013B2360636813B16368013B63606A
:1003F0000D4D2B7833B963687BB9022000F024FCE3
:10040000322363602B78032B07D163682BB902205A
:1004100000F01AFC4FF47A73636038BD402200206C
:10042000B50300086023002058220020084B1870F4
:1004300003280CD8DFE800F008050208022000F0CD
:10044000F9BB022000F0ECBB024B00225A6070475F
:100450005822002060230020234B244A10B51C465C
:10046000196801313FD004339342F9D16268A24246
:1004700039D31F4B9B6803F1006303F540439A4255
:1004800031D2002000F030FB0220FFF7CFFF194BE4
:100490001A6C00221A64196E1A66196E596C5A6425
:1004A000596E5A665A6E5A6942F080025A615A6908
:1004B00022F080025A615A691A6942F000521A61A8
:1004C0001A6922F000521A611B6972B64FF0E023DC
:1004D0003021C3F8084DD4E9003281F311889D46DC
:1004E00083F30888104710BD00C0000820C0000832
:1004F00000220020003802402DE9F04F93B0AA4BB3
:1005000000902022FF210AA89D6800F0DDFBA74A89
:100510001378A3B9A648012103601170302383F337
:10052000118803680BB101F03FFAA24AA0480023EA
:100530004FF47A7101F02EFA002383F31188009BA7
:1005400013B19D4B009A1A609C4A009C1378032BB0
:100550001EBF00231370984A4FF0000A18BF536063
:10056000D3465646D146012000F064FB24B1924B9D
:100570001B68002B00F01182002000F06DFA039040
:10058000039B002BF2DB012000F04AFB039B213B85
:10059000162BE8D801A252F823F000BFF905000895
:1005A00021060008B5060008670500086705000871
:1005B000670500083F0700080F0900082908000820
:1005C0008B080008B3080008D90800086705000870
:1005D000EB080008670500085D0900089906000897
:1005E00067050008A109000805060008990600082B
:1005F000670500088B0800080220FFF7C7FE0028E7
:1006000040F0F581009B0221BAF1000F08BF1C46A3
:1006100005A841F21233ADF8143000F03BFAA2E71E
:100620004FF47A7000F018FA071EEBDB0220FFF798
:10063000ADFE0028E6D0013F052F00F2DA81DFE8A9
:1006400007F0030A0D10133605230593042105A8AE
:1006500000F020FA17E054480421F9E75848042133
:10066000F6E758480421F3E74FF01C08404600F035
:100670003DFA08F104080590042105A800F00AFAE3
:10068000B8F12C0FF2D1012000FA07F747EA0B0B63
:100690005FFA8BFB4FF0000900F062FB26B10BF014
:1006A0000B030B2B08BF0024FFF778FE5BE74648DF
:1006B0000421CDE7002EA5D00BF00B030B2BA1D10D
:1006C0000220FFF763FE074600289BD0012000F0C0
:1006D0000BFA0220FFF7AAFE00261FFA86F8404612
:1006E00000F012FA044690B10021404600F01CFAD6
:1006F00001360028F1D1BA46044641F21213022114
:1007000005A8ADF814303E4600F0C4F92BE70120EF
:10071000FFF78CFE2546244B9B68AB4207D9284641
:1007200000F0E4F9013040F067810435F3E7234B32
:1007300000251D70204BBA465D603E46ACE7002E9A
:100740003FF460AF0BF00B030B2B7FF45BAF022089
:10075000FFF76CFE322000F07FF9B0F10008FFF6E1
:1007600051AF18F003077FF44DAF0F4A926808EBC2
:10077000050393423FF646AFB8F5807F3FF742AF9F
:10078000124B0193B84523DD4FF47A7000F064F901
:100790000390039A002AFFF635AF019B039A03F8F2
:1007A000012B0137EDE700BF002200205C23002071
:1007B00040220020B50300086023002058220020BA
:1007C00004220020082200200C2200205C220020AD
:1007D000C820FFF7DBFD074600283FF413AF1F2DAD
:1007E00011D8C5F1200242450AAB25F0030028BF0D
:1007F000424683490192184400F040FA019A804829
:10080000FF2100F061FA4FEAA8037D490193C8F384
:100810008702284600F060FA064600283FF46DAFD4
:10082000019B05EB830537E70220FFF7AFFD0028AA
:100830003FF4E8AE00F0A4F900283FF4E3AE00274F
:10084000B846704B9B68BB4218D91F2F11D80A9B22
:1008500001330ED027F0030312AA134453F8203CAF
:1008600005934046042205A900F0AEFA04378046FD
:10087000E7E7384600F03AF90590F2E7CDF8148042
:10088000042105A800F006F906E70023642104A866
:10089000049300F0F5F800287FF4B4AE0220FFF7CF
:1008A00075FD00283FF4AEAE049800F051F90590B4
:1008B000E6E70023642104A8049300F0E1F800288F
:1008C0007FF4A0AE0220FFF761FD00283FF49AAE4E
:1008D000049800F04DF9EAE70220FFF757FD0028E1
:1008E0003FF490AE00F05CF9E1E70220FFF74EFD27
:1008F00000283FF487AE05A9142000F057F9042121
:100900000746049004A800F0C5F83946B9E732203C
:1009100000F0A2F8071EFFF675AEBB077FF472AEBB
:10092000384A926807EB090393423FF66BAE022008
:10093000FFF72CFD00283FF465AE27F003074F4476
:10094000B9453FF4A9AE484600F0D0F8042105901F
:1009500005A800F09FF809F10409F1E74FF47A7057
:10096000FFF714FD00283FF44DAE00F009F9002810
:1009700044D00A9B01330BD008220AA9002000F0C2
:10098000ABF900283AD02022FF210AA800F09CF9F8
:10099000FFF704FD1C4800F041FF13B0BDE8F08FE5
:1009A000002E3FF42FAE0BF00B030B2B7FF42AAE7F
:1009B0000023642105A8059300F062F8074600288B
:1009C0007FF420AE0220FFF7E1FC804600283FF4D0
:1009D00019AEFFF7E3FC41F2883000F01FFF0598E5
:1009E00000F0F0F9464600F0BBF93C46BBE5064690
:1009F00052E64FF0000905E6BA467EE637467CE649
:100A00005C22002000220020A086010070B50F4B60
:100A10001B780133DBB2012B0C4611D80C4D296831
:100A20004FF47A730E6AA2FB03320146224628462F
:100A3000B047844204D1074B00221A70012070BDD8
:100A40004FF4FA7000F0EAFE0020F8E710220020D0
:100A5000082600209423002007B500230246012128
:100A60000DF107008DF80730FFF7D0FF20B19DF89A
:100A7000070003B05DF804FB4FF0FF30F9E700001A
:100A80000A4608B50421FFF7C1FF80F00100C0B29B
:100A9000404208BD30B4054C2368DD69044B0A466A
:100AA000AC460146204630BC604700BF0826002007
:100AB000A086010070B501F0CDF9094E094D3080D6
:100AC000002428683388834208D901F0BDF92B68D7
:100AD00004440133B4F5404F2B60F2D370BD00BF26
:100AE000962300206823002001F062BA00F1006024
:100AF00000F540400068704700F10060920000F58A
:100B0000404001F0EDB90000054B1A68054B1B8809
:100B10009B1A834202D9104401F096B90020704715
:100B2000682300209623002038B5084D044629B1DB
:100B300028682044BDE8384001F0A6B92868204460
:100B400001F08AF90028F3D038BD00BF68230020E7
:100B500010F003030AD1B0F5047F05D200F1005074
:100B6000A0F51040D0F80038184670470023FBE786
:100B700000F10050A0F51040D0F8100A70470000B6
:100B8000064991F8243033B10023086A81F82430F3
:100B90000822FFF7B1BF0120704700BF6C2300207F
:100BA000014B1868704700BF002004E070B5194B76
:100BB0001D68194B0138C5F30B0408442D0C0422A1
:100BC0001E88A6420BD15C680A46013C824213464D
:100BD0000FD214F9016F4EB102F8016BF6E7013A3A
:100BE00003F10803ECD181420B4602D22C2203F818
:100BF000012B0A4A05241688AE4204D1984284BFCC
:100C0000967803F8016B013C02F10402F3D1581A03
:100C100070BD00BF002004E08C3400087834000868
:100C2000022802BF024B4FF000429A61704700BF9A
:100C300000080240022802BF024B4FF400429A61B2
:100C4000704700BF00080240022801BF024A5369F2
:100C500083F40043536170470008024070B50446B6
:100C60004FF47A764CB1412C254628BF412506FB2E
:100C700005F000F0D3FD641BF4E770BD10B5002350
:100C8000934203D0CC5CC4540133F9E710BD00009B
:100C900010B5013810F9013F3BB191F900409C4279
:100CA00003D11AB10131013AF4E71AB191F90020E8
:100CB000981A10BD1046FCE703460246D01A12F9F6
:100CC000011B0029FAD1704702440346934202D027
:100CD00003F8011BFAE770472DE9F8431F4D14464E
:100CE00095F824200746884652BBDFF870909CB3E5
:100CF00095F824302BB92022FF2148462F62FFF7B8
:100D0000E3FF95F82400C0F10802A24228BF224662
:100D1000D6B24146920005EB8000FFF7AFFF95F891
:100D20002430A41B1E44F6B2082E17449044E4B2AB
:100D300085F82460DBD1FFF723FF0028D7D108E036
:100D40002B6A03EB82038342CFD0FFF719FF002801
:100D5000CBD10020BDE8F8830120FBE76C23002005
:100D6000024B1A78024B1A70704700BF9423002080
:100D70001022002010B5104C104800F0B5F82146A4
:100D80000E4800F0DDF82468626DD2F8043843F0B4
:100D90000203C2F804384FF47A70FFF75FFF084986
:100DA000204600F0D3F9626DD2F8043823F0020334
:100DB000C2F8043810BD00BF5835000808260020CE
:100DC000603500087047000030B5094D0A44914273
:100DD0000DD011F8013B5840082340F30004013BBB
:100DE0002C4013F0FF0384EA5000F6D1EFE730BD4A
:100DF0002083B8ED026843681143016003B11847CE
:100E00007047000013B5446BD4F894341A68117815
:100E1000042915D1217C022912D1197912890123C3
:100E20008B4013420CD101A904F14C0001F0F4FEF7
:100E3000D4F89444019B21790246206800F0D0F94F
:100E400002B010BD143001F077BE00004FF0FF3348
:100E5000143001F071BE00004C3001F049BF0000B9
:100E60004FF0FF334C3001F043BF0000143001F06D
:100E700045BE00004FF0FF31143001F03FBE0000CE
:100E80004C3001F015BF00004FF0FF324C3001F044
:100E90000FBF00000020704710B5D0F894341A68D6
:100EA00011780429044617D1017C022914D15979FB
:100EB000528901238B4013420ED1143001F0D8FD2A
:100EC000024648B1D4F894444FF4807361792068A5
:100ED000BDE8104000F072B910BD0000406BFFF794
:100EE000DBBF0000704700007FB5124B036000239A
:100EF0004360C0E90233012502260F4B0574044606
:100F00000290019300F18402294600964FF4807309
:100F1000143001F089FD094B0294CDE9006304F51A
:100F200023724FF48073294604F14C0001F050FE07
:100F300004B070BDAC340008DD0E0008050E0008DA
:100F40000B68302282F311880A7903EB82029061E8
:100F50004A79093243F822008A7912B103EB8203FD
:100F600098610223C0F894140374002080F3118860
:100F70007047000038B5037F044613B190F8543031
:100F8000ABB9201D01250221FFF734FF04F1140045
:100F900025776FF0010100F069FC84F8545004F1EA
:100FA0004C006FF00101BDE8384000F05FBC38BD77
:100FB00010B5012104460430FFF71CFF00232377FE
:100FC00084F8543010BD000038B5044600251430B4
:100FD00001F042FD04F14C00257701F011FE201DC7
:100FE00084F854500121FFF705FF2046BDE8384042
:100FF000FFF752BF90F8443003F06003202B07D175
:1010000090F84520212A4FF0000303D81F2A06D864
:1010100000207047222AFBD1C0E90E3303E0034AC7
:1010200082630722C26303640120704711220020FB
:1010300037B5D0F894341A681178042904461AD1C7
:10104000017C022917D11979128901238B4013429F
:1010500011D100F14C05284601F092FE58B101A9CA
:10106000284601F0D9FDD4F89444019B2179024629
:10107000206800F0B5F803B030BD0000F0B500EB1B
:10108000810385B09E6904460D46FEB1302383F38B
:10109000118804EB8507301D0821FFF7ABFEFB68C4
:1010A0005B691B6806F14C001BB1019001F0C2FDA9
:1010B000019803A901F0B0FD024648B1039B2946FF
:1010C000204600F08DF8002383F3118805B0F0BDB1
:1010D000FB685A691268002AF5D01B8A013B13404D
:1010E000F1D104F14402EAE7093138B550F8214062
:1010F000DCB1302383F31188D4F894241368527937
:1011000003EB8203DB689B695D6845B104216018CD
:10111000FFF770FE294604F1140001F0B3FC2046ED
:10112000FFF7BAFE002383F3118838BD7047000033
:1011300001F012B8012303700023C0E90133C36139
:1011400083620362C36243620363704738B5044637
:10115000302383F311880025C0E90355C0E9055504
:10116000416001F009F80223237085F311882846B5
:1011700038BD000070B500EB810305465069DA60A8
:101180000E46144618B110220021FFF79DFDA069FC
:1011900018B110220021FFF797FD31462846BDE81F
:1011A000704001F0B3B80000826802F00112826062
:1011B0000022C0E90422826101F034B9F0B400EBEE
:1011C00081044789E4680125A4698D403D43458138
:1011D00023600023A2606360F0BC01F04FB90000FF
:1011E000F0B400EB81040789E468012564698D404F
:1011F0003D43058123600023A2606360F0BC01F0E1
:10120000C9B9000070B50223002504460370C0E987
:101210000255C0E90455C564856180F8345001F079
:1012200011F863681B6823B129462046BDE8704069
:10123000184770BD0378052B10B504460AD080F816
:1012400050300523037043681B680BB10421984795
:101250000023A36010BD00000178052906D190F895
:101260005020436802701B6803B1184770470000A4
:1012700070B590F83430044613B1002380F8343050
:1012800004F14402204601F0EFF863689B68B3B9AB
:1012900094F8443013F0600535D00021204601F069
:1012A0008FFB0021204601F081FB63681B6813B1AE
:1012B000062120469847062384F8343070BD204626
:1012C00098470028E4D0B4F84A30E26B9A4288BFCD
:1012D000E36394F94430E56B002B4FF0300380F268
:1012E0000381002D00F0F280092284F8342083F37A
:1012F00011880021D4E90E232046FFF771FF002357
:1013000083F31188DAE794F8452003F07F0343EA7A
:10131000022340F20232934200F0C58021D8B3F597
:10132000807F48D00DD8012B3FD0022B00F0938056
:10133000002BB2D104F14C02A2630222E2632364C7
:10134000C1E7B3F5817F00F09B80B3F5407FA4D166
:1013500094F84630012BA0D1B4F84C3043F002038E
:1013600032E0B3F5006F4DD017D8B3F5A06F31D090
:10137000A3F5C063012B90D8636894F846205E689B
:1013800094F84710B4F848302046B047002884D07D
:101390004368A3630368E3631AE0B3F5106F36D0C4
:1013A00040F6024293427FF478AF5C4BA363022382
:1013B000E3630023C3E794F84630012B7FF46DAF5D
:1013C000B4F84C3023F00203C4E90E55A4F84C30B5
:1013D000256478E7B4F84430B3F5A06F0ED194F8E3
:1013E000463084F84E30204600F084FF63681B6866
:1013F00013B1012120469847032323700023C4E939
:101400000E339CE704F14F03A3630123C3E7237862
:10141000042B10D1302383F311882046FFF7C4FE3C
:1014200085F311880321636884F84F5021701B688D
:101430000BB12046984794F84630002BDED084F854
:101440004F300423237063681B68002BD6D0022121
:1014500020469847D2E794F848301D0603F00F0164
:1014600020460AD500F0F2FF012804D002287FF4BC
:1014700014AF2B4B9AE72B4B98E700F0D9FFF3E71B
:1014800094F84630002B7FF408AF94F8483013F0FE
:101490000F01B3D01A06204602D501F0A5FAADE738
:1014A00001F098FAAAE794F84630002B7FF4F5AEE5
:1014B00094F8483013F00F01A0D01B06204602D547
:1014C00001F07EFA9AE701F071FA97E7142284F8A6
:1014D000342083F311882B462A4629462046FFF7FD
:1014E0006DFE85F31188E9E65DB1152284F834209C
:1014F00083F311880021D4E90E232046FFF75EFE16
:10150000FDE60B2284F8342083F311882B462A460B
:1015100029462046FFF764FEE3E700BFDC340008FD
:10152000D4340008D834000838B590F83430044674
:10153000002B3ED0063BDAB20F2A34D80F2B32D81C
:10154000DFE803F0373131082232313131313131C6
:1015500031313737C56BB0F84A309D4214D2C36879
:101560001B8AB5FBF3F203FB12556DB9302383F3ED
:1015700011882B462A462946FFF732FE85F311884B
:101580000A2384F834300EE0142384F834303023F6
:1015900083F3118800231A4619462046FFF70EFEF2
:1015A000002383F3118838BD036C03B198470023EF
:1015B000E7E70021204601F003FA0021204601F070
:1015C000F5F963681B6813B1062120469847062386
:1015D000D7E7000010B590F83430142B044629D01A
:1015E00017D8062B05D001D81BB110BD093B022B23
:1015F000FBD80021204601F0E3F90021204601F04C
:10160000D5F963681B6813B1062120469847062365
:1016100019E0152BE9D10B2380F83430302383F304
:10162000118800231A461946FFF7DAFD002383F3D9
:101630001188DAE7C3689B695B68002BD5D1036C1E
:1016400003B19847002384F83430CEE700230375B4
:10165000826803691B6899689142FBD25A680360EB
:101660004260106058607047002303758268036908
:101670001B6899689142FBD85A6803604260106009
:101680005860704708B50846302383F311880B7DF6
:10169000032B05D0042B0DD02BB983F3118808BD83
:1016A0008B6900221A604FF0FF338361FFF7CEFF92
:1016B0000023F2E7D1E9003213605A60F3E700003B
:1016C000FFF7C4BF054BD9680875186802681A602F
:1016D000536001220275D860FEF714BE98230020E3
:1016E00030B50C4BDD684B1C87B004460FD02B4641
:1016F000094A684600F04EF92046FFF7E3FF009BD9
:1017000013B1684600F050F9A86907B030BDFFF783
:10171000D9FFF9E79823002085160008044B1A68C2
:10172000DB6890689B68984294BF00200120704756
:1017300098230020084B10B51C68D86822681A60EE
:10174000536001222275DC60FFF78EFF01462046C0
:10175000BDE81040FEF7D6BD9823002038B5074CF1
:1017600007490848012300252370656001F040FB0C
:101770000223237085F3118838BD00BF00260020A6
:10178000E43400089823002000F044B9034A51686B
:1017900053685B1A9842FBD8704700BF001000E006
:1017A0008B60022308618B82084670478368A3F12F
:1017B000840243F8142C026943F8442C426943F82C
:1017C000402C094A43F8242CC26843F8182C022202
:1017D00003F80C2C002203F80B2C044A43F8102CBD
:1017E000A3F12000704700BF1D03000898230020CC
:1017F00008B5FFF7DBFFBDE80840FFF761BF000059
:10180000024BDB6898610F20FFF75CBF9823002034
:10181000302383F31188FFF7F3BF000008B50146BA
:10182000302383F311880820FFF75AFF002383F346
:10183000118808BD064BDB6839B1426818605A60F0
:10184000136043600420FFF74BBF4FF0FF30704739
:10185000982300200368984206D01A6802605060FE
:1018600099611846FFF72CBF7047000038B5044651
:101870000D462068844200D138BD036823605C6057
:101880008561FFF71DFFF4E710B503689C68A2426D
:101890000CD85C688A600B604C6021605960996864
:1018A0008A1A9A604FF0FF33836010BD1B68121BC9
:1018B000ECE700000A2938BF0A2170B504460D463E
:1018C0000A26601901F08EFA01F07AFA041BA5428B
:1018D00003D8751C2E460446F3E70A2E04D9BDE84A
:1018E0007040012001F0C4BA70BD0000F8B5144B7F
:1018F0000D46D96103F1100141600A2A196982601D
:1019000038BF0A22016048601861A818144601F027
:101910005BFA0A2701F054FA431BA342064606D39A
:101920007C1C281901F05EFA27463546F2E70A2F9B
:1019300004D9BDE8F840012001F09ABAF8BD00BF13
:1019400098230020F8B506460D4601F039FA0F4AF3
:10195000134653F8107F9F4206D12A46014630466F
:10196000BDE8F840FFF7C2BFD169BB68441A2C1923
:1019700028BF2C46A34202D92946FFF79BFF2246E7
:1019800031460348BDE8F840FFF77EBF98230020AA
:10199000A823002010B4C0E9032300235DF8044B02
:1019A0004361FFF7CFBF000010B5194C236998427F
:1019B0000DD0D0E90032816813605A609A680A44F9
:1019C0009A60002303604FF0FF33A36110BD2346EC
:1019D000026843F8102F53600022026022699A4285
:1019E00003D1BDE8104001F0F7B9936881680B445A
:1019F000936001F0E5F92269E1699268441AA24214
:101A0000E4D91144BDE81040091AFFF753BF00BFE5
:101A1000982300202DE9F047DFF8BC8008F110077B
:101A20002C4ED8F8105001F0CBF9D8F81C40AA6819
:101A3000031B9A423ED81444D5E900324FF0000906
:101A4000C8F81C4013605A60C5F80090D8F81030F0
:101A5000B34201D101F0C0F989F31188D5E903310E
:101A600028469847302383F311886B69002BD8D020
:101A700001F0A6F96A69A0EB04094A4582460DD235
:101A8000022001F0F5F90022D8F81030B34208D155
:101A900051462846BDE8F047FFF728BF121A2244F6
:101AA000F2E712EB090938BF4A4629463846FFF7E4
:101AB000EBFEB5E7D8F81030B34208D01444211A31
:101AC000C8F81C00A960BDE8F047FFF7F3BEBDE809
:101AD000F08700BFA8230020982300200020704733
:101AE000FEE70000704700004FF0FF307047000035
:101AF00002290CD0032904D00129074818BF00206F
:101B00007047032A05D8054800EBC2007047044817
:101B100070470020704700BFBC350008202200201D
:101B20007035000870B59AB00546084601A91446FC
:101B300000F0C2F801A8FFF7BFF8431C5B00C5E93D
:101B400000340022237003236370C6B201AB023459
:101B50001046D1B28E4204F1020401D81AB070BD11
:101B600013F8011B04F8021C04F8010C0132F0E721
:101B700008B5302383F311880348FFF759FA00238F
:101B800083F3118808BD00BF0826002090F8443078
:101B900003F01F02012A07D190F845200B2A03D138
:101BA0000023C0E90E3315E003F06003202B08D1B9
:101BB000B0F848302BB990F84520212A03D81F2AC5
:101BC00004D8FFF717BA222AEBD0FAE7034A826358
:101BD0000722C26303640120704700BF182200205F
:101BE00007B5052917D8DFE801F0191603191920E0
:101BF000302383F31188104A01900121FFF7BAFACC
:101C000001980E4A0221FFF7B5FA0D48FFF7DCF9FB
:101C1000002383F3118803B05DF804FB302383F3C2
:101C200011880748FFF7A6F9F2E7302383F31188FC
:101C30000348FFF7BDF9EBE710350008343500081D
:101C40000826002038B50C4D0C4C0D492A4604F1ED
:101C50000800FFF767FF05F1CA0204F11000094907
:101C6000FFF760FF05F5CA7204F118000649BDE8E8
:101C70003840FFF757BF00BFD02A002020220020A5
:101C8000F0340008FA3400080535000870B5044641
:101C900008460D46FFF710F8C6B220460134037817
:101CA0000BB9184670BD32462946FEF7F1FF0028F1
:101CB000F3D10120F6E700002DE9F84F05460C4668
:101CC000FEF7FAFF2949C6B22846FFF7DFFF08B141
:101CD000013EF6B226492846FFF7D8FF08B1103674
:101CE000F6B2632E0DD8DFF88490DFF884A0214F80
:101CF000DFF888B0DFF888802E7846B92670BDE816
:101D0000F88F29462046BDE8F84F01F097BB252EF5
:101D100028D1072249462846FEF7BAFF40B9D8F82D
:101D200000302360B8F80430A38007350634E3E7B9
:101D3000082251462846FEF7ABFF98B90E4BA21C6D
:101D4000197809090232C95D02F8041C13F8011B55
:101D500001F00F015B45C95D02F8031CF0D1183496
:101D60000835C9E704F8016B0135C5E7DC35000823
:101D700005350008EB350008107AFF1F1C7AFF1F9D
:101D8000E4350008BFF34F8F024AD368DB03FCD46D
:101D9000704700BF003C024008B5094B1B7873B97F
:101DA000FFF7F0FF074B1A69002ABFBF064A5A60C7
:101DB00002F188325A601A6822F480621A6008BD03
:101DC0002E2D0020003C02402301674508B50B4B37
:101DD0001B7893B9FFF7D6FF094B1A6942F000420E
:101DE0001A611A6842F480521A601A6822F480520A
:101DF0001A601A6842F480621A6008BD2E2D002015
:101E0000003C02400B28F0B516D80C4C0C49237846
:101E10007BB90C4D0E460C234FF0006255F8047B45
:101E200046F8042B013B13F0FF033A44F6D101239B
:101E3000237051F82000F0BD0020FCE7602D002049
:101E4000302D0020FC350008014B53F8200070476E
:101E5000FC3500080C2070470B2810B5044601D94A
:101E6000002010BDFFF7CEFF064B53F82430184476
:101E7000C21A0BB90120F4E712680132F0D1043B19
:101E8000F6E700BFFC3500080B2810B5044621D842
:101E9000FFF778FFFFF780FF0F4AF323D360C300FB
:101EA000DBB243F4007343F002031361136943F49C
:101EB00080331361FFF766FFFFF7A4FF074B53F86A
:101EC000241000F0D9F8FFF781FF2046BDE810404C
:101ED000FFF7C2BF002010BD003C0240FC350008E7
:101EE000F8B512F00103144642D18218B2F1016F25
:101EF00057D82D4B1B6813F0010352D02B4DFFF721
:101F00004BFFF323EB60FFF73DFF40F20127032C6B
:101F100015D824F001046618244C401A40F2011729
:101F2000B142236900EB010524D123F001032361B1
:101F3000FFF74CFF0120F8BD043C0430E7E78307BE
:101F4000E7D12B6923F440732B612B693B432B6151
:101F500051F8046B0660BFF34F8FFFF713FF036860
:101F60009E42E9D02B6923F001032B61FFF72EFF7E
:101F70000020E0E723F44073236123693B4323619E
:101F80000B882B80BFF34F8FFFF7FCFE2D8831F8B5
:101F9000023BADB2AB42C3D0236923F001032361FE
:101FA000E4E71846C7E700BF00380240003C0240A3
:101FB000084908B50B7828B11BB9FFF7EDFE0123DE
:101FC0000B7008BD002BFCD0BDE808400870FFF77F
:101FD000FDBE00BF2E2D002010B50244064BD2B22C
:101FE000904200D110BD441C00B253F8200041F8CB
:101FF000040BE0B2F4E700BF502800400F4B30B5AF
:102000001C6F240407D41C6F44F400741C671C6FFD
:1020100044F400441C670A4C236843F48073236033
:102020000244084BD2B2904200D130BD441C00B2F1
:1020300051F8045B43F82050E0B2F4E70038024066
:10204000007000405028004007B5012201A900207F
:10205000FFF7C2FF019803B05DF804FB13B5044617
:10206000FFF7F2FFA04205D0012201A90020019450
:10207000FFF7C4FF02B010BD70470000034B1A68A1
:102080001AB9034AD2F874281A607047642D0020E8
:102090000030024008B5FFF7F1FF024B1868C0F3AB
:1020A000407008BD642D002070470000FEE700006E
:1020B0000A4B0B480B4A90420BD30B4BDA1C121AFB
:1020C000C11E22F003028B4238BF00220021FEF71E
:1020D000FBBD53F8041B40F8041BECE7A8370008CD
:1020E000602E0020602E0020602E002070B5D0E908
:1020F00015439E6800224FF0FF3504EB4213510157
:10210000D3F800090028BEBFD3F8000940F0804092
:10211000C3F80009D3F8000B0028BEBFD3F8000BAA
:1021200040F08040C3F8000B013263189642C3F8B8
:102130000859C3F8085BE0D24FF00113C4F81C380B
:1021400070BD0000890141F02001016103699B0617
:10215000FCD41220FFF71ABB10B5054C2046FEF741
:10216000E9FF4FF0A0436365024BA36510BD00BFBC
:10217000682D00205036000870B50378012B054605
:1021800050D12A4B446D98421BD1294B5A6B42F0D7
:1021900080025A635A6D42F080025A655A6D5A693C
:1021A00042F080025A615A6922F080025A610E217F
:1021B00043205B6900F022FC1E4BE3601E4BC4F819
:1021C00000380023C4F8003EC02323606E6D4FF436
:1021D0000413A3633369002BFCDA012333610C2061
:1021E000FFF7D4FA3369DB07FCD41220FFF7CEFAED
:1021F0003369002BFCDA0026A6602846FFF776FF3D
:102200006B68C4F81068DB68C4F81468C4F81C680C
:102210004BB90A4BA3614FF0FF336361A36843F0EE
:102220000103A36070BD064BF4E700BF682D0020DA
:10223000003802404014004003002002003C30C03F
:10224000083C30C0F8B5446D054600212046FFF734
:1022500079FFA96D00234FF001128F68C4F834385C
:102260004FF00066C4F81C284FF0FF3004EB431217
:1022700001339F42C2F80069C2F8006BC2F8080936
:10228000C2F8080BF2D20B686A6DEB65636210232B
:102290001361166916F01006FBD11220FFF776FACB
:1022A000D4F8003823F4FE63C4F80038A36943F47B
:1022B000402343F01003A3610923C4F81038C4F885
:1022C00014380A4BEB604FF0C043C4F8103B084B86
:1022D000C4F8003BC4F81069C4F80039EB6D03F191
:1022E000100243F48013EA65A362F8BD2C3600089F
:1022F00040800010426D90F84E10D2F8003823F460
:10230000FE6343EA0113C2F8003870472DE9F84331
:1023100000EB8103456DDA68166806F00306731E4C
:10232000022B05EB41130C4680460FFA81F94FEA68
:1023300041104FF00001C3F8101B4FF0010104F1F0
:10234000100398BFB60401FA03F391698EBF334EB0
:1023500006F1805606F5004600293AD0578A04F166
:102360005801490137436F50D5F81C180B43C5F885
:102370001C382B180021C3F8101953690127611E5E
:10238000A7409BB3138A928B9B08012A88BF5343B3
:10239000D8F85C20981842EA034301F1400205EBAB
:1023A0008202C8F85C00214653602846FFF7CAFE47
:1023B00008EB8900C3681B8A43EA845348346401EC
:1023C0001E432E51D5F81C381F43C5F81C78BDE8B4
:1023D000F88305EB4917D7F8001B21F40041C7F833
:1023E000001BD5F81C1821EA0303C0E704F13F03E2
:1023F00005EB83030A4A5A6028462146FFF7A2FEEE
:1024000005EB4910D0F8003923F40043C0F8003937
:10241000D5F81C3823EA0707D7E700BF0080001073
:1024200000040002826D1268C265FFF75FBE000003
:102430005831436D49015B5813F4004004D013F444
:10244000001F0CBF02200120704700004831436D7F
:1024500049015B5813F4004004D013F4001F0CBF73
:10246000022001207047000000EB8101CB68196A4F
:102470000B6813604B6853607047000000EB8103EA
:1024800030B5DD68AA691368D36019B9402B84BFE1
:10249000402313606B8A1468426D1C44013CB4FBFA
:1024A000F3F46343033323F0030302EB411043EAE5
:1024B000C44343F0C043C0F8103B2B6803F0030350
:1024C000012B09B20ED1D2F8083802EB411013F4F7
:1024D000807FD0F8003B14BF43F0805343F000539B
:1024E000C0F8003B02EB4112D2F8003B43F004433A
:1024F000C2F8003B30BD00002DE9F041244D6E6D67
:1025000006EB40130446D3F8087BC3F8087B380772
:102510000AD5D6F81438190706D505EB84032146E9
:10252000DB6828465B689847FA071FD5D6F8143849
:10253000DB071BD505EB8403D968CCB98B69488AC6
:102540005A68B2FBF0F600FB16228AB91868DA68FE
:1025500090420DD2121AC3E90024302383F311886C
:102560000B482146FFF78AFF84F31188BDE8F0810C
:10257000012303FA04F26B8923EA02036B81CB681F
:10258000002BF3D021460248BDE8F041184700BFB8
:10259000682D002000EB810370B5DD68436D6C6928
:1025A0002668E6604A0156BB1A444FF40020C2F880
:1025B00010092A6802F00302012A0AB20ED1D3F8E8
:1025C000080803EB421410F4807FD4F8000914BF0C
:1025D00040F0805040F00050C4F8000903EB421274
:1025E000D2F8000940F00440C2F80009D3F83408DA
:1025F000012202FA01F10143C3F8341870BD19B980
:10260000402E84BF4020206020682E8A8419013C1F
:10261000B4FBF6F440EAC44040F000501A44C6E768
:102620002DE9F8433B4D6E6D06EB40130446D3F89D
:102630000889C3F8088918F0010F4FEA40171AD02B
:10264000D6F81038DB0716D505EB8003D9684B693F
:102650001868DA68904230D2121A4FF000091A60F6
:10266000C3F80490302383F3118821462846FFF7EE
:1026700091FF89F3118818F0800F1CD0D6F83438F8
:102680000126A640334216D005EB84036D6DD3F8C6
:102690000CC0DCF814200134E4B2D2F800E005EB01
:1026A00004342F445168714515D3D5F8343823EAE2
:1026B0000606C5F83468BDE8F883012303FA04F27E
:1026C0002B8923EA02032B818B68002BD3D0214670
:1026D00028469847CFE7BCF81000AEEB01038342D1
:1026E00028BF0346D7F8180980B2B3EB800FE2D8B1
:1026F0009068A0F1040959F8048FC4F80080A0EB99
:1027000009089844B8F1040FF5D818440B449060B8
:102710005360C7E7682D00202DE9F74FA24C656D87
:102720006E69AB691E4016F480586E6107D0204672
:10273000FEF768FD03B0BDE8F04F00F047BC002E87
:1027400012DAD5F8003E98489B071EBFD5F8003E28
:1027500023F00303C5F8003ED5F8043823F0010345
:10276000C5F80438FEF778FD370505D58E48FFF724
:10277000BDFC8D48FEF75EFDB0040CD5D5F80838D9
:1027800013F0060FEB6823F470530CBF43F410539F
:1027900043F4A053EB6031071BD56368DB681BB9BA
:1027A000AB6923F00803AB612378052B0CD1D5F876
:1027B000003E7D489A071EBFD5F8003E23F0030374
:1027C000C5F8003EFEF748FD6368DB680BB176484C
:1027D0009847F30274D4B70227D5D4F85490DFF8A1
:1027E000C8B100274FF0010A09EB4712D2F8003BAD
:1027F00003F44023B3F5802F11D1D2F8003B002B16
:102800000DDA62890AFA07F322EA0303638104EB13
:102810008703DB68DB6813B1394658469847A36DD8
:1028200001379B68FFB29F42DED9F00617D5676D6E
:102830003A6AC2F30A1002F00F0302F4F012B2F582
:10284000802F00F08580B2F5402F08D104EB830380
:102850000022DB681B6A07F5805790426AD130037B
:10286000D5F8184813D5E10302D50020FFF744FE40
:10287000A20302D50120FFF73FFE630302D5022029
:10288000FFF73AFE270302D50320FFF735FE750355
:102890007FF550AFE00702D50020FFF7C1FEA1078A
:1028A00002D50120FFF7BCFE620702D50220FFF728
:1028B000B7FE23077FF53EAF0320FFF7B1FE39E7F0
:1028C000636DDFF8E4A0019300274FF00109A36DC9
:1028D0009B685FFA87FB9B453FF67DAF019B03EB4F
:1028E0004B13D3F8001901F44021B1F5802F1FD10B
:1028F000D3F8001900291BDAD3F8001941F09041F0
:10290000C3F80019D3F800190029FBDB5946606DA4
:10291000FFF718FC218909FA0BF321EA030323814D
:1029200004EB8B03DB689B6813B15946504698470C
:102930000137CCE7910708BFD7F80080072A98BF76
:1029400003F8018B02F1010298BF4FEA182884E7CF
:10295000023304EB830207F580575268D2F818C09F
:10296000DCF80820DCE9001CA1EB0C0C00218842FB
:102970000AD104EB830463689B699A6802449A60F5
:102980005A6802445A606AE711F0030F08BFD7F88B
:1029900000808C4588BF02F8018B01F1010188BFDE
:1029A0004FEA1828E3E700BF682D0020436D03EBD2
:1029B0004111D1F8003B43F40013C1F8003B7047CC
:1029C000436D03EB4111D1F8003943F40013C1F812
:1029D00000397047436D03EB4111D1F8003B23F4FC
:1029E0000013C1F8003B7047436D03EB4111D1F870
:1029F000003923F40013C1F80039704700F1604337
:102A000003F561430901C9B283F80013012200F004
:102A10001F039A4043099B0003F1604303F56143A0
:102A2000C3F880211A60704730B5039C01720433EB
:102A300004FB0325C0E90653049B03630021059BA7
:102A4000C160C0E90000C0E90422C0E90842C0E951
:102A50000A11436330BD0000416A0022C0E904113D
:102A6000C0E90A22C2606FF00101FEF7FFBE00005C
:102A7000D0E90432934201D1C2680AB9181D7047E7
:102A80000020704703691960C2680132C260C269E0
:102A9000134482690361934224BF436A03610021A6
:102AA000FEF7D8BE38B504460D46E3683BB162690F
:102AB000131D1268A3621344E362002007E0237A27
:102AC00033B929462046FEF7B5FE0028EDDA38BDB9
:102AD0006FF00100FBE70000C368C269013BC360FF
:102AE0004369134482694361934224BF436A43614B
:102AF00000238362036B03B11847704770B530231E
:102B0000044683F31188866A3EB9FFF7CBFF05467A
:102B100018B186F31188284670BDA36AE26A13F8DB
:102B2000015BA362934202D32046FFF7D5FF002347
:102B300083F31188EFE700002DE9F84F04460E46B5
:102B4000174698464FF0300989F311880025AA46A8
:102B5000D4F828B0BBF1000F09D141462046FFF759
:102B6000A1FF20B18BF311882846BDE8F88FD4E986
:102B70000A12A7EB050B521A934528BF9346BBF1E7
:102B8000400F1BD9334601F1400251F8040B43F8C2
:102B9000040B9142F9D1A36A40334036A362403519
:102BA000D4E90A239A4202D32046FFF795FF8AF31D
:102BB0001188BD42D8D289F31188C9E730465A46F8
:102BC000FEF75CF8A36A5B445E44A3625D44E7E7FA
:102BD00010B5029C0172043303FB0421C0E9061303
:102BE0000023C0E90A33039B0363049BC460C0E96C
:102BF0000000C0E90422C0E90842436310BD0000A0
:102C0000026AC260426AC0E904220022C0E90A22C4
:102C10006FF00101FEF72ABED0E904239A4201D1E8
:102C2000C26822B9184650F8043B0B607047002375
:102C30001846FAE7C368C2690133C36043691344A5
:102C400082694361934224BF436A43610021FEF7D6
:102C500001BE000038B504460D46E3683BB1236968
:102C60001A1DA262E2691344E362002007E0237A9E
:102C700033B929462046FEF7DDFD0028EDDA38BDE0
:102C80006FF00100FBE7000003691960C268013AB8
:102C9000C260C269134482690361934224BF436ADC
:102CA000036100238362036B03B118477047000080
:102CB00070B530230D460446114683F31188866AA9
:102CC0002EB9FFF7C7FF10B186F3118870BDA36A54
:102CD0001D70A36AE26A01339342A36204D3E169DF
:102CE00020460439FFF7D0FF002080F31188EDE77C
:102CF0002DE9F84F04460D46904699464FF0300AAC
:102D00008AF311880026B346A76A4FB94946204680
:102D1000FFF7A0FF20B187F311883046BDE8F88F98
:102D2000D4E90A073A1AA8EB0607974228BF1746C4
:102D3000402F1BD905F1400355F8042B40F8042B14
:102D40009D42F9D1A36A4033A3624036D4E90A23F5
:102D50009A4204D3E16920460439FFF795FF8BF3CB
:102D600011884645D9D28AF31188CDE729463A46DB
:102D7000FDF784FFA36A3B443D44A3623E44E5E77C
:102D8000D0E904239A4217D1C3689BB1836A8BB1FF
:102D9000043B9B1A0ED01360C368013BC360C36938
:102DA0001A44836902619A4224BF436A0361002383
:102DB00083620123184670470023FBE700F030B917
:102DC0004FF08043586A70474FF0804300225863A9
:102DD0001A610222DA6070474FF080430022DA6005
:102DE000704700004FF0804358637047FEE70000D3
:102DF00070B51B4B01630025044686B058608562A0
:102E00000E4600F0BFF804F11003C4E904334FF09C
:102E1000FF33C4E90635C4E90044A560E562FFF765
:102E2000CFFF2B460246C4E9082304F134010D4AC2
:102E3000256580232046FEF7B3FC0123E0600A4AA3
:102E40000375009272680192B268CDE90223074BC4
:102E50006846CDE90435FEF7CBFC06B070BD00BF77
:102E6000002600205C36000861360008ED2D0008C1
:102E7000024AD36A1843D062704700BF98230020EB
:102E80004B6843608B688360CB68C3600B694361A8
:102E90004B6903628B6943620B68036070470000F3
:102EA00008B5264B26481A6940F2FF110A431A61F9
:102EB0001A6922F4FF7222F001021A611A691A6B70
:102EC0000A431A631A6D0A431A651E4A1B6D11469E
:102ED000FFF7D6FF02F11C0100F58060FFF7D0FF7D
:102EE00002F1380100F58060FFF7CAFF02F15401DA
:102EF00000F58060FFF7C4FF02F1700100F580600B
:102F0000FFF7BEFF02F18C0100F58060FFF7B8FF0C
:102F100002F1A80100F58060FFF7B2FF02F1C401E1
:102F200000F58060FFF7ACFF02F1E00100F5806082
:102F3000FFF7A6FFBDE8084000F0EEB800380240F9
:102F4000000002406836000808B500F059FAFEF7A4
:102F500005FCFFF793F8BDE80840FEF773BE0000DC
:102F600070470000EFF3098305494A6B22F0010224
:102F70004A63683383F30988002383F31188704719
:102F800000EF00E0302080F3118862B60C4B0D4A50
:102F9000D96821F4E0610904090C0A43DA60D3F826
:102FA000FC20094942F08072C3F8FC200A6842F014
:102FB00001020A602022DA7783F82200704700BFFE
:102FC00000ED00E00003FA05001000E010B530232A
:102FD00083F311880E4B5B6813F4006314D0F1EE99
:102FE000103AEFF30984683C4FF08073E361094BBA
:102FF000DB6B236684F30988FEF790FB10B1064B68
:10300000A36110BD054BFBE783F31188F9E700BF0F
:1030100000ED00E000EF00E02F030008320300089D
:103020000F4B1A6C42F001021A641A6E42F0010250
:103030001A660C4A1B6E936843F0010393604FF0CD
:10304000804353229A624FF0FF32DA6200229A6183
:103050005A63DA605A6001225A611A60704700BFF1
:1030600000380240002004E04FF0804208B51169AA
:10307000D3680B40D9B2C9439B07116107D53023F0
:1030800083F31188FEF780FB002383F3118808BDCA
:103090001F4B1A696FEAC2526FEAD2521A611A695B
:1030A000C2F308021A614FF0FF301A695A69586179
:1030B00000215A6959615A691A6A62F080521A628B
:1030C0001A6A02F080521A621A6A5A6A58625A6A76
:1030D00059625A6A1A6C42F080521A641A6E42F0AF
:1030E00080521A661A6E0B4A106840F480701060A5
:1030F000186F00F44070B0F5007F1EBF4FF48030B1
:1031000018671967536823F40073536000F054B9CB
:103110000038024000700040334B4FF080521A6478
:10312000324A4FF4404111601A6842F001021A60BD
:103130001A689107FCD59A6822F003029A602A4B1C
:103140009A6812F00C02FBD1196801F0F9011960BC
:103150009A601A6842F480321A601A689203FCD5A9
:103160005A6F42F001025A671F4B5A6F9007FCD505
:103170001F4A5A601A6842F080721A601B4A5368EC
:103180005904FCD5184B1A689201FCD5194A9A606B
:10319000194B1A68194B9A42194B21D1194A1168D7
:1031A000194A91421CD140F205121A60144A136860
:1031B00003F00F03052BFAD10B4B9A6842F0020281
:1031C0009A609A6802F00C02082AFAD15A6C42F40A
:1031D00080425A645A6E42F480425A665B6E70476F
:1031E00040F20572E1E700BF003802400070004085
:1031F0000854400700948838002004E0116400203F
:10320000003C024000ED00E041C20F41074A08B512
:10321000536903F00103536123B1054A13680BB1ED
:1032200050689847BDE80840FFF7D0BE003C014019
:10323000E02D0020074A08B5536903F002035361EB
:1032400023B1054A93680BB1D0689847BDE80840A0
:10325000FFF7BCBE003C0140E02D0020074A08B546
:10326000536903F00403536123B1054A13690BB199
:1032700050699847BDE80840FFF7A8BE003C0140F0
:10328000E02D0020074A08B5536903F00803536195
:1032900023B1054A93690BB1D0699847BDE808404E
:1032A000FFF794BE003C0140E02D0020074A08B51E
:1032B000536903F01003536123B1054A136A0BB13C
:1032C000506A9847BDE80840FFF780BE003C0140C7
:1032D000E02D0020164B10B55C6904F478725A6139
:1032E000A30604D5134A936A0BB1D06A98476006C7
:1032F00004D5104A136B0BB1506B9847210604D5C7
:103300000C4A936B0BB1D06B9847E20504D5094A80
:10331000136C0BB1506C9847A30504D5054A936C08
:103320000BB1D06C9847BDE81040FFF74FBE00BF0F
:10333000003C0140E02D0020194B10B55C6904F4FD
:103340007C425A61620504D5164A136D0BB1506D6B
:103350009847230504D5134A936D0BB1D06D984758
:10336000E00404D50F4A136E0BB1506E9847A104C8
:1033700004D50C4A936E0BB1D06E9847620404D505
:10338000084A136F0BB1506F9847230404D5054AC0
:10339000936F0BB1D06F9847BDE81040FFF716BE92
:1033A000003C0140E02D002008B5FFF75DFEBDE8C0
:1033B0000840FFF70BBE0000062108B50846FFF7DE
:1033C0001DFB06210720FFF719FB06210820FFF748
:1033D00015FB06210920FFF711FB06210A20FFF744
:1033E0000DFB06211720FFF709FB06212820FFF718
:1033F00005FBBDE8084007211C20FFF7FFBA0000CD
:1034000008B5FFF745FE00F00BF8FDF791FEFDF75C
:1034100069FDFFF7A5FDBDE80840FFF7CFBC000040
:103420000023054A19460133102BC2E9001102F1AD
:103430000802F8D1704700BFE02D0020034611F8C4
:10344000012B03F8012B002AF9D1704753544D3357
:1034500032463F3F3F0053544D33324634307800BC
:1034600053544D3332463432780053544D33324640
:103470003434365858000000012033000010410059
:1034800001105A000310590007103100000000001D
:103490004C340008130400005634000819040000DE
:1034A00060340008210400006A34000800000000B5
:1034B000610E00084D0E0008890E0008750E000808
:1034C000810E00086D0E0008590E0008450E000818
:1034D000950E000800000000010000000000000040
:1034E00063300000E0340008F023002000260020B4
:1034F0004172647550696C6F740025424F415244AB
:10350000252D424C002553455249414C25000000D1
:1035100002000000000000007D100008E910000813
:1035200040004000A02A0020B02A00200200000035
:103530000000000003000000000000002D11000842
:103540000000000010000000C02A00200000000061
:103550000100000000000000682D002001010200B1
:10356000E11B0008F11A00088D1B0008711B000800
:10357000430000007835000809024300020100C042
:1035800032090400000102020100052400100105B7
:10359000240100010424020205240600010705821B
:1035A000030800FF09040100020A000000070501EA
:1035B00002400000070581024000000012000000E8
:1035C000C4350008120110010200004009124157E1
:1035D00000020102030100000403090425424F41D7
:1035E00052442500574647303031003031323334B1
:1035F00035363738394142434445460000400000E3
:1036000000400000004000000040000000000100F9
:1036100000000200000002000000020000000200A2
:103620000000020000000200000002000000000094
:103630007112000829150008D51500084000400047
:10364000C82D0020C82D002001000000D82D00202A
:103650008000000040010000030000006D61696E01
:103660000069646C650000000000802A0000000012
:10367000AAAAAAAA00000024FFFF00000000000080
:1036800000A00A000000000000000000AAAAAAAAE8
:1036900000000000FFFF000000000000000000002C
:1036A0000000004000000000AAAAAAAA0000000032
:1036B000FF7F00000000000000000000000000008C
:1036C00000000000AAAAAAAA00000000FFFF000054
:1036D00000000000000000000000000000000000EA
:1036E000AAAAAAAA00000000FFFF00000000000034
:1036F000000000000000000000000000AAAAAAAA22
:1037000000000000FFFF00000000000000000000BB
:103710000000000000000000AAAAAAAA0000000001
:10372000FFFF00000000000000000000000000009B
:10373000000000000A00000000000000030000007C
:103740000000000000000000000000000000000079
:103750000000000000000000000000000000000069
:103760000000000000000000FE0700000000000054
:1037700000400F0000000000FF009600000000085D
:10378000009600000000080004000000D835000882
:103790000000000000000000000000000000000029
:1037A0000000000000000000FFFFFFFFFFFFFFFF21
:1037B000FFFFFFFFFFFFFFFFFFFFFFFFFFFFFFFF19
:1037C000FFFFFFFFFFFFFFFFFFFFFFFFFFFFFFFF09
:1037D000FFFFFFFFFFFFFFFFFFFFFFFFFFFFFFFFF9
:1037E000FFFFFFFFFFFFFFFFFFFFFFFFFFFFFFFFE9
:10C000000006002089D20008D5E8090831E80908AF
:10C010009DE8090831E8090869E809088BD2000899
:10C020008BD200088BD200088BD20008E9FD0B08E8
:10C030008BD200088BD200088BD200088BD200086C
:10C040008BD200088BD200088BD200088BD200085C
:10C050008BD200088BD2000805100C082D100C089C
:10C0600055100C087D100C08A5100C08A1BC0B087D
:10C07000C9BC0B08F5BC0B0821BD0B084DBD0B0856
:10C0800075BD0B08A1BD0B0825BC0B088BD20008A1
:10C090008BD200088BD200088BD20008CD100C0880
:10C0A00005120C0809120C081D120C0821120C08AC
:10C0B00025120C0839120C084D120C082DC30B0860
:10C0C000D5C40B088BD200088BD200088BD2000895
:10C0D0008BD20008A1110C08B5110C08C9110C086D
:10C0E00031110C088BD200088BD2000871120C0899
:10C0F00075120C0889120C088D120C08CDBD0B08A6
:10C100008BD200088BD2000861120C088BD2000879
:10C11000DD110C08F1110C088BD200088BD200083D
:10C12000F9BD0B0821BE0B084DBE0B0879BE0B08EC
:10C13000A5BE0B088BD200088BD200088BD200085A
:10C140008BD200088BD200088BD2000815050C0892
:10C15000CDBE0B08F9BE0B0825BF0B088BD200081B
:10C160008BD200088BD200088BD200088BD200083B
:10C170008BD200088BD200088BD200088BD200082B
:10C180008BD200088BD200088BD200088BD200081B
:10C190008BD200088BD200088BD200088BD200080B
:10C1A0008BD200088BD200088BD200088BD20008FB
:10C1B0008BD200088BD200088BD200088BD20008EB
:10C1C0008BD200088BD200088BD200088BD20008DB
:10C1D0008BD200088BD200088BD200088BD20008CB
:10C1E00071240108DDF50208D16F0408A5F90508DE
:10C1F000C9FF0508D56A060885B9060849C10608B9
:10C2000081C40608F9240708414A070809E107081C
:10C21000C1320808A9E1090805D90A0865450B08D3
:10C220007D6B0B08CD760B0845A40B080DAA0B08F7
:10C2300081F0004102E000BF83F0004330B54FEAD7
:10C2400041044FEA430594EA050F08BF90EA020F44
:10C250001FBF54EA000C55EA020C7FEA645C7FEAD7
:10C26000655C00F0E2804FEA5454D4EB5555B8BFFA
:10C270006D420CDD2C4480EA020281EA030382EA6B
:10C28000000083EA010180EA020281EA0303362DFD
:10C2900088BF30BD11F0004F4FEA01314FF4801CD0
:10C2A0004CEA113102D0404261EB410113F0004FE2
:10C2B0004FEA03334CEA133302D0524263EB430399
:10C2C00094EA050F00F0A780A4F10104D5F1200E37
:10C2D0000DDB02FA0EFC22FA05F2801841F1000192
:10C2E00003FA0EF2801843FA05F359410EE0A5F166
:10C2F00020050EF1200E012A03FA0EFC28BF4CF097
:10C30000020C43FA05F3C01851EBE37101F000454C
:10C3100007D54FF0000EDCF1000C7EEB00006EEB59
:10C320000101B1F5801F1BD3B1F5001F0CD34908E3
:10C330005FEA30004FEA3C0C04F101044FEA44523A
:10C3400012F5800F80F09A80BCF1004F08BF5FEAC1
:10C35000500C50F1000041EB045141EA050130BDA1
:10C360005FEA4C0C404141EB0101013C28BFB1F5B3
:10C37000801FE9D291F0000F04BF01460020B1FAFE
:10C3800081F308BF2033A3F10B03B3F120020CDAD1
:10C390000C3208DD02F1140CC2F10C0201FA0CF0AF
:10C3A00021FA02F10CE002F11402D8BFC2F1200C14
:10C3B00001FA02F120FA0CFCDCBF41EA0C019040CA
:10C3C000E41AA2BF01EB0451294330BD6FEA040413
:10C3D0001F3C1CDA0C340EDC04F11404C4F12002FE
:10C3E00020FA04F001FA02F340EA030021FA04F310
:10C3F00045EA030130BDC4F10C04C4F1200220FA67
:10C4000002F001FA04F340EA0300294630BD21FAA4
:10C4100004F0294630BD94F0000F83F4801306BF6A
:10C4200081F480110134013D4EE77FEA645C18BF5E
:10C430007FEA655C29D094EA050F08BF90EA020FF5
:10C4400005D054EA000C04BF1946104630BD91EAED
:10C45000030F1EBF0021002030BD5FEA545C05D1F0
:10C460004000494128BF41F0004130BD14F580042F
:10C470003CBF01F5801130BD01F0004545F0FE41A3
:10C4800041F470014FF0000030BD7FEA645C1ABFD8
:10C49000194610467FEA655C1CBF0B46024650EA0F
:10C4A000013406BF52EA033591EA030F41F400213B
:10C4B00030BD00BF90F0000F04BF0021704730B5C1
:10C4C0004FF4806404F132044FF000054FF0000196
:10C4D00050E700BF90F0000F04BF0021704730B557
:10C4E0004FF4806404F1320410F0004548BF40422C
:10C4F0004FF000013EE700BF42004FEAE2014FEA81
:10C5000031014FEA02701FBF12F07F4393F07F4F5B
:10C5100081F06051704732F07F4208BF704793F05E
:10C520007F4F04BF41F40021704730B54FF4607471
:10C5300001F0004521F000411CE700BF50EA010274
:10C5400008BF704730B54FF000050AE050EA01021D
:10C5500008BF704730B511F0004502D5404261EB8D
:10C5600041014FF4806404F132045FEA915C3FF4CE
:10C57000D8AE4FF003025FEADC0C18BF03325FEA6B
:10C58000DC0C18BF033202EBDC02C2F1200300FA1C
:10C5900003FC20FA02F001FA03FE40EA0E0021FA41
:10C5A00002F11444BDE600BF70B54FF0FF0C4CF42F
:10C5B000E06C1CEA11541DBF1CEA135594EA0C0FE1
:10C5C00095EA0C0F00F0DEF82C4481EA030621EA1C
:10C5D0004C5123EA4C5350EA013518BF52EA033557
:10C5E00041F4801143F4801338D0A0FB02CE4FF009
:10C5F0000005E1FB02E506F00042E0FB03E54FF039
:10C600000006E1FB03569CF0000F18BF4EF0010E30
:10C61000A4F1FF04B6F5007F64F5407404D25FEA2C
:10C620004E0E6D4146EB060642EAC62141EA5551DF
:10C630004FEAC52040EA5E504FEACE2EB4F1FD0C21
:10C6400088BFBCF5E06F1ED8BEF1004F08BF5FEA9F
:10C65000500E50F1000041EB045170BD06F0004651
:10C6600046EA010140EA020081EA0301B4EB5C04FE
:10C67000C2BFD4EB0C0541EA045170BD41F48011F6
:10C680004FF0000E013C00F3AB8014F1360FDEBF1B
:10C69000002001F0004170BDC4F10004203C35DAF7
:10C6A0000C341BDC04F11404C4F1200500FA05F37A
:10C6B00020FA04F001FA05F240EA020001F000421B
:10C6C00021F0004110EBD37021FA04F642EB060191
:10C6D0005EEA430E08BF20EAD37070BDC4F10C04BB
:10C6E000C4F1200500FA04F320FA05F001FA04F27F
:10C6F00040EA020001F0004110EBD37041F100016B
:10C700005EEA430E08BF20EAD37070BDC4F1200575
:10C7100000FA05F24EEA020E20FA04F301FA05F2DD
:10C7200043EA020321FA04F001F0004121FA04F285
:10C7300020EA020000EBD3705EEA430E08BF20EA55
:10C74000D37070BD94F0000F0FD101F0004640008F
:10C7500041EB010111F4801F08BF013CF7D041EA11
:10C76000060195F0000F18BF704703F00046520015
:10C7700043EB030313F4801F08BF013DF7D043EAE6
:10C780000603704794EA0C0F0CEA135518BF95EA9C
:10C790000C0F0CD050EA410618BF52EA4306D1D123
:10C7A00081EA030101F000414FF0000070BD50EA42
:10C7B000410606BF1046194652EA430619D094EACC
:10C7C0000C0F02D150EA013613D195EA0C0F05D1B6
:10C7D00052EA03361CBF104619460AD181EA03010A
:10C7E00001F0004141F0FE4141F470014FF00000C2
:10C7F00070BD41F0FE4141F4780170BD70B54FF05D
:10C80000FF0C4CF4E06C1CEA11541DBF1CEA1355DC
:10C8100094EA0C0F95EA0C0F00F0A7F8A4EB0504BE
:10C8200081EA030E52EA03354FEA013100F08880B5
:10C830004FEA03334FF0805545EA131343EA12637E
:10C840004FEA022245EA111545EA10654FEA002633
:10C850000EF000419D4208BF964244F1FD0404F5EC
:10C86000407402D25B084FEA3202B61A65EB030548
:10C870005B084FEA32024FF480104FF4002CB6EB05
:10C88000020E75EB030E22BFB61A754640EA0C0085
:10C890005B084FEA3202B6EB020E75EB030E22BFC5
:10C8A000B61A754640EA5C005B084FEA3202B6EB06
:10C8B000020E75EB030E22BFB61A754640EA9C00C5
:10C8C0005B084FEA3202B6EB020E75EB030E22BF95
:10C8D000B61A754640EADC0055EA060E18D04FEA53
:10C8E000051545EA16754FEA06164FEAC30343EAF3
:10C8F00052734FEAC2025FEA1C1CC0D111F4801FC0
:10C900000BD141EA00014FF000004FF0004CB6E7B8
:10C9100011F4801F04BF01430020B4F1FD0C88BF57
:10C92000BCF5E06F3FF6AFAEB5EB030C04BFB6EB62
:10C93000020C5FEA500C50F1000041EB045170BD55
:10C940000EF0004E4EEA113114EB5C04C2BFD4EB82
:10C950000C0541EA045170BD41F480114FF0000E06
:10C96000013C90E645EA060E8DE60CEA135594EA82
:10C970000C0F08BF95EA0C0F3FF43BAF94EA0C0F85
:10C980000AD150EA01347FF434AF95EA0C0F7FF4FA
:10C9900025AF104619462CE795EA0C0F06D152EA4E
:10C9A00003353FF4FDAE1046194622E750EA410632
:10C9B00018BF52EA43067FF4C5AE50EA41047FF443
:10C9C0000DAF52EA43057FF4EBAE12E74FF0FF3CA8
:10C9D00006E000BF4FF0010C02E000BF4FF0010C79
:10C9E0004DF804CD4FEA410C7FEA6C5C4FEA430CF2
:10C9F00018BF7FEA6C5C1BD001B050EA410C0CBF41
:10CA000052EA430C91EA030F02BF90EA020F0020A2
:10CA1000704710F1000F91EA030F58BF994208BF09
:10CA200090422CBFD8176FEAE37040F001007047C6
:10CA30004FEA410C7FEA6C5C02D150EA013C07D11D
:10CA40004FEA430C7FEA6C5CD6D152EA033CD3D068
:10CA50005DF8040B704700BF8446104662468C4662
:10CA60001946634600E000BF01B5FFF7B7FF002895
:10CA700048BF10F1000F01BD4DF808EDFFF7F4FFBE
:10CA80000CBF012000205DF808FB00BF4DF808ED49
:10CA9000FFF7EAFF34BF012000205DF808FB00BF6C
:10CAA0004DF808EDFFF7E0FF94BF012000205DF88E
:10CAB00008FB00BF4DF808EDFFF7CEFF94BF012043
:10CAC00000205DF808FB00BF4DF808EDFFF7C4FF3C
:10CAD00034BF012000205DF808FB00BF4FEA410C85
:10CAE0007FEA6C5C02D150EA013C0AD14FEA430C68
:10CAF0007FEA6C5C02D152EA033C02D14FF00000A5
:10CB000070474FF0010070474FEA410212F50012E2
:10CB100015D211D56FF47873B3EB625212D94FEA84
:10CB2000C12343F0004343EA505311F0004F23FA6E
:10CB300002F018BF404270474FF00000704750EAC3
:10CB4000013005D111F0004008BF6FF00040704780
:10CB50004FF00000704700BF4A0011D212F50012DA
:10CB600011D20DD56FF47873B3EB62520ED44FEA45
:10CB7000C12343F0004343EA505323FA02F07047C5
:10CB80004FF00000704750EA013002D14FF0FF3003
:10CB900070474FF0000070474FEA4102B2F1E043A6
:10CBA00024BFB3F5001CDCF1FE5C0DD901F0004C94
:10CBB0004FEAC0024CEA5070B2F1004F40EB8300E4
:10CBC00008BF20F00100704711F0804F21D113F110
:10CBD0003872BCBF01F00040704741F480114FEA49
:10CBE0005252C2F11802C2F1200C10FA0CF320FAD2
:10CBF00002F018BF40F001004FEAC1234FEAD323EF
:10CC000003FA0CFC40EA0C0023FA02F34FEA430358
:10CC1000CCE77FEA625307D150EA01331EBF4FF0E1
:10CC2000FE4040F44000704701F0004040F0FE40FC
:10CC300040F40000704700BF80F0004002E000BFF9
:10CC400081F0004142001FBF5FEA410392EA030FF7
:10CC50007FEA226C7FEA236C6AD04FEA1262D2EB41
:10CC60001363C1BFD218414048404140B8BF5B4246
:10CC7000192B88BF704710F0004F40F4000020F0DF
:10CC80007F4018BF404211F0004F41F4000121F0F5
:10CC90007F4118BF494292EA030F3FD0A2F101023F
:10CCA00041FA03FC10EB0C00C3F1200301FA03F17D
:10CCB00000F0004302D5494260EB4000B0F5000FA0
:10CCC00013D3B0F1807F06D340084FEA310102F15F
:10CCD0000102FE2A51D2B1F1004F40EBC25008BF11
:10CCE00020F0010040EA03007047490040EB0000DB
:10CCF000013A28BFB0F5000FEDD2B0FA80FCACF1DC
:10CD0000080CB2EB0C0200FA0CF0AABF00EBC25008
:10CD100052421843BCBFD0401843704792F0000FF6
:10CD200081F4000106BF80F400000132013BB5E749
:10CD30004FEA41037FEA226C18BF7FEA236C21D0BF
:10CD400092EA030F04D092F0000F08BF0846704724
:10CD500090EA010F1CBF0020704712F07F4F04D1F2
:10CD6000400028BF40F00040704712F100723CBF05
:10CD700000F50000704700F0004343F0FE4040F42F
:10CD8000000070477FEA226216BF08467FEA2363ED
:10CD90000146420206BF5FEA412390EA010F40F4D8
:10CDA000800070474FF0000304E000BF10F0004324
:10CDB00048BF40425FEA000C08BF704743F096430B
:10CDC00001464FF000001CE050EA010208BF704726
:10CDD0004FF000030AE000BF50EA010208BF7047AD
:10CDE00011F0004302D5404261EB41015FEA010CC2
:10CDF00002BF84460146002043F0B64308BFA3F1BA
:10CE00008053A3F50003BCFA8CF2083AA3EBC2539B
:10CE100010DB01FA02FC634400FA02FCC2F12002BA
:10CE2000BCF1004F20FA02F243EB020008BF20F0F1
:10CE30000100704702F1200201FA02FCC2F1200257
:10CE400050EA4C0021FA02F243EB020008BF20EA4C
:10CE5000DC7070477BB972B90029BEBF00204FF06B
:10CE6000004106E008BF00281CBF6FF000414FF0F2
:10CE7000FF3000F007BAADF1080C6DE904CE0029CF
:10CE800009DB002B1ADB00F095F8DDF804E0DDE9A2
:10CE9000022304B07047404261EB4101002B1BDBD1
:10CEA00000F088F8DDF804E0DDE9022304B0404238
:10CEB00061EB4101524263EB43037047524263EB23
:10CEC000430300F077F8DDF804E0DDE9022304B065
:10CED000404261EB41017047524263EB430300F073
:10CEE00069F8DDF804E0DDE9022304B0524263EBA7
:10CEF0004303704753B94AB9002908BF00281CBF33
:10CF00004FF0FF314FF0FF3000F0BCB9ADF1080C2D
:10CF10006DE904CE00F04EF8DDF804E0DDE902230F
:10CF200004B07047430803F05533C01A830803F078
:10CF3000333300F03330184400EB101000F00F30A2
:10CF400000EB002000EB0040000E704707EE900A57
:10CF5000F5EEC07AF1EE10FA01D400F00BB8F1EE64
:10CF6000677A08B517EE900A00F004F8404261EBCA
:10CF7000410108BDD0B5FFF7BFFA0C4B00220646B1
:10CF80000F46FFF711FBFFF7E7FD0446FFF792FAA4
:10CF9000074B0022FFF708FB02460B463046394696
:10CFA000FFF74AF9FFF7D8FD2146D0BD0000F03D5C
:10CFB0000000F0412DE9F047089D04468E46002B05
:10CFC0004DD18A42944669D9B2FA82F252B101FA3D
:10CFD00002F3C2F1200120FA01F10CFA02FC41EA4D
:10CFE000030E94404FEA1C48210CBEFBF8F61FFAD2
:10CFF0008CF708FB16E341EA034306FB07F199426D
:10D000000AD91CEB030306F1FF3080F01F8199421F
:10D0100040F21C81023E63445B1AA4B2B3FBF8F0F9
:10D0200008FB103344EA034400FB07F7A7420AD980
:10D030001CEB040400F1FF3380F00A81A74240F2A8
:10D0400007816444023840EA0640E41B00261DB113
:10D05000D4400023C5E900433146BDE8F0878B4248
:10D0600009D9002D00F0EF800026C5E90001304607
:10D070003146BDE8F087B3FA83F6002E4AD18B42E1
:10D0800002D3824200F2F980841A61EB030301208B
:10D090009E46002DE0D0C5E9004EDDE702B9FFDE77
:10D0A000B2FA82F2002A40F09280A1EB0C014FEA22
:10D0B0001C471FFA8CFE0126200CB1FBF7F307FB7F
:10D0C000131140EA01410EFB03F0884208D91CEB22
:10D0D000010103F1FF3802D2884200F2CB804346BF
:10D0E000091AA4B2B1FBF7F007FB101144EA01449E
:10D0F0000EFB00FEA64508D91CEB040400F1FF312D
:10D1000002D2A64500F2BB800846A4EB0E0440EA1A
:10D1100003409CE7C6F12007B34022FA07FC4CEA23
:10D12000030C20FA07F401FA06F31C43F9404FEA16
:10D130001C4900FA06F3B1FBF9F8200C1FFA8CFE2B
:10D1400009FB181140EA014108FB0EF0884202FA7F
:10D1500006F20BD91CEB010108F1FF3A80F0888040
:10D16000884240F28580A8F102086144091AA4B2FD
:10D17000B1FBF9F009FB101144EA014100FB0EFE7E
:10D180008E4508D91CEB010100F1FF346CD28E45AD
:10D190006AD90238614440EA0840A0FB0294A1EB3E
:10D1A0000E01A142C846A64656D353D05DB1B3EB9B
:10D1B000080261EB0E0101FA07F722FA06F3F140CB
:10D1C0001F43C5E9007100263146BDE8F087C2F172
:10D1D0002003D8400CFA02FC21FA03F391400143EA
:10D1E0004FEA1C471FFA8CFEB3FBF7F007FB103623
:10D1F0000B0C43EA064300FB0EF69E4204FA02F4CF
:10D2000008D91CEB030300F1FF382FD29E422DD921
:10D21000023863449B1B89B2B3FBF7F607FB163356
:10D2200041EA034106FB0EF38B4208D91CEB0101D6
:10D2300006F1FF3816D28B4214D9023E6144C91A56
:10D2400046EA004638E72E46284605E70646E3E666
:10D250001846F8E64B45A9D2B9EB020864EB0C0E70
:10D260000138A3E74646EAE7204694E74046D1E77F
:10D27000D0467BE7023B614432E7304609E764442D
:10D28000023842E7704700BF02E000F000F8FEE716
:10D2900072B6374880F30888364880F309883648E4
:10D2A0003649086040F20000CCF200004EF63471BE
:10D2B000CEF200010860BFF34F8FBFF36F8F40F2D3
:10D2C0000000C0F2F0004EF68851CEF20001086076
:10D2D000BFF34F8FBFF36F8F4FF00000E1EE100AE6
:10D2E0004EF63C71CEF200010860062080F31488EF
:10D2F000BFF36F8FB2F0D6FDB3F020FD4FF0553085
:10D300001F491B4A91423CBF41F8040BFAE71D49F3
:10D31000184A91423CBF41F8040BFAE71A491B4AEC
:10D320001B4B9A423EBF51F8040B42F8040BF8E73E
:10D3300000201849184A91423CBF41F8040BFAE713
:10D34000B2F0B4FDB3F04EFD144C154DAC4203DA0F
:10D3500054F8041B8847F9E701F06CFB114C124D9F
:10D36000AC4203DA54F8041B8847F9E7B2F09CBDDD
:10D37000000600200022002000C0000808ED00E0A8
:10D38000000000200006002020CF0E080022002010
:10D390005C2B0020602B002040530120E0C10008DE
:10D3A00030C2000830C2000830C200082DE9F04F3A
:10D3B0002DED108AC1F80CD0C3689D46BDEC108AD3
:10D3C000BDE8F08F002383F311882846A047002092
:10D3D000B1F060FDFEE7B1F0CDFB00DFFEE700003D
:10D3E00001F0FF01102A2BDB10F0070F08D010F816
:10D3F000013B013A8B422DD010F0070F42B3F6D11A
:10D40000F0B441EA012141EA014122F007047FF032
:10D4100000070023F0E80256083C85EA010586EA89
:10D42000010685FA47F5A3FA87F586FA47F6A5FAC5
:10D4300087F68EB9EED1F0BC01F0FF0102F00702D1
:10D4400032B110F8013B013A83EA010313B1F8D17C
:10D450000020704701387047002D06BF354603385D
:10D46000073815F0010F07D1013015F4807F02BF96
:10D47000013015F4C03F0130F0BC0138704700BFE7
:10D4800010F8012B11F8013B012A28BF9A42F7D06E
:10D49000D01A7047034613F8012B002AFBD1181A43
:10D4A0000138704738B50022002304460D46FFF7C7
:10D4B000EDFA28B920462946BDE8384000F00AB800
:10D4C000204605F1004100F005F8404261EB4101C2
:10D4D00038BD00BFD0B50C4B002206460F46FFF703
:10D4E00063F8FFF739FB0446FEF7E4FF074B002221
:10D4F000FFF75AF802460B4630463946FEF79CFEC7
:10D50000FFF72AFB2146D0BD0000F03D0000F041AE
:10D51000036800221B68184710B503685B6804465F
:10D52000984708B194F84D0010BD00002DE9F04176
:10D53000674B03F5A04490B094F9A42A06460F4621
:10D54000002A00F0C28094F8EC5A35B9614A7FF0A5
:10D5500023FE284610B0BDE8F081B3F9A4201AB923
:10D56000B3F8A220A3F8A420B3F8A430632B05D805
:10D57000594A394630467FF00FFE002500212E2201
:10D5800004A80391B6F044FCD4F8040A036803AA83
:10D590001B6832219847804630B9504A03AB394660
:10D5A00030467FF0F9FD4546B4F8E039A3F57A73CB
:10D5B0009BB241F65832934206D9494B3A46202154
:10D5C00030467FF0E1FB002594F9143C002B6BDD25
:10D5D00094F9CC3B002B5BDD424B3A462021304690
:10D5E0007FF0D2FB00254049D4F8100A322303AA69
:10D5F0008AF094FD804640B903AB00933A463B4B1A
:10D60000202130467FF0C0FB45463949D4F80C0A4A
:10D61000322303AA87F0B4FD804640B903AB0093E0
:10D620003A46324B202130467FF0AEFB4546202162
:10D6300030467FF0A1FBC8B104F52663D3ED007A34
:10D640009FED2C7AF0EEE77AF4EEC77AF1EE10FA5D
:10D650000CD594F9143C002B02DD94F8783C2BB9DE
:10D66000254A394630467FF097FD002594F9143C51
:10D67000002B7FF76EAF94F9D13A002B3FF469AFDE
:10D680001E4B3A46202130467FF07EFB002560E7A6
:10D6900094F8788CB8F1000F06D1194B3A46202146
:10D6A00030467FF071FB454694F9CC3B002B9ADD68
:10D6B00094F8FD8BB8F1000F95D1124B3A4620211A
:10D6C00030467FF061FB45468DE7012541E700BF0D
:10D6D000702B002060820C0882820C08A9820C0842
:10D6E000B4820C08C6820C0837830C083B830C08F4
:10D6F0004D830C080000003451830C086B830C0828
:10D70000EC820C0812830C0838B504467FF018FB35
:10D71000114B93F8B01B114B1D68EB6A1A68002976
:10D7200008BF01461268184690475AF0B1FFEB6AED
:10D7300093F89C105AF014F994F837305BB191F0DB
:10D74000FFF8EB6AD3F8A030C01AB0F5FA6F24BF27
:10D75000002384F8373038BD707B00206C2B00200C
:10D7600008B5FFF7D1FF054B05481B68DB6A93F846
:10D770009C10BDE8084010F0BBBE00BF6C2B002021
:10D780004885002070B50E46054665F0D5F865F071
:10D7900097F810B90124204670BD0A4B93F9BA33AB
:10D7A000012BF7D165F0C8F8437A002BF2D165F070
:10D7B000C3F8847A002CEDD1034A314628467FF025
:10D7C000EBFCE8E7704B002084830C087FF06EBA16
:10D7D0002DE9F0472DED028BC47F90B006460F4631
:10D7E0008CB990F90430002B00F00381824B1D6846
:10D7F000A86A03685B6B9847044650B97F4A39466C
:10D8000030467FF0C9FC204610B0BDEC028BBDE86D
:10D81000F087B3684BB933685B6B3946304610B05C
:10D82000BDEC028BBDE8F0471847E86AFFF774FECD
:10D8300004460028E7D13946304680F037FBDFF850
:10D84000F0810546394630467FF0CEFC98EDF37AFC
:10D85000D8EDF27AB4EEE77A2840F1EE10FAC5B2CC
:10D8600009D598F9C433032B05D0654A39463046AB
:10D870007FF092FC2546D8EDDB7AB0EE088AF4EE14
:10D88000C87AF1EE10FA0BD517EE900AFEF734FEC7
:10D890005C4ACDE90001394630467FF07DFC002529
:10D8A000D8EDDC7AF4EEC87AF1EE10FA0BD517EE6B
:10D8B000900AFEF721FE544ACDE900013946304670
:10D8C0007FF06AFC0025D8EDDD7AB8EE087AF4EE38
:10D8D000C77AF1EE10FA0BDD17EE900AFEF70CFE98
:10D8E0004A4ACDE90001394630467FF055FC002513
:10D8F000B8F95833042B07DC052200923946444A14
:10D9000030467FF049FC0025D8F8D80D65F070F856
:10D9100080B198F9BA336BB1D8F8D83DB8F9BC23C7
:10D92000B3F90E309A4205DA3A4A394630467FF06A
:10D9300033FC002539463046FFF724FFDFF8F4A01A
:10D94000814639463046FFF7F1FD9AF8DD30002B6D
:10D9500048D109EA050500EA05042F484FF4806123
:10D9600001F04AF878B1D8F8D83DB3F90C30A3F2F9
:10D97000E24292B2B2F5FA7F05D9284A39463046DA
:10D980007FF00AFC00249AF8303753B1244838F06D
:10D990009FFB054628B9234A394630467FF0FCFBF9
:10D9A0002C4600212E2204A80DF10C080391B6F09C
:10D9B0002FFADAF8C8004246322109F09DFA0546EE
:10D9C00000287FF420AFDAF8C80003689B68984706
:10D9D000154ACDF800800346394630467FF0DCFB1F
:10D9E0002C4610E7114A394630467FF0D5FB00241B
:10D9F000B3E7012407E700BF6C2B002094830C08D9
:10DA0000AB830C08CE830C08EE830C0810840C0842
:10DA100032840C0851840C08702B00208C840C0874
:10DA200098820020B4840C0828520D0877840C08D2
:10DA3000704B0020707B002070B505460E46FFF746
:10DA4000A1FE31460446284680F0E8F82040C0B2E6
:10DA500070BD0000F0B591B005460E467FF07AFC2F
:10DA60000446D8B1102128467FF086F9B0B10021D4
:10DA70002E2204A803AF0391B6F0CAF91BF066FC8E
:10DA800032233A4601211AF021FF044630B9054BF2
:10DA900000973246102128467FF076F9204611B0D3
:10DAA000F0BD00BFC8840C0870B505460E46B1B97C
:10DAB00090F910408CB1164813F05EFCDFED157A3A
:10DAC000B0EEC00AB4EEE70AF1EE10FA07D4124A3B
:10DAD000012128467FF060FB3446204670BDAB68CC
:10DAE0009BB10E4B1B68D86AFFF716FD044630B198
:10DAF00063F076FC0A4A04215CF0EAFDEDE731466A
:10DB00002846BDE870407FF0F1BE0124E5E700BF84
:10DB1000702B002000000034D4840C086C2B0020F3
:10DB2000E6840C0838B5044680F07AFA0546A8B1B8
:10DB30000B4806F0DFF838B10A490B481BF01EF815
:10DB400010B1074800F02AFF2046FFF709FE012325
:10DB5000064984F83730204680F078F9284638BDE9
:10DB6000702B002080840020C83F002008850C080E
:10DB7000F8B506460D461746C2B1232901D0012942
:10DB800014D8234808F090FC044668B100242046CD
:10DB9000F8BD96F91030022B08D063F021FC1D4A25
:10DBA00006215CF095FDF2E7002DF2D03A462946B9
:10DBB000304680F0E1FA04460028E7D0164DD5F84B
:10DBC000C820A5F5EC739A4203D005F5E56038F05E
:10DBD000B5FED5F8C80003689B6B9847D5F8283A7E
:10DBE00085F80007012B07D164F0A6FE542165F0EB
:10DBF00067FE08B9C5F8280A3046FFF7B1FD4FF0B7
:10DC0000FF330649C5F80031304680F01FF9BEE702
:10DC1000702B002018850C08707B002030850C08C4
:10DC20002DE9F04F2DED028BDFF8449191B00746BE
:10DC300088467FF04DF999F98F530446CDB9454890
:10DC4000BD2138F011FE38B1434B42464FF48041BC
:10DC500038467FF099F82C463E48BC2138F004FE47
:10DC600038B13E4B42464FF4804138467FF08CF845
:10DC700000243B4E96F8EC3A002B64D01C22002185
:10DC800002A8B6F85CA7DFED378AB6F0C1F804A8A1
:10DC900021F0AAF806F5E56B0125A6F5A046554545
:10DCA00051D20BA821F0A0F809AA2946584636F00F
:10DCB00097FA002847D0BDF82610304607F018FD27
:10DCC00080B3BDF80A30102B2CD104A90BA821F089
:10DCD000BBFB09F56F63B0EE408A93ED000A224862
:10DCE000B4EEE80AF1EE10FAB8BF99EDD70A20EECB
:10DCF000000A0EF029FDF6EE087A60EE277AB4EEFF
:10DD0000E78AF1EE10FA0DD517EE900AFEF7F4FB54
:10DD1000164BCDE9000142464FF4804138467FF072
:10DD200033F800240DF1240CBCE80F000DF1080EAF
:10DD3000AEE80F009CE80700AEE8030001358EF85E
:10DD40000020ADB2ABE7204611B0BDEC028BBDE8C0
:10DD5000F08F00BF9882002044850C0870850C0865
:10DD6000707B00200000003448850020A3850C084B
:10DD7000704B002000207047014800F08FBD00BFAD
:10DD8000702B002003685B681847000068F016B825
:10DD900064F020BD2FF012BF59F048BF08F0CCBC92
:10DDA0000DF0FAB814F02CBD03F0A2BA57F05EBE25
:10DDB0001FF030BA67F0A8BB14F086BD13F05ABB51
:10DDC0001EF0AEBD69F07ABD64F01EBA62F0D8BB39
:10DDD00007F06EBE05F0C4B90CF0E8BB0DF040B81A
:10DDE00014F04EBB14F01CBE13F078B914F084BCD0
:10DDF00001F07ABB00F2545022F08EB808F0E6B978
:10DE000090F8C432B02202FB030390F8082393F881
:10DE1000A13012B1012B28BF012318467047000022
:10DE200090F814310BB190F841311846704700005A
:10DE3000034808602921117008221A60704700BF4A
:10DE4000D4880C08F8B5044604F5A25600F5B34092
:10DE500010301836FFF758FC002130461BF0E8F967
:10DE60008021204615F046F818B131F02BFD2FF037
:10DE7000F7FA04F50055D5EDDB7A9FED2F7A67EEC2
:10DE8000877A05F6EC57FDEEE77A04F5B84017EE11
:10DE9000903AC5F8E83DD5F874333B60103015F082
:10DEA0002DFAD8B9D5F8E83D07EE903A04F5A2531B
:10DEB00093ED997AF8EEE77A67EE877AFDEEE77AE6
:10DEC00017EE902AC5F8E82DD3ED987A97ED007AF1
:10DED000F0EEE77A67EE877AC7ED007A04F5BC5179
:10DEE000103106F5457035F0F9FB04F5AD4594EDBC
:10DEF000467AD5ED007AE7EE007AC5ED007AB0EE0D
:10DF0000670A32F04DFA04F5B34085ED000A583047
:10DF10000DF02AFD04F5B3400021643084F06CF864
:10DF20004FF40011204614F0E5FF20B13046BDE863
:10DF3000F84019F09DBAF8BD0000C842FFF782BF53
:10DF4000F8B500F5A0470546D7F8C80003689B6BF5
:10DF5000984705F5B34458340646204610F08CFA2D
:10DF600097F8BF36002818BF002623B91EB105F563
:10DF70003A5083F0A5FF20460FF01EFF18B9204647
:10DF8000FFF74EFF20B12046BDE8F84010F0BCBCC2
:10DF9000F8BD0000FFF7D4BF38B54FF48011054637
:10DFA00014F0A8FF044620B90121284614F0A2FF6E
:10DFB00004460221284614F09DFF50B114B92846AA
:10DFC00003F0BAF805F5A2501830BDE8384019F052
:10DFD0004DB9002CF6D138BDFFF7DEBF38B54FF490
:10DFE0008011044614F086FF01210546204614F0F6
:10DFF00081FF18B115B9204603F09EF81021204684
:10E0000014F078FF60B1204603F08AF94FF48001E4
:10E01000204614F06FFF18B931F054FC2FF01CFBB0
:10E020002021204614F066FF28B1204603F0EEF9C7
:10E03000204603F009FB4FF40051204614F05AFF2C
:10E0400010B1204603F0E6FA8021204614F052FF7A
:10E0500028B131F037FCBDE838402FF025BA38BD83
:10E06000FFF7BCBF10B5044622F046F890F9213006
:10E070008BB190F8403373B194F978355BB1064BAE
:10E080001B68DB6A93F89C302BB904F25450BDE84E
:10E09000104021F059BD10BD6C2B0020FFF7E2BFEE
:10E0A0002DE9F843424B1B68DB6A93F89C30044629
:10E0B000002B7AD000F5805898F86137002B74D087
:10E0C00008F0F2F9002870D004F5025604F5005566
:10E0D000183695F8E611304618F06CFC002864D02C
:10E0E00004F590773846FFF78BFE02285DD994F847
:10E0F000E4234FF0B00909FB024292ED777AF1EE8A
:10E10000007AB4EEE77AF1EE10FA4ED495F8E61103
:10E11000304618F0FFFEB5F9583307EE903AB8EEE6
:10E12000E77AB4EEC07AF1EE10FA0CDD94F8E4333D
:10E1300009FB0343F8EE677A93ED777AF4EEC77A3A
:10E14000F1EE10FA31DCD8F85036D5F8E82D002B76
:10E15000B8BF5B42934228DC08F25463D3ED007AE7
:10E16000D5EDDC6A9FED136AF8EEE77A66EE866A13
:10E17000F4EEE67AF1EE10FA17DC05F6EC5393EDC7
:10E18000007A27EE067AF4EEC77AF1EE10FA0CD494
:10E1900094F8E413B5F95A23B02303FB0171304618
:10E1A000D431BDE8F84318F083BABDE8F88300BF66
:10E1B0006C2B00200000C842FFF772BF2DE9F04130
:10E1C00090F8E4332C4F00EB03133E68D3F89481AE
:10E1D00000F5907504462846FFF712FE464512D01A
:10E1E000022812D904F5A046C7F8008096F8F83046
:10E1F000012B13D815D1D6F81839E3B9D6F81C3944
:10E20000CBB905230BE0022810D804F5A04393F8FE
:10E21000F8205AB1052283F8F82007E0013B86F880
:10E22000F83004F5C45014301CF044FA2046BDE820
:10E23000F0410CF095BB114B1B68D86A03685B6812
:10E24000984707460028ECD194F8E413B02303FB69
:10E250000151AC31204605F0BFFDD6F8FC380FCB9C
:10E2600004F5B24506F5126C85E80F008CE80F0046
:10E2700086F8F870D5E700BF602B00206C2B0020DB
:10E28000FFF79CBFF8B500F5A047044697F8EC3AB5
:10E2900000F58056BBB100F5B840103015F034FBE6
:10E2A00018B1012386F86137F8BD04F5B345583538
:10E2B00028460FF081FD08B10023F3E72846FFF759
:10E2C000AFFD0028F8D197F8BF36002BF4D1D7F86E
:10E2D0000437042BE5D104F5B04040308DF002F84E
:10E2E00086F86107E0E7000010B500F5A04400F5EE
:10E2F0009C43D4F8C82028339A4208D000F59F43A5
:10E3000030339A421CBF4FF0FF33C4F8783604F51F
:10E31000CD63074A1A6004F26C63064A1A60FFF77D
:10E32000B1FFD4F8C8000368BDE810401B69184766
:10E330000000C8420000C8C2FFF7D6BFF7B500F51D
:10E34000A0470446D7F804378B420D4624D00B1F54
:10E3500000F5B046594206F1400659413046019158
:10E360008CF0B0FE019930468CF0ACFE072D0BD13D
:10E3700004F55650D7F888266423052192FBF3F361
:10E380001030064A5CF0A4F92046C7F8045703B0E1
:10E39000BDE8F04003F0A2B803B0F0BD34860C082D
:10E3A00070B500F5A0450446D5F8C80003689B6B1E
:10E3B0009847A8B195F8003793B9D5F8C82004F567
:10E3C0009C4328339A424CD104F5B3465836304624
:10E3D0000EF018FF60B995F8B8367BB9012108E056
:10E3E00004F5B345583528460FF0E6FC00283ED02A
:10E3F00002212046BDE87040FFF7A0BFB5F86637A0
:10E40000152B27D195F8441811F0010120D1D5F82A
:10E410000437072B1CD095F9BA380BB90421E8E76B
:10E42000204612F0A9FFDFED137AB4EEE70AF1EE11
:10E4300010FAF3DB04F5B04040308CF093FE002876
:10E44000ECD004F556500C4A062110305CF040F92F
:10E450000721CEE73046FFF7E3FC0028C8D10321AF
:10E46000C7E704F59F4330339A42F8D170BD284680
:10E47000F1E700BF0000B44258860C0838B52F4CB5
:10E48000D4F8C820A4F5EC739A422DED028B054612
:10E49000B0EE408A03D00020BDEC028B38BD04F6FC
:10E4A000D8100EF0AFFE40B1BDEC028B05F5B340C5
:10E4B0005830BDE838400FF0ADBFD4F80437042B16
:10E4C00032D194F8F93033B11D49A1F5F47038F028
:10E4D000ADFC0028E0D194F8EC3A4BB119480EF0AD
:10E4E00091FE0028D7D117480EF04CFE0028D2D15B
:10E4F0009FED157AF0EEC87AF4EEC77AF1EE10FAD5
:10E5000009D49FED120A28EE008ABDEEC88A18EEE3
:10E51000103AC4F888360E488CF024FE0028BAD091
:10E52000002384F8BB36B7E7B4F86617A4F5A0401B
:10E5300007F0DEF80028C4D1ADE700BF707B0020F3
:10E540008084002048850020000000340000C8427C
:10E55000B083002010B52DED028B00F5A0430446DA
:10E56000D3F80427042A0BD105F08CF82046B0EE2E
:10E57000408A05F0F9F838EE400ABDEC028B10BD78
:10E5800003F5146393ED000AF7E700002DE9F0416D
:10E590002DED028B00F586658AB0044628461DF0F5
:10E5A0008BFA04F5A250002307A9183007930893AB
:10E5B00009931AF0C9FC002800F08B809DED090A30
:10E5C000DFED5A7A04F5A04505F5D36393ED007AA3
:10E5D00020EE270ADFED567AA7EE270A04F5B040B1
:10E5E000203083ED000A69F0BDFA2046FFF7D8FE1F
:10E5F000D5F8C80003689B6B9847064604F5B340FE
:10E6000058300FF039FF95F8BF36002818BF0026A4
:10E61000002B59D1002E57D095F80037002B53D13D
:10E62000D5F80437042B6BD09FED428A204605F0C5
:10E63000BDF8D5F8C820C5F83C0D04F59C4354330B
:10E640009A4204F500571AD195F88839BBB9B7F941
:10E65000B43D002B04DC384AD2F8942DD2060ED5F6
:10E66000D5F8FC18D5F8042949680A33521A6421F0
:10E670004B438242ACBF9B181B18C5F83C3DD5F8F4
:10E680003C1DD5F80437D5F8FC20059120460492AE
:10E69000039316F03BF9B5F90A8106462046FFF7C9
:10E6A00059FFCDE9006805F5E465F0EE400ADDE9C3
:10E6B0000332D7EDFD1A95ED001A0599B0EE480A20
:10E6C00004F53A5083F0A0F80AB0BDEC028BBDE827
:10E6D000F08104F59070FFF793FB02280AD994F8B3
:10E6E000E433B02202FB034393F8102212B193EDFE
:10E6F0007F0A65E728461DF079F8B1EE400A5FE72A
:10E7000004F5B24604F5B247103620373A4604F510
:10E71000B241304620F004FE002885D0394630460C
:10E7200020F092FEB0EE408A80E700BFCDCC4C3E98
:10E73000CDCC4C3F00000000704B0020FFF726BFFF
:10E74000F8B500F5A04600F59D43D6F8C82048333B
:10E750009A420F4621D000F5B344583420460FF0BA
:10E760002BFB054698B120460DF0B8FF60B1D6F8F6
:10E77000140A03689B689847DFED097A20EE270AA0
:10E7800087ED000A2846F8BD9FED060AF8E706F572
:10E79000D466012533683B60F4E70025F2E700BF4B
:10E7A0000AD7233C000000002DE9F04100F5A04805
:10E7B00000F59D43D8F8C82048339A4204460E46D7
:10E7C0002FD000F5B347583738460FF0F5FA054615
:10E7D000A0B138460DF082FF68B1D8F8140A03687A
:10E7E000DB68984707EE900AF8EEE77AC6ED007A04
:10E7F0002846BDE8F081DFED0C7AF7E704F54054D8
:10E800000125D4F8AC0703681B69984707EE900A06
:10E810009FED067AF8EEE77A67EE877AC6ED007A22
:10E82000E6E70025E4E700BF000000000AD7233C2C
:10E830002DE9F04100F5A04800F59D43D8F8C82027
:10E8400048339A4204460E4623D000F5B347583762
:10E8500038460FF0B1FA054680B138460DF03EFF5C
:10E8600048B1D8F8143A186988F0C2FB86ED000A5E
:10E870002846BDE8F0819FED080AF7E704F540540B
:10E880000125D4F8AC0703685B69984786ED000A58
:10E89000EEE70025ECE700BF0000000030B50546BC
:10E8A0000FC985B06C4684E80F0040F279322146EA
:10E8B000284605F02BF90C4BA3F5BA72D3F8C830F3
:10E8C00093420ED19DF8001011F0040102D12046B0
:10E8D00020F022FB0548214605F0CAF9012005B0C9
:10E8E00030BD0020FBE700BF707B0020702B0020B4
:10E8F00010B5044606480FF099F840B904F5A04455
:10E90000D4F8C8000368BDE810409B6C184710BDE0
:10E910004885002010B5044606480EF0DBFC40B9DF
:10E9200004F5A044D4F8C8000368BDE81040DB6CCF
:10E93000184710BD4885002070B5044600F5B34067
:10E9400058300E4615460EF029F850B104F5A04493
:10E95000D4F88C3C9B682B60D4F88C3C5B683360AB
:10E9600070BD04F5A2531833D3F808222A60D3F8F7
:10E970000432336004F50054D4F8943D9B05EFD481
:10E98000D4EDFD6AD5ED007A9FED037AE6EEC77A05
:10E99000C5ED007AE4E700BF35FA8E3C70B50D4E48
:10E9A000054631460C481AF0FBF905F5A04406F17E
:10E9B000300184F8F90005F5A25004F5146418300C
:10E9C0001AF086F8D4ED007AF1EE677AC4ED007A99
:10E9D00070BD00BF80840020C83F002010B50446F1
:10E9E00000F5907029F00AFF2046BDE81040FFF7BF
:10E9F000D5BF0000FFF7F2BF00F50050D0F8943DFE
:10EA0000194214BF012000207047000010B500F526
:10EA1000A0430446D3F8C80003689B6D984701469D
:10EA200004F5A0400830BDE810408EF009BE00009B
:10EA3000FFF7ECBF38B5054B1C6823680A461D6814
:10EA4000034B01462046A847002038BD6C2B002010
:10EA5000702B002070B52DED028B0446036804F581
:10EA600000559B6D9847D5F8943D1B0618D5B5F910
:10EA70005833B5F95A13CA1A0B4402EBD27203EB9E
:10EA8000D37352105B1000EE902A00EE103A04F59A
:10EA9000A250F8EEE00AB8EEC00A183019F09EFD58
:10EAA0005A4BB5F88A231A7004F5B34565F0C2FFD6
:10EAB000103565F051FC00212846FEF789FE544EC2
:10EAC0000123B0712846F3717EF03AF928B928463F
:10EAD0007FF0D0F9B0FA80F04009307128467EF01E
:10EAE0002FF904F5A045D8B994F8E43304EB0313E7
:10EAF00041F28832D3F89461D5F88C39F31A9342F5
:10EB00000ED904F59070FFF77BF9022808D9C5F8F3
:10EB10008C69204605F0EEF805F5046300221A60C2
:10EB2000B4F9A4301BB9B4F8A230A4F8A430B4F8F6
:10EB3000A430DFED388A07EE903AF8EEE77AB7EEC8
:10EB4000008A88EE270AD4ED2B7AF0EEE77AF4EE0D
:10EB5000E87AF1EE10FA09D5B4F9A23007EE903A4E
:10EB6000F8EEE77A88EE277A84ED2B7AD4ED2B0A3B
:10EB700031F018FB70BB58F015F940F27D124FF4DC
:10EB8000801158F0C7F857F027F856F08FFC95F829
:10EB9000EC3AB0EE408A23B1D5F80C0A03681B6F3B
:10EBA000984704F54450B0EE480A3C3076F0C2F87D
:10EBB00004F54A50B0EE480A183076F0BBF8B0EED3
:10EBC000480ABDEC028B04F54F500C30BDE8704094
:10EBD00076F0B0B8D4ED2B7A94ED460AF0EEE77AF1
:10EBE000F4EEE87AF1EE10FA09D5B4F9A23007EEA6
:10EBF000903AF8EEE77A88EE277A84ED2B7AD4ED16
:10EC00002B0A31F0CFFA0028B5D0BCE771230020E1
:10EC10005D89002000000034FFF71CBF70B500F5CF
:10EC2000A046044696F9B838002B28DD07F03CFCD6
:10EC300028BB04F5B345103528467FF01BF9F0B129
:10EC400028467EF07DF8D0B18FF07AFED6F8A8364F
:10EC5000C01A96F9B8384FF47A72534398420ED3DB
:10EC600001221C212846FEF783FF40B104F55650CF
:10EC7000034ABDE87040062110305BF029BD70BD2D
:10EC800078860C0800B52DED028B9FED0B8AD0ED38
:10EC90004E7A67EE887A83B0C0ED4E7A38300190B4
:10ECA00076F0A6F8019820EE080A03B0BDEC028BBE
:10ECB0005DF804EB76F0B4B952B87E3F00B52DEDA7
:10ECC000028B9FED0B8AD0ED4F7A67EE887A83B086
:10ECD000C0ED4F7A3C30019076F08AF8019820EE32
:10ECE000080A03B0BDEC028B5DF804EB76F098B92E
:10ECF00052B87E3F70B52DED048B044682B000F50E
:10ED0000A25001A918301AF0F1F8002800F0B780DD
:10ED100004F5A04606F5D26595ED007ADDED017AA1
:10ED2000B4EEE77AF1EE10FA07D504F5B3401030EF
:10ED30007EF010F808B1019B2B6004F5005595EDAD
:10ED4000EB7AB5F95833DFED5F6A052BB8BF0523C1
:10ED500007EE903AB5F95A33F8EEE78A07EE903AA3
:10ED6000F8EEE77AB6EE009A77EEA77A1820C7EEAB
:10ED7000270ADFED557A68EEA77AF4EE490A87EEA6
:10ED8000271AF0EE007AF1EE10FAB4EE671AC8BF57
:10ED9000F0EE490AF1EE10FA48BFB0EE671ADDED69
:10EDA000017AF4EEE67AF1EE10FACCBF87EE270A8C
:10EDB000B0EE410A31F008FB04F5B3405830B0EE34
:10EDC000408A0EF0F9FF28B996F8EC3AD3B396F8DA
:10EDD000193BBBB304F5B34010307DF0BBFF88B3E3
:10EDE00028EE892A9DED011AB4EEC21AF1EE10FA4E
:10EDF00028D5D5EDEB0ADFED351A9FED350AC0EECB
:10EE0000820A31F013FA04F544500430B4EE408A1B
:10EE1000F0EE408AF1EE10FA48BFF0EE488AFFF7B4
:10EE200031FF04F549501C3004F55454FFF746FFF8
:10EE3000D4ED037A9FED277A67EE877AB0EE688A81
:10EE4000C4ED037A244818F0FFFF90B9234840210D
:10EE5000FFF7D2FD68B1224BD3F80437012B08D15C
:10EE6000F7EE007AB4EEE78AF1EE10FA58BFB0EE92
:10EE7000678AB0EE480A02B0BDEC048B70BD04F5A1
:10EE8000B34010307DF066FFB7EE008A0028D9D07D
:10EE9000462065F077F8B4EEC80ADFED127AF1EE9D
:10EEA00010FAD8BFB0EE480A87EE800AB2F000FF31
:10EEB0002F209FED0D1ADFED0D0A31F085FAB0EE2F
:10EEC000408ABFE717B7D1383333333F0000000023
:10EED0006F12833A52B87E3FC83F0020702B00204B
:10EEE000707B0020000034428FC2D53F9A99193FB1
:10EEF000F8B5044663F020FD0368DB6898470546D3
:10EF000010B900252846F8BD04F5A046204607F0B4
:10EF10004BF9D6F8C82004F59E4358339A42074669
:10EF200003D196F8AC3B022BEBD804F5B340583034
:10EF30000FF062F90028E4D1D6F8C80003689B6B93
:10EF4000984758B996F8DC30002BDBD004F5005414
:10EF500094F9C453023D18BF0125D3E7084BD3F8F9
:10EF6000C80003685B6B98470028EBD004F5005499
:10EF700094F90134002BC4D0032BC2D03D46C1E725
:10EF8000707B0020F0B52DED028B044600F5A04704
:10EF900000F5B34083B0583097ED468A0FF042F841
:10EFA00004F544550435002840D1D7F80C0A03680D
:10EFB0009B689847D7F89C3C5B0221D5D7F80C3A60
:10EFC00093ED437AD3ED097A67EE877A9FED2F7A36
:10EFD000F4EEC77AF1EE10FA12DB04F5405494ED2A
:10EFE000427A67EE877AF7EE006A86EEA77AB4EE89
:10EFF000667AF1EE10FAC8BFB0EE667A84ED8A7ACE
:10F00000DFED237A90ED250AF0EE480A20EE270A7C
:10F0100028467FF0C9FD28468DED010AFFF732FE34
:10F020009DED010A03B0BDEC028BF0BDD7F8C820FE
:10F0300004F59A4338339A4226D104F50053D3F8A5
:10F04000D03DB3F90860003E18BF012604F5805496
:10F05000D7F81837D4F850461C1B97F814373BB133
:10F060000C484FF40061FFF7C7FC80F00100C3B209
:10F070003246B0EE480A2146284603B0BDEC028B6A
:10F08000BDE8F0407FF094BD0026DFE700000034CB
:10F09000E02E6542702B002010B5044606F04EFCB1
:10F0A00098B104F5A042D2F8183703F58C415031DD
:10F0B000C2F8181704F58051D1F850160029BEBFC8
:10F0C000A3F58C43503BC2F818372046FFF75AFF90
:10F0D000BDE81040042064F041BF00002DE9F04776
:10F0E00000F5B3442DED048B5834054600F5A046D9
:10F0F0002046D6ED468A0EF095FF05F549571C3798
:10F10000002842D1D6F80C0A0368DB689847D6F885
:10F110009C3C5B0221D5D6F80C3A93ED447AD3EDB2
:10F120000B7A67EE877A9FED517AF4EEC77AF1EEAB
:10F1300010FA12DB05F5405595ED987A67EE877A5F
:10F14000F7EE006A86EEA77AB4EE667AF1EE10FA70
:10F15000C8BFB0EE667A85EDE17A90ED250ADFED65
:10F16000447AF0EE680A20EE270A38467FF076F9F6
:10F170003846B0EE408AFFF7A1FDBDEEC80ABDECEF
:10F18000048BB8EEC00ABDE8F087204605F50058AC
:10F190000DF0D0FA9FED379A98EDFD8AD6F81C371E
:10F1A00028EE098A8146BDEEC88A462018EE102A4C
:10F1B0001A4408EE102A64F0E5FEB8EEC88AD8EDCD
:10F1C000E77AD6F8C800A0EE278A05F59A433833C7
:10F1D0009842FDEEC87A17EE904A43D1D8F8D43D54
:10F1E000B3F90880B8F1000818BF4FF00108B9F171
:10F1F000000F1CD103685B699847C0B9D6F8C800F6
:10F2000003689B6B984790B9D6F8343D022B0ED11A
:10F21000284611F001FF50B106F69803D3ED007AAD
:10F2200067EE897AFDEEE77A17EE903A1CB205F5A3
:10F230008055D5F85436E41A96F814373BB10E4889
:10F240004FF40061FFF7D8FB80F00100C3B2B0EECD
:10F25000680ABDEC048B424621463846BDE8F047BB
:10F260007FF0E2B94FF00008C1E700BF00000034B2
:10F27000E02E65420000C842702B002010B5044605
:10F2800015F08EFC68B100B200EB4000C0EB00133B
:10F2900000EE103AB8EEC00ABDE81040132064F04A
:10F2A0005DBE2046FFF71AFFF6E7000010B51048D4
:10F2B000FFF71EFED0B10F480FF0D4F8B0B10E4CDE
:10F2C000042064F05FFED4F8D00D63F0A5FD0420A7
:10F2D00064F044FE132064F055FED4F8D40D63F0BE
:10F2E0009BFDBDE81040132064F038BE10BD00BF88
:10F2F000702B002048850020704B002070B52DED4C
:10F30000028B0446FFF7F4FD002800F0A58004F509
:10F31000A04504F59A42D5F8C8307032934200F007
:10F320009B8004F59B422C32934200F0958004F5BB
:10F330009C420C32934200F08F8004F59B4248328D
:10F34000934200F0898004F59B426432934200F0BE
:10F35000838004F59D42643293427DD004F59E4241
:10F36000934279D01C32934276D004F59E423C32CF
:10F37000934271D004F59E42783293426CD004F5EA
:10F38000B34058300FF06EF8002865D0D5F8C8208B
:10F3900004F59A4354339A425ED004F50056F6EED3
:10F3A000008AD6F8D00D63F0F7FBB4EEE80AF1EE70
:10F3B00010FA3EDDB0EE087AFFEE007AE0EE077A52
:10F3C000B0EE670AD6F8E82DD5F8183707EE902A80
:10F3D000B8EEE77A07EE903AF8EEE77A5142E7EEB8
:10F3E000007AFDEEE77A17EE900AC5F8180731F0BB
:10F3F0008BF8D5F8C820C5F8180704F59C4370337E
:10F400009A4222D0D6F8D40D63F0C6FBB4EEE80AD7
:10F41000F1EE10FAB0EE408A21DCFEEE007AB4EE96
:10F42000E70AF1EE10FA22D5B0EE087AF7EE007A8C
:10F4300019E0FEEE007AB4EEE70AF1EE10FAC1D55B
:10F44000B0EE087AF7EE007AB8E725484FF480511D
:10F45000FFF7D2FA0028D5D0BDEC028B70BDB0EE1C
:10F46000087AFFEE007AE8EE077AB0EE678A204667
:10F4700006F064FA08B1B1EE488AD5F81C37D6ED2B
:10F48000DC6A9FED186A06F6EC5696ED007AB5EE4A
:10F49000C08A07EE903AF1EE10FACCBF28EE268A29
:10F4A00027EE488AF8EEE77A66EE866AE8EE067A94
:10F4B00027EE067AFDEEE77AFDEEE66A17EE903A61
:10F4C000BDEEC77A16EE902A17EE101A17EE900AC4
:10F4D000C5F81C3731F018F8C5F81C07BCE700BFA9
:10F4E000702B00200000C84270B5044604F5A0450A
:10F4F0008FF026FA95F8EC3A064653B1D5F8140B7E
:10F50000036804F5AE4204F5AE411B6A18321C31A3
:10F510009847D5F8D830F31AB3F5FA6F03D9D5F870
:10F52000C80007F003FD2E4BC5F8D860D3F8C8001B
:10F530000268136898470021204611F01DFFDFED97
:10F54000297AB0EEC00AB4EEE70AF1EE10FA45D51A
:10F5500005F51465D5ED007AB1EE047AF0EEE77AA0
:10F56000F4EEC77AF1EE10FA38D504F586601CF097
:10F570003DF9F6EE007AB0EEC00AB4EEE70AF1EE1D
:10F5800010FA2BD504F5C25595ED077AF0EE087AFE
:10F59000B4EEE77AF1EE10FA05F11C051ED504F57C
:10F5A000445004307FF074FB04F549501C307FF068
:10F5B000EBF804F54E50343080F018F895ED007AF1
:10F5C000F7EE007AB4EEE77AF1EE10FA06D504F51C
:10F5D00054502830BDE870407FF05EBD70BD00BF64
:10F5E000707B00200000003400F5005393F94F3386
:10F5F000012BC3BF00F53A5090ED290ADFED047AE4
:10F600009FED040AC8BF20EE270A462064F0A6BC7E
:10F610000000C842000000002DE9F0412DED028BF2
:10F6200000F5A0480546D8ED468A11F0FBFA0746DA
:10F63000D8F8C80003681B6A984705F54E5634365B
:10F6400098B14C4CD4F8E436002B0EDD8FF078F9ED
:10F65000D4F8E436C01A40F6B733984205D8B4F966
:10F66000D84630467FF0CEFF76E098F8293D05F584
:10F67000005443B1B4F9E033002B04DD05F54053E9
:10F6800093F9CA3303BBD8F8C83005F59A45383525
:10F69000AB426BD00021B0EE680A30467FF04AFDE5
:10F6A0000546042064F06EFC2BB207EE903A94ED10
:10F6B000E57AF8EEE77AE0EE077AFDEEE77A17EE04
:10F6C000904A3C4424B2CCE70121284611F09AFC30
:10F6D0009FED297AB4F9E033C0EE077A08EE103ACC
:10F6E000D8F818379FED250AB8EEC88A28EE278A81
:10F6F00007EE903AF8EEE77A67EE807A9FED200AFF
:10F7000027EE800AB2F0F8F8B4F95833DFED1D7A2D
:10F7100020EE270A07EE903A08F2247393ED007A60
:10F72000F8EEE77A0021B4EEE77AF1EE10FA58BF6E
:10F73000F0EE477A80EE277A3046DFED137AB0EEAE
:10F74000480AA7EE270AF0EE680A7FF04FFEBDEEEA
:10F75000C00A10EE103A1CB2BDEC028B20460B49D9
:10F76000BDE8F04141F2941230F0DEBE391E18BF00
:10F77000012190E7707B002000A08C450AD7233C34
:10F7800035FA8E3C0AE81C41E02E65426CEEFFFF24
:10F7900038B500F540530546D3F8AC070368DB687D
:10F7A0009847014605F5545028307FF057FC04B2C5
:10F7B0002846FFF79DFB70B107EE904A05F500550E
:10F7C000B8EEE70AD5F8DC0D63F026FBBDEEC00A03
:10F7D00010EE103A1CB220460349BDE8384041F211
:10F7E000941230F0A1BE00BF6CEEFFFF38B590F868
:10F7F000E433B02202FB030393ED777AF7EE007A4D
:10F80000B4EEE77AF1EE10FA044600F5A0451DD5F6
:10F81000002111F0B1FDDFED427AB0EEC00AB4EE86
:10F82000E70AF1EE10FA11D5D5F80437012B0DD007
:10F83000072B0BD0002385F87C3604F5AD4300225E
:10F840001A602046BDE8384011F0ECB98FF078F826
:10F85000D5F88436C5F88406C31AB3F57A7F84BF19
:10F86000002385F87C36204611F0DCF9D5F8043702
:10F87000012B07EE100A2DD0072B2BD0B8EEC77A3C
:10F88000DFED286AC7EE267A04F50052B2F9A42308
:10F8900000EE102AB8EEC00A27EE800ADFED207ACB
:10F8A000B0EEC07AB4EEE77AF1EE10FA14D4002389
:10F8B00085F87C3695F87C3604F554502830DBB951
:10F8C0007FF0B4FABDE83840174900B241F2941213
:10F8D00030F02ABE9FED150A95F87C26002AE9D162
:10F8E0000122934285F87C26E4D0072B1EBF04F545
:10F8F000AD4300221A60DDE704F5AD4494ED007AD3
:10F90000DFED0B7A67EEC77A9FED0A7A67EE877AAA
:10F91000FDEEE77A17EE901A7FF0A0FBD2E700BF6A
:10F920000000003400A08C456CEEFFFF00000000DA
:10F93000E02E65420000C84270B52DED028B00F547
:10F94000B046403682B0044630468BF03BFB05465D
:10F95000D8B904F50052D2F8D03DB3F9083073B9E4
:10F9600004F5B243D3ED107A92EDE87AF0EEE77A3F
:10F97000F4EEC77AF1EE10FA4CBF012500253046AF
:10F980008BF034FB002808BF002530468BF01AFBB3
:10F9900050BB04F5A043D3F8783601331ED01DBB0D
:10F9A0009FED1C8A2046FFF737FE07EE900AB8EE5F
:10F9B000E70A8DED010AFDB9152064F0CFFA9DED3F
:10F9C000010A1A2064F0CAFA04F5B440603002B0AB
:10F9D000BDEC028BBDE8704003F094BB002DDFD07E
:10F9E0002046FFF703FF02E02046FFF7D1FE07EEB7
:10F9F000900AB8EEE78AD5E71A2064F05BFD9DED2A
:10FA0000010A08B9B0EE480A152064F0A7FAB0EE72
:10FA1000480AD6E70000000010B500F50053D3ED0A
:10FA2000DC6ADFED137A9FED136A03F6EC5393ED76
:10FA3000007A00F53A5366EEA76A27EE277AD3EDEF
:10FA40002A7A67EE867AFDEEE66ABDEEC77AFDEEAB
:10FA5000E77A044616EE902A17EE101A17EE900A6F
:10FA600030F052FD04F5A044C4F81C0710BD00BFDF
:10FA70000000C842A00CB34510B5044613F040FA8C
:10FA8000031E2ADB04F5005191F94F239A4224DD2D
:10FA900004F5A040D0F80447022C1ED0D1EDEA7A3C
:10FAA000DFED0E6AD31A66EEE76A07EE102A07EE5C
:10FAB000903AB8EEC77AF8EEE77AD0F81C3787EEBE
:10FAC000876A07EE903AF8EEE77AE6EE867AFDEE80
:10FAD000E77A17EE903AC0F81C3710BD0000C84214
:10FAE00070B52DED028B00F5A0449FED540AD4F8BB
:10FAF00018379FED537A07EE903AF8EEE77A05460D
:10FB000067EE807A9FED4F0AF0EEE76AF4EE476AFF
:10FB1000F1EE10FAC8BFF0EE477A27EE800AB1F096
:10FB20005BFD30F073FBB7EE008AC8EE007A04F597
:10FB3000E46305F50056C3ED007A94F8EC3AA3B1FE
:10FB4000D4F8140B036805F537515B6A28319847E0
:10FB500058B1D6F8E82DD4F81807514230F0D4FC4B
:10FB6000C4F81807BDEC028B70BD96F98033002BEA
:10FB7000F8D0284605F0E2FE0028F3D105F5B8409C
:10FB8000103013F0BBFB0028ECD1B6F95833012B31
:10FB9000B8BF012307EE903A04F22472F8EEE77A38
:10FBA000D2ED006A86EEA77AB4EEC87AF1EE10FACA
:10FBB00013D840F6C4122449D4F8180730F0A4FC36
:10FBC000C4F81807D6F8E82D40F6C4139A42D4BFFB
:10FBD000C6F8E82DC6F8E83DC4E704F5E463D3EDC4
:10FBE000007AF4EEC77AF1EE10FABBDD88EE070A70
:10FBF00020EE000AB1F0AAFEDFED147AD4F818075F
:10FC000020EE270ADFED127A20EE270A40F6C41311
:10FC1000FDEEC07A17EE905A9D42B8BF1D462A46A7
:10FC2000694230F071FCC4F81807D6F8E83DAB42E1
:10FC3000D4BFC6F8E83DC6F8E85D93E70AD7233C91
:10FC40000000AA4235FA8E3C3CF6FFFFE02E6542EA
:10FC50000000C84210B500F540530446D3F8AC0785
:10FC600003681B68984704F50053D3F8E82D514208
:10FC700030F04AFC04F5A043C3F818072046BDE85D
:10FC80001040FFF72DBF00007047000001207047B3
:10FC90000820704701207047014B93F88C03704790
:10FCA000704B0020034B93F98C0B003818BF0120D8
:10FCB000704700BF704B0020014B93F98E037047D3
:10FCC000704B002013B5064BD3F8C8004B6904688D
:10FCD000009308310EC9646CA04702B010BD00BF8C
:10FCE000707B0020704700007047000038B5254D3C
:10FCF000D5F8C80003685B68984719283BD8DFE847
:10FD000000F00D38360D0D363636363A383838387C
:10FD100038383A36363636383A0D383840241A4BA9
:10FD200093F8892512B193F888350BB944F0100483
:10FD3000164BD5F8C8209A42A3F11C0303D09A426F
:10FD400018BF44F01004124991F90114A9B19A4264
:10FD500015D0032902D10F4B9A4201D144F040043F
:10FD60000D487CF0EDFF50B144F0800407E0102412
:10FD7000D5E71824D3E70124D1E79A42F0D144F023
:10FD8000010038BD707B0020705B0020387A0020B5
:10FD9000704B0020987900200085002008B50448A9
:10FDA00006F082FB00280CBF0120022008BD00BF26
:10FDB000702B0020F0B52DED028B8BB0054619F0AD
:10FDC000C5FA4FF48071D0F8047290ED828AD0F8B1
:10FDD0000C6204461948FEF70FFE30B9184BDFEDF0
:10FDE000197A93EDFD7AA7EE678A17480CF0D6FDD5
:10FDF00030B1164BD3F88C3C5F6893ED028ADE6815
:10FE00002D7C8EF09DFDD4F81823D4F81C33D4F843
:10FE100014130892099327221C23CDE90032039082
:10FE2000079103AA1E21284604978DED058A0696A0
:10FE30005BF06CFC0BB0BDEC028BF0BD702B0020B6
:10FE4000704B002035FA8E3C48850020707B0020E6
:10FE500038B5C5780B46352D044628BF35253522E3
:10FE600000211846B3F0D4FF2A4604F10C01BDE886
:10FE70003840B3F083BF000008B5024813F040F8E3
:10FE800000B208BD702B002037B50D46134840F274
:10FE9000EF2203F03BFE2C7814F004040AD06968CA
:10FEA00003220F481EF0A6FF0C4803B0BDE8304007
:10FEB00003F04CBA01AA214628461FF03DF800285D
:10FEC000F2D0DDED017A9FED077A67EE877A224660
:10FED000FDEEE77A17EE901AE3E700BF702B0020E3
:10FEE000908400200000C84210B5054C012384F81E
:10FEF0008B355DF08DF8002384F88B3510BD00BF85
:10FF0000705B002060F0EAB92DE9F0412DED028B25
:10FF10004FF0000882B0CDE900281E4F9FED1E8AE9
:10FF20000C461546B0EE480AB1F90220D7F8D01DAC
:10FF30004FF47A73064660F0ABFC0123CDE9005321
:10FF4000B4F90020D7F8D41DB0EE480A30464FF47B
:10FF50007A7360F09DFCB4F90420D7F8D81D9FEDAA
:10FF60000F0A43463046CDE9005860F091FCCDE9D8
:10FF70000058B4F90620D7F8DC1DB0EE480A4FF45B
:10FF80007A73304660F084FC02B0BDEC028BBDE8B1
:10FF9000F08100BF704B00200000FA4400007A445A
:10FFA00008B55CF02DFE40F4A67040F0010008BDDD
:10FFB00010B504461FF020FB204610BD10B50B4CB9
:10FFC000002384F8BB365DF01DFDD4F8C820A4F5ED
:10FFD000EC739A4208D194F82C372BB904F5E560FC
:10FFE000BDE8104036F07CBE10BD00BF707B002025
:10FFF00013B5124C94F8E61104F1980016F0DAFCEF
:020000040801F1
:1000000078B194F8E61104F1980016F041FF40B180
:1000100094F8E61104F1980002B0BDE8104016F023
:1000200079BF19F093F901A918F060FF18B19DED9F
:10003000010A02B010BD9FED020AFAE7704B0020E2
:1000400000000000044B93F8EC0A20B1D3F8140B25
:1000500003681B6B18477047707B002008B5084B7E
:10006000D3F8782D002A03DCBDE808405CF00CBE14
:1000700003F6984059F01EFF90ED000A08BD00BF3E
:10008000704B002008B51148D0F8C820A0F5AA731D
:100090009A4214D0B0F9E0309BB990F8453683B954
:1000A00090F8DD306BB990F8F13663B9A0F5A04057
:1000B00006F0FAF900280CBF0320042008BD022036
:1000C000FCE70520FAE70620F8E700BF707B002078
:1000D00030B5224CD4F8C820A4F59C739A4291B054
:1000E000054639D0002304F5126002931EF06CFE21
:1000F000014620B902AA04F512601EF0B1FE2D7C63
:100100008EF01EFCD4F82C39DDED027A0593002325
:10011000D4F828299FED127A0793F8EEE77A08932E
:1001200009930A930B930C930D930E934FF6F85388
:10013000ADF83C300023CDE9030267EE877A9622C2
:100140008DF83E303323CDE90032572103AA2846EB
:10015000CDED067A5BF0DAFA11B030BD707B00208D
:100160000AD7233CF0B58DB004468EF0E9FB184A5F
:10017000D2F8103BC31A642B28D8D2F80C3A02905C
:10018000D3F88C10D3F89020D3F88460D3F888503B
:10019000D3F8DC70D3F894E0D3F898C0D3F89C304F
:1001A000099300238DF82C30069225231622CDE9E1
:1001B00000320591207CCDF81CE002AA5321CDF835
:1001C00020C00A97039604955BF0A0FA0DB0F0BD2D
:1001D000707B002010B55CF05DFF044678B90948DB
:1001E000D0F8C82080F8BB46A0F5EC739A4206D13F
:1001F00090F82C371BB900F5E56036F071FD20460C
:1002000010BD00BF707B00202DE9F043894C2DED1F
:10021000088BD4F8C820A4F59C739A4291B0054687
:1002200000F0E38004F6D8100CF0B8FBDFED828A12
:10023000DFED829A9FED829A002866D004F6D810EE
:100240000CF04CFA002860D0D4F80C0A9FED7D0A1F
:100250006C3033F0C7F904F6E410B0EE60AAB0EEEB
:10026000418ACDED070A8DED081AF0EE40AA8DED1A
:10027000060A81F015FFD4F8103A0146D3F85C2342
:10028000D3F85833059204A8049332F0ABFF09A8C1
:100290008DED090AB0EE680ACDED0A0A32F0B2FF20
:1002A00028EE288A02A8BDEEC88A95F81080CDED08
:1002B000030A18EE103A8DED020A1EB233F016F85A
:1002C000DFED617A20EE270A02A8BDEEC00A6AEED1
:1002D000A8AA10EE103A1FB233F052F8B4EEE90AB1
:1002E000F1EE10FA58BFB0EE690ABCEEC00AD4F8BD
:1002F000C82010EE103A9DB2A4F58E739A422AEEF1
:1003000028AA77D1DFED518A7AE0D4F81837DFF8E0
:10031000409195F81080D9F8AC7707EE903AD4F870
:100320001C37B8EEE7BA07EE903A3B6838469B6850
:10033000F8EEE7AA984707EE900AF8EEE77A384613
:1003400067EEA87A2BEE28BAFDEEE77A6AEEA8AA45
:1003500017EE903A1EB23B681B69984707EE900A69
:10036000F8EEE77AA9F5405067EEA87AFDEEE77A55
:1003700017EE903A1DB204F5D46393ED00AADFEDB9
:100380002F7AB4EEE9AAF1EE10FA58BFB0EE67AAE0
:1003900003F07EF83B68D4ED417A5B6908EE100A01
:1003A000384627EE899A9847B8EEC88ABCEECAAAA2
:1003B00068EE288A1AEE103A8DED09BACDED0AAA38
:1003C000CDED0B8A8DED0C9A8DED0D0AADF83860F0
:1003D000ADF83A50ADF83C30B7221A23CDE90032DF
:1003E0003E2109AA40465BF091F911B0BDEC088BA3
:1003F000BDE8F083D4F8103AD3ED0F7A67EEA88AFF
:10040000D4F8143AD4ED417A186927EE899A86F027
:10041000EFFDCDED09AA8DED0AAACDED0B8A8DED8C
:100420000C9A8DED0D0AADF83860ADF83A70ADF864
:100430003C50D1E7707B00200AD7233C00FF7F4768
:100440000000C8429F0CB345E02E6542000000004A
:10045000705B002001480CF051B900BF48850020B6
:1004600008B5034BD3F8C80003685B68984708BD1C
:10047000707B002030B587B0054618F067FF044652
:100480002D7C8EF051FAD4F88422D4F8883204926C
:10049000059300211023CD22CDE900320290039173
:1004A00002AA42F60C3128465BF030F907B030BDA5
:1004B00030B52DED028B89B0054618F047FF00F5E9
:1004C0005A7393E8070002AC84E80700DDED020AE6
:1004D0009DED030A2D7CF1EE600AB1EE400AB1F009
:1004E0009DFA2046B0EE408A33F000FDDFED0B7A36
:1004F000049B079328EE278A0C230122CDE90032C2
:10050000A82105AA28468DED058A8DED060A5BF027
:10051000FDF809B0BDEC028B30BD00BFE02E654296
:10052000422938B505461BD00AD824290CD04029C9
:1005300024D01B2922D02846BDE8384060F0DABC20
:10054000432917D05329F5E70C215AF0DDFA044668
:1005500010B90024204638BD2846FFF7A9FFF9E767
:1005600010215AF0D1FA04460028F2D02846FFF7AD
:1005700081FFEFE7017C02488AF022FD0124E9E7D0
:10058000B0830020F0B52DED028B05468DB01646E8
:10059000B0EE408A0C46002930D0007C5BF04CF86D
:1005A0000746287C5BF04CFF00F121039F4207D2F5
:1005B000287C0DB0BDEC028BBDE8F0405AF092BA39
:1005C00063690893636A2269CDF82530236AA069BC
:1005D000E1680792CDF8293062222123276805902F
:1005E000CDE900320691287C0397192303AAC22182
:1005F0008DED048A8DF824605BF088F80DB0BDECB9
:10060000028BF0BDF8B5474CD4F8C820A4F59C7314
:100610009A42054600F08580A4F54056B6F82A3483
:10062000DB0712D504F6D8100DF0C6FB002872D0F7
:10063000D4F80C0A03689B68984700F1940191ED87
:10064000010A01222846FFF79DFFB6F82A349F07CA
:1006500011D535480DF0B0FB00285ED0D4F80C0A57
:100660000368DB68984700F1940191ED010A0222CA
:100670002846FFF787FFB6F82A34580711D52A48CD
:100680000DF09AFB00284AD0D4F80C0A03681B69C5
:10069000984700F1940191ED010A03222846FFF7E3
:1006A00071FFB6F82A34190708D520490B4693ED97
:1006B000000A043905222846FFF764FFB6F82A34F9
:1006C000DA0614D5D4F80437042B10D118F03EFE06
:1006D000074617488AF0A4FC97EDC70ADFED157AA4
:1006E000014620EE270A06222846FFF74BFFB6F800
:1006F0002A349B0615D50C480DF05EFB88B1D4F862
:10070000101A284691EDAB0ABDE8F840042201F525
:100710002A71FFF737BF084991E70849A5E708495B
:10072000B9E7F8BD707B002048850020CC60002030
:10073000B0830020E02E65429C5D0020F85E002022
:100740006C60002070B504460E4628F095F890F8CD
:10075000C412B02303FB0101AC31204603F03CFB83
:100760000546C0B13EB118F0F1FD90F87C3243F07F
:10077000020380F87C3204F5A043D3F8C80004F5E6
:100780009C435433984204D004F59E445834A0420C
:1007900001D106F0F5FA284670BD000073B5164683
:1007A0000191044618F0D2FD019918F0E7F90546C9
:1007B000C0B13EB118F0CAFD90F87C3243F002039C
:1007C00080F87C3204F5A043D3F8C80004F59C43BC
:1007D0005433984204D004F59E445834A04201D1C9
:1007E00006F0CEFA284602B070BD000030B50546CE
:1007F00085B00C46D1E9040130F0EAFE40B168460C
:100800001EF0F2FA6A46214628465FF0B1FF08B9A9
:10081000022067E0344840F24F32694603F076F92F
:10082000D4ED037AF4EE677AF1EE10FA22D69FED5A
:100830002F7AF0EEE77AF4EEC77AF1EE10FA54BFB1
:10084000012200229DF80030294962F341036846E5
:100850008DF800301EF000FC0028D9D125486946EB
:100860006CF0D0F840B957F013FF0522162157F06D
:100870006BFECDE70022E5E7D4ED017AFDEEE77AE5
:1008800017EE903ADB0706D41B4BA3F5BA72D3F8E8
:10089000C830934225D119491348022212F040F979
:1008A0009DF8001011F0040102D168461EF034FBDF
:1008B0000D48694603F0DCF994ED020AB4EE400AF3
:1008C000F1EE10FA0BD6B5EEC00AF1EE10FA06DD25
:1008D0009DF800100948C1F3400107F021FC0020F9
:1008E00000E0042005B030BD702B00200000003473
:1008F00080840020C04D0020707B0020FC79002007
:1009000010B52DED028BD1ED017A91ED008AFCEE50
:10091000E77A8AB0CDED037A9DF80C1005AA04465B
:100920005FF010FFC8B1DFED0E7A059B009368EE13
:10093000277A0022FDEEE77A114617EE903A06A8D4
:100940001EF072FA23682046D3F8C43006A99847EF
:1009500000200AB0BDEC028B10BD0220F9E700BFF9
:100960000000C84237B5124DD5F8C80003681B6AAD
:100970000C46984740B9D5F8C820A5F5EC739A42C3
:1009800002D0042003B030BDD4ED007AD4ED020AC9
:1009900094ED010A0748FCEEE77ACDED017A9DF867
:1009A000041003F0C3FE0028EBD00020EAE700BFEC
:1009B000707B0020702B0020134610B524220C46BB
:1009C00018460021B3F024FAA27F8277E27FC27733
:1009D000072280F82020A28B8283D4ED067AF1EEE4
:1009E000677AC0ED067A10BD10B48C8B162C03D13B
:1009F0005DF8044BFFF7E0BF5DF8044B5FF0E0B833
:100A000008B591F82030072B0ED1094890F8EC3A40
:100A100043B191ED060A00F6D810B1EE400A0CF091
:100A200099FF18B9042008BD0220FCE70020FAE76E
:100A3000707B002008B5D1ED007A9FED087A084858
:100A4000F0EEE77AF4EEC77AF1EE10FA54BF012126
:100A5000002104F06DFF002008BD00BF000000343D
:100A6000702B002010B5D1ED007AFCEEE77A17EE7E
:100A7000903A9CB2012C02D0022C06D084B91148C5
:100A8000214666F0DDFF002010BD0F4890F8343895
:100A90005B0707D560F0A4FC0C4A052159F018FE4D
:100AA0000420F1E790F920381BB960F099FC084A5E
:100AB000F3E7A0F5A0400AF09BFA002814BF00203D
:100AC0000420E1E790830020707B0020108C0C084C
:100AD0002B8C0C081FB5D1ED017AFCEEE77A0B46A2
:100AE000CDED027AD1ED007A1A7C017C0192FCEE08
:100AF000E77A0B48CDED037AD3ED027AFCEEE77A84
:100B000017EE902A92B2009293ED030A9DF80C2002
:100B10009DF8083009F0F2FB05B05DF804FB00BF5A
:100B20004885002007B5D1ED007A0848FCEEE77A49
:100B3000CDED017A9DF804100BF0E6F900280CBF0A
:100B40000420002003B05DF804FB00BF48850020AE
:100B500070B58B8BC02B05460C4633D8B12B0DD806
:100B6000142B00F0AE80162B59D0112B00F0A6806C
:100B700021462846BDE8704061F054B8B23B0E2BC8
:100B8000F6D801A151F823F00D0C0108710B0108F2
:100B9000710B0108710B0108710B0108710B010841
:100BA000710B0108710B0108030C0108710B01089E
:100BB000370C0108710C0108710B0108270C0108A2
:100BC000F90B0108D42B13D007D8D02B23D0D12B6D
:100BD000CED1BDE87040FFF77DBFB3F5967F53D00F
:100BE00040F6B836B342C3D1BDE87040FFF79ABFB4
:100BF000BDE87040FFF71EBF2146BDE87040FFF71B
:100C0000F5BD2146BDE87040FFF77ABE2146BDE83C
:100C10007040FFF7A7BEBDE87040FFF723BFBDE8F7
:100C20007040FFF7EDBE94ED000A2848FDF726FC62
:100C3000E0B100201BE0264C94F8F930B3B104F584
:100C4000116104F5E56036F049F978B1012384F8C3
:100C500061370222A4F5EC71A4F5A04011F060FF09
:100C60000028E6D11A4B002283F86127042070BDCA
:100C7000174C94F8F930002BF8D004F5116104F505
:100C8000E56036F0AFF8E0E7D1ED007A9FED117A3C
:100C9000F0EEE77AF4EEC77AF1EE10FA14D5D1ED62
:100CA000017AF0EEE77AF4EEC77AF1EE10FA0BD59E
:100CB00009490222054811F033FFBAE70749022229
:100CC000F8E707490222F5E70220D0E7702B002061
:100CD000707B00200000003498790020E07900202B
:100CE000C4790020F0B5414CD4F8C820A4F5BA73FB
:100CF0009A428FB00D4677D1CE78272E28BF27266F
:100D00002722002104A8B3F083F8324605F10C0134
:100D100004A8B3F033F8059B9DF836500093069B6A
:100D20000193ED43079B0293EDB2089B03938DF86B
:100D300036508DF005FE15F0810F05F08707064649
:100D400001D1802F12D1684631F0B6FFDFED287A4D
:100D5000C4F8DC6620EE270ADFED267A20EE270AAB
:100D6000BDEEC00A10EE103AC4F8D03615F0820F6E
:100D700001D1802F12D1684631F0B8FFDFED1C7A27
:100D8000C4F8E06620EE270ADFED1A7A20EE270A83
:100D9000BDEEC00A10EE103AC4F8D43615F0840F38
:100DA00001D1802F12D1684631F0B0FFDFED107A0B
:100DB000C4F8E46620EE270ADFED0E7A20EE270A5B
:100DC000BDEEC00A10EE103AC4F8D8366B060BD54B
:100DD000DDED0C7A9FED077AC4F8EC6667EE877A52
:100DE00004F5DD63C3ED007A0FB0F0BD707B002029
:100DF000E02E65420000C84230B5204C91B0084654
:100E000002A9FFF725F8D4F8C820A4F5BA739A42CE
:100E100031D19DF83C30072B2DD1D4F82439DDEDAC
:100E2000056A9FED177A07EE903AF8EEE77AE6EE5C
:100E3000C77AFDEEE77A17EE903AC4F8243960F0ED
:100E4000CFFAD4F8FC28D4F8243952689FED0D7AF3
:100E50009B1A07EE903AF8EEE77A054667EE877A36
:100E600017EE900AFBF748FB074ACDE9000106217F
:100E7000284659F02DFC11B030BD00BF707B00201A
:100E80000000C8420AD7233C448C0C0810B51D4B07
:100E9000A3F5BA72D3F8C8309342044696B0084618
:100EA0000FD108A9FEF7D4FF9DF8541003AA2046DD
:100EB0005FF048FC38B960F093FA134A042159F006
:100EC00007FC16B010BDBDF8503023F004039BB2F0
:100ED000002BF6D0DDED0B7A9FED0C7A039B00938F
:100EE00067EE877A0022FDEEE77A114617EE903A18
:100EF00004A81DF099FF236804A9D3F8C430204644
:100F00009847DEE7707B0020588C0C080000C84230
:100F100030B48D7A4B7A43EA0523CD7A43EA054310
:100F2000562B04460A4618D008D8522B0FD0542B03
:100F300010D02046114630BC5FF00CBD03F1807329
:100F4000863B23F07F43012BF3D830BC704730BC85
:100F5000FFF7C8BE30BCFFF74FBF30BCFFF796BFEE
:100F600000207047C820704701207047002070475C
:100F70000020704790F890308B4286BF00EB8100D4
:100F8000D0F894000020704790F890308B4286BFD4
:100F900000EB8100D0F894000020704703207047D8
:100FA000014B93F88A037047704B002070B50446DC
:100FB0003E4810F0DBF918B1236A43F400032362C2
:100FC0003A4810F0D3F988B1462062F0DBFFDFED3C
:100FD000387AB4EEE70AF1EE10FA07D8636A43F400
:100FE00000036362A36A43F40003A362236A43F429
:100FF000F84323622F4BD3F8C80003685B68984717
:101000000138182815D8DFE800F0343C0D3E3C3C90
:101010003C3C14343434343434143C3C3C3C3414C0
:101020003E343400244A92F8883553B392F8892527
:1010300052B3224B1D68DDB1214E284696F8C21DE1
:101040004FF00CFAA0B1236A43F48073236296F93F
:1010500028341BB1636A43F48073636296F8C21D3F
:1010600028464FF033FA18B1A36A43F48073A362A1
:1010700070BDD4E9092342F4E04243F4E0436262E4
:10108000A362012300E00023616A41F4806262628E
:10109000A26A42F48060A062002BCAD041F4406191
:1010A00042F440626162A262C3E700BF702B00207D
:1010B000000000B4707B0020705B0020048A0020D8
:1010C000704B002013B54FF44470CDE900211EF0A1
:1010D0008BFA044628B1DDE9002160F09FF9024B4C
:1010E0002360204602B010BD548E0C0800207047CB
:1010F00000207047002070470020704700F50F5017
:101100002C30704700487047A0B40C0800F5A04090
:10111000D0F8C80003685B681847000000F5A043DA
:1011200000F59C40D3F8C83028301B1A584258416B
:1011300070470000A22070472DE9F04100F5A0465D
:10114000DFED696AD6F8183707EE903AD6F81C3703
:10115000B8EEE77A07EE903AF8EEE77A00F5B34892
:1011600090B027EE267A67EEA67A08F15808044672
:10117000002340468DED017ACDED027A03930BF00A
:101180000DFC002800F0A980D6F80C3A84330FCB70
:101190000CAF87E80F0008AD04AF87E80F0085E8C3
:1011A0000F0001A9384603AB02AA31F0C9FD9FED3B
:1011B0004F0AD6F88C7C01A832F014FA294638463A
:1011C0008DED080ACDED090A8DED0A1A16F0AEF97B
:1011D0008DF0B6FBD6F8103BC01A04F58D55632888
:1011E00005F110052DD8D6F80C0A03689B689847BE
:1011F000042100F19402284656F0B2FAD6F80C0AFF
:101200000368DB689847052100F19402284656F0F0
:10121000A7FAD6F80C0A03681B699847062100F163
:101220009402284656F09CFAD6F8102A284602F571
:101230002A72072156F094FA04F5B840103013F0E2
:10124000C3F840460CF0B8FD90B1D6F8100A85F00E
:10125000ABFB68B1D6F8102A6E219032284656F0C2
:101260007FFAD6F8102A6F21BC32284656F078FA59
:1012700004F548522C326921284656F071FA04F5DB
:101280004E5208326A21284656F06AFA04F5405355
:1012900093F9CA2332B9D3EDF07AF5EEC07AF1EEC4
:1012A00010FA06DD04F553523C326B21284656F005
:1012B00057FA04F55454283420467DF0F1FE28B145
:1012C00004F130026D21284656F04AFA18F03EF833
:1012D00017F050FD10B0BDE8F08104F5A25001A94F
:1012E000183015F0EBFF73E70AD7233CE02E654278
:1012F00010B54FF48011044611F0FCFD10B12046EA
:10130000FFF71AFF4FF48001204611F0F3FD28B1DA
:101310002EF0D8FABDE810402CF09EB910BD0000A8
:1013200070B500F5A25590B000231835029302A9BC
:10133000002304460DF1070228468DF8073017F008
:10134000DBFD03A9284616F0CFFD08B92D4B03930A
:101350003022002104A8B2F05BFD04F5A046A323CF
:101360008DF8103095238DF811308DF0F1FAD6F804
:101370001837ADF81B3004F58053CDF81300D3F8BF
:101380005026ADF81D20D3F85436D6F81C27CDF8DA
:1013900017104620ADF81F20ADF8213062F0F2FDA5
:1013A00010EE103A1520CDF8233062F0EBFD10EE70
:1013B000103ACDF8273004F53A539FED137AD3ED68
:1013C000297A67EE877A284617EE903ACDF82B30C7
:1013D000029BCDF82F309DF807308DF83330039BFA
:1013E0000D9317F08FFF04F58D50D6F80C318DED6D
:1013F0000E0A302204A910300F9356F0C9FA10B02B
:1014000070BD00BF2292CA7F0000C84270B58EB086
:101410003522054600216846B2F0FAFCA3238DF878
:10142000003095238DF80130012305F5A0448DF897
:1014300002308DF08DFA05F5405604F5D463CDF8F1
:1014400003001B68D6F8AC07CDF80710CDF80B30B9
:1014500003681B699847ADF80F00D6F8AC0703681E
:101460009B689847ADF811001B4802F011F8ADF8E1
:101470001300D6F8AC0703685B69984710EE103A82
:10148000D6F8AC07CDF8153003689B69984710EE85
:10149000103ACDF81930D4F80431CDF81D30D4F815
:1014A0002839CDF82130D4F82C39CDF82530D4F8AE
:1014B0002439CDF8293005F58D50D4F83C3DCDF8D0
:1014C0002D303522D4F8FC30CDF83130694610305B
:1014D00056F05EFA0EB070BD702B002030B587B0AC
:1014E0001622044600216846B2F092FCA3238DF830
:1014F000003095238DF8013002238DF802308DF0F5
:1015000027FA04F5A045CDF803002046CDF80710D2
:1015100004F0CAFF05F5E1638DF80B001B68039327
:10152000134B1B68D86A90F89C308DF81030036814
:10153000DB69984795F8F1368DF812308DF8110077
:101540002EF0C0F92DF0B4F9D5F804378DF813005A
:1015500004F58D508DF81430162295F8F2368DF87A
:1015600015306946103056F013FA07B030BD00BF91
:101570006C2B002010B58AB0272204460021684653
:10158000B2F046FCA3238DF8003095238DF801308E
:1015900009238DF802308DF0DBF9CDF8030004202B
:1015A000CDF8071062F0EEFC10EE103A1320CDF8E3
:1015B0000B3062F0E7FC10EE103A4620CDF80F3009
:1015C00062F0E0FC10EE103A1520CDF8133062F016
:1015D000D9FC10EE103A0320CDF8173062F0E2FC8F
:1015E00010EE103A1A20CDF81B3062F0CBFC10EE52
:1015F000103ACDF81F3004F5A04304F58D50D3F810
:101600001831CDF8233027226946103056F0C0F942
:101610000AB010BD13B5044600F58D50103001908E
:1016200055F00CFD019855F0A3FD04F58053019889
:1016300093F968320BB155F043FE204602B0BDE885
:101640001040FFF797BF00007047000070B500F52D
:10165000A04600F58D5596F8EC3A88B00446103552
:1016600053B1D6F8040A1E22694687F0CDFA0F4915
:101670006A46284656F010FBD6F8C80003685B6837
:10168000984704F50053014693F80C23284656F07A
:1016900027FB04F5A250183018F0D2F804F590702A
:1016A00008B0BDE8704026F051B900BF608F0C084B
:1016B0009FED020A00224CF0BDBF00BF0AD7233CB9
:1016C000134B70B5044640F8043B60F0B5FF114E73
:1016D000114B63605425601961F064F9665130352F
:1016E000B5F5557FF7D104F5557063F041F80B4A15
:1016F00004F5EC6002F634318AF0EEFA012320465C
:10170000074984F891394DF093FB204670BD00BF26
:10171000A039002080DF0C0894DF0C08BC4E0020AC
:1017200090CF0C082DE9F04100F50E519AB00D2232
:101730000831044654F074FD0022BD4827214CF0C6
:10174000F1FE0421002062F09DFF1321012062F0D0
:1017500099FF4621022062F095FF1521032062F0D7
:1017600091FF62F05FFD04F5A04393F9A43A23B121
:101770009FEDB00AB0484DF003FF4DF05FFDAF4A5A
:10178000AF4E138843F0040313804FF000080AAFF4
:10179000002110223846B2F03BFB01238DF8303097
:1017A0003388ADF8283005A973680B9338464CF0A0
:1017B000C1FDC8B19DF91430002B15DD61F0BCF8F6
:1017C0009DF81410036801391B68C9B2984758B1D5
:1017D000051D28464CF04CFD30B9B368ADF8183003
:1017E00006A928464EF0E6F908F10608B8F12A0FD6
:1017F00006F10C06CCD1934800220DF10B014CF000
:101800001FFB06AD064620B34CF032FD08BB8E4BE5
:101810000FCB85E80F0004A928464CF08BFD00286B
:1018200040F032814FF00408884B0FCB87E80F005F
:1018300005A938464CF07EFD28B105A84CF018FDEE
:1018400008B148F0010803A930468DF80C804EF02D
:101850005FF97F4B0FCB85E80F0003A928464CF0BA
:1018600069FD002846D00998002204A94CF0E8FA46
:10187000064600283ED04CF0FBFC0546002839D136
:101880009DF80C30013BDBB2032B96BF714A034637
:10189000D35C8DF82830304639464EF039F96E4821
:1018A000002205A94CF0CCFA06466BF0EDFA78B1AF
:1018B0006BF0E8FA90F8302090F8281090F8483053
:1018C000114490F840200A44D34214BF012500255A
:1018D00086B130469DF90C804CF0CAFC50B91DB160
:1018E000B8F1000518BF0125394630468DF828505B
:1018F0004EF00EF90022B7EE000A022104F50F5057
:101900004CF098FE012304F502510093534A002342
:1019100018318E204CF00AFE94F9ACC9BCF1000FCE
:101920001AD14F4E0FCE3D460FC50FCE0FC50FCE6D
:101930000FC596E80F0085E80F006246042138467F
:101940004CF0F0FD9FED470A47484DF019FE47481F
:10195000B7EE000A4DF014FE012504F50951444A82
:1019600000950023103140F205104CF0DFFD04F526
:101970000F5002213430FFF79BFE04F50D50032178
:101980001C30FFF795FE04F50D5003212430FFF7BE
:101990008FFE04F50F5003213030FFF789FE04F568
:1019A0000F5002213830FFF783FE04F50D5002215D
:1019B0003030FFF77DFE04F50D5002213430FFF783
:1019C00077FE04F50D5002212C30FFF771FE04F56F
:1019D000B040403089F088FC264A1368D90705D406
:1019E0002549156004F5075338330B6004F5105092
:1019F0002149012230304CF0EBFD012504F58D51D9
:101A00001E4A009500231031FD204CF08FFD1C4B29
:101A10001A68D20705D41B4A1D6004F59B541C3478
:101A20001460184801214CF0EFFD1AB0BDE8F081B8
:101A3000CCCC0C0800009643B4B50D08E889002012
:101A40003CCF0C0890CC0C0824800C0834800C0887
:101A500044800C08C8CC0C089BCC0C0890100D08D6
:101A600054800C0800000000A8CC0C08B7CC0C086F
:101A700030430E08642B002000220020389E0D0801
:101A8000682B00200C22002004A84CF0F1FB002859
:101A90003FF4C8AE4FF00C08C6E600BF7047000028
:101AA00000207047002070470020704700207047DA
:101AB00000207047704700000020704700207047EA
:101AC00084B001A880E80E0004B000207047000038
:101AD00000207047002070477047000010207047BA
:101AE000004870477CDB0C08004870478CDB0C0812
:101AF00000207047704700000120704701207047A8
:101B000000207047002343608360C360036143612A
:101B1000002303767047000010B50446FFF7F2FF7C
:101B20000023637610BD0000027E531CDBB2042B41
:101B3000037600EB820288BF002382ED010A88BF92
:101B40000376704710B50446FFF7EEFFD4ED017A37
:101B50009FED107A94ED020A637E77EE877A042B6C
:101B600077EE807A94ED030A94BF0133052377EE74
:101B7000807A94ED040A637677EE807A637E94ED42
:101B8000050A77EE807A00EE103AB8EEC00A87EECA
:101B9000800A10BD0000000010B504461DF02CFDA9
:101BA000204610BD04F0A0B902F0CEBF03F084BD02
:101BB00002F0D8BF01F076BC01F028BB01F050BCA8
:101BC00001F0E6BCFDF72AB8FCF7EABB70B5224B82
:101BD000036000F540530446D3F840071F4AC3F89A
:101BE000902508B11DF00CFD1D4B236004F500533A
:101BF00093F834203AB91D6B2DB128462AF0A4FD84
:101C000028461DF0F9FC04F59B507AF0DFFB04F543
:101C10009350083063F0ACFE04F6B46504F65466E5
:101C2000B54204D0183D28462AF0E4F9F8E70D4BF8
:101C3000C4F8983804F6F81057F018FE04F6CC10E3
:101C400057F014FE04F62C1057F010FE04F5106047
:101C500057F00CFE204670BD38C30C08C8B60D08FE
:101C6000B0970D08005F0D0838B5474B044640F8A3
:101C7000043B64F0C3F904F110001AF077FF04F19B
:101C8000680053F081FC04F5907025F041FA04F5EA
:101C9000866019F081FD04F254501DF0B3FC04F687
:101CA00098002BF0D1FD04F5636063F085FF04F527
:101CB00070604EF0F9FA04F58D50103055F0B0FD1B
:101CC00004F59350083063F03BFE04F59550043062
:101CD0001CF03EFA04F59B507AF064FB04F59B502F
:101CE0001C3054F013F804F59E50103065F030FBB2
:101CF00004F580530025254A83F8F45304F5A050D9
:101D000004F59F5314330430136049F053FF04F576
:101D1000A2502946183015F0BFFD04F5D65073F0D7
:101D20003DFA04F5F650043077F082FB04F5FE50DE
:101D30001C3079F091FC04F501507AF0C7F804F5F5
:101D40000250183014F0CAFC04F50750383073F014
:101D500083FE04F5095010306AF06CFB04F5005363
:101D600004F50C5083F80C53094D24307AF0EEFE44
:101D70002B6813B107488CF0B1FD204606494DF0A1
:101D800057F82C60204638BDB0970D08D892002037
:101D9000388A002094DB0C08D8960D082DE9F04F06
:101DA0002DED028B04469FB0FFF75EFFE14B2360F1
:101DB00004F510503030FFF783FC04F5375008303D
:101DC00004F500557CF0F8F904F50F531233C5F80B
:101DD000F03D04F53850062385F8F43D1C3063F0DF
:101DE000C1F904F5B0434033C5F8983E0E934FF463
:101DF000006304F53A58C5F89C3E04F50D5A5A2381
:101E000004F5A25985F81C3F0AF10C0ACA4BC5F823
:101E100094AE09F11809C5F8909EC8F86031C74B17
:101E2000C8F86431B7EE008AC54BC8F8683104F5CC
:101E30004150C8F8CC3188ED578A1C3058F036F83C
:101E400004F5415004F54056283058F02FF800278B
:101E5000BC4BB36786F8907008F5FC70FFF752FE34
:101E6000B94BBA49B36786F8917040464CF0E0FF31
:101E7000B74BC6F8A080C6E926390023C6F8CC3097
:101E8000C6F8D43004F54255012304F5435086F8D2
:101E9000DC30183530301CF0A7FFAE4986F80071F1
:101EA00028464CF0C5FF04F54450514604307CF000
:101EB00039FD04F5495051461C307CF097F904F582
:101EC0004E50514634307DF0F7F82C22394606F555
:101ED000AB60B1F09DFF04F554509F49283004F5E4
:101EE00056574CF0A5FF10379C4BC6F8903507F1BC
:101EF00008008BF0EFFE04F5565B04F558530BF128
:101F00003C0B203358460F935CF04CFD0F9B0BF1BC
:101F1000140B5B45F6D10723C6F844370023A6F817
:101F200048374FF4CB701DF065FBC6F8400704F549
:101F30005D500C308BF0CEFE04F55E5010308BF00F
:101F4000C9FE874B1A6802B91F60864BC6F89035E8
:101F500004F55E504FF48051C6F8AC5730301AF09B
:101F6000DFFE04F5605030304DF0DAFE04F56150CC
:101F700004306CF005FB04F59A4004F580451C30F4
:101F800004F0D2FE784BC5F81C3D04F59A40383079
:101F900004F0CAFE754BC5F8383D04F59A4054303C
:101FA00004F0C2FE724BC5F8543D04F59A407030FF
:101FB00004F0BAFE6F4BC5F8703D05F69853002249
:101FC00004F59B40DA609A605A6083ED008A2C30F9
:101FD00004F0AAFE684BC5F8AC3D04F59B404830C0
:101FE00004F0A2FE654BC5F8C83D04F59B40643083
:101FF00004F09AFE624BC5F8E43D04F59C400C30B9
:1020000004F092FE5F4BC5F80C3E04F59C4028306E
:1020100004F08AFE5C4BC5F8283E04F59C40543021
:1020200004F082FE594BC5F8543E04F59C407030D4
:1020300004F07AFE564BC5F8703E04F59D400C3016
:1020400004F59D4704F070FE2C37524BC5F88C3ECA
:10205000384604F069FE504BC5F8AC3E04F59D408F
:10206000483004F061FE4D4BC5F8C83E04F59D4074
:10207000643004F059FE4A4BC5F8E43E04F59E4036
:1020800004F052FE474BC5F8003F04F59E401C305B
:1020900004F04AFE444BC5F81C3F04F59E403C301A
:1020A00004F042FE414BC5F83C3F04F59E405830D9
:1020B00004F03AFE3E4BC5F8583F04F59E40783098
:1020C00004F032FE3B4BC5F8783F04F59F401430D6
:1020D00004F02AFE384BC5F8943F04F59F40303099
:1020E00007F06AFE04F59F406C3004F01DFE334B90
:1020F000C5F8EC3F04F5A045314BAB6028464FF4E2
:10210000C0533049A5F85C3008304CF091FEFE23F6
:1021100085F8D430052385F8F8304FF0FF33C5F843
:102120000031294B119304F5A240284B85ED468AD6
:102130004EE000BF38C30C08000080BF0000B4426E
:102140000000B4C2CCDB0C08DCDB0C08D47A0E082F
:1021500034780E08DC770E0834760E08C8B60D0801
:10216000548D0020288F0C08DCE60C08D8ED0C08F4
:10217000F8F00C08D8E40C08ECE70C0874E80C083C
:1021800054E70C085CE60C08D8E50C0868ED0C0870
:1021900064E90C08F4E80C0814DC0C08E4E90C0809
:1021A000F0EC0C08E4EA0C08D4EB0C0854EB0C0837
:1021B0006CEC0C0864EA0C0868E40C0874F00C0879
:1021C00004DC0C08949B0E08A51B0108088C0C0865
:1021D0004FF40071C5E93277224600931C30874BDB
:1021E00010941AF01BF84FF0FF33C5F8783605F558
:1021F000D163834ADA6003230027C5F8043705F565
:10220000E463C5F8D076C5F8D476C5F8D876C5F8B5
:10221000DC76C5F8E076C5F8E47683ED008A794B84
:10222000C5F84837784BC5F8503704F5AE40774BC2
:10223000C5F85837C5F84447C5F84C47C5F8544762
:102240006C301CF0D1FD04F5AF4008301CF0CCFD23
:1022500004F5AF4024301CF0C7FD04F5AE4B6C4BC9
:10226000C5F8B8370BF1280B4FF0FF33A5F8BC3792
:102270000BF198001CF0B8FD4FF0FF32654BC5F82C
:102280001C286549C3F800B058464CF0D1FD4FF604
:10229000FF73A5F864374FF0FF33A5F8803704F5D6
:1022A000B0405E4B5E49203018604CF0C1FD5D4B84
:1022B000D6F8AC271294CDE913345B4BCDE9153435
:1022C0005A4BCDE917345A4BCDE91934594BCDE966
:1022D0001B34594B1D931EA911E903000CAB83E875
:1022E0000300DDE91A010AAB83E80300DDE9180108
:1022F00008AB83E80300DDE9160106AB83E80300C1
:10230000DDE9140104AB83E80300DDE9120102AB4F
:1023100083E803005946CDE9002A43464A460E9811
:1023200088F0ECFD09F51B73C5F8FC3804F5B240E4
:102330001CF05AFD04F5B24010301CF055FD04F5B8
:10234000B240203004F5B3461CF04EFD103610228A
:10235000394605F51360B1F05BFD30467AF0B0FC0C
:10236000364B3749C5F8903930464CF061FD354A57
:102370003549116004F5B34348331426B8B206FB5F
:1023800000120137127C002AF8D1304A1080304AFE
:10239000166816B12F488CF0A1FA04F5B3404C3002
:1023A00013607AF077FC2C4BC5F8CC3904F5B340B8
:1023B0004946583008F0E4FF284BC5F8D03C642368
:1023C00085F8D43C264BC5F8083D04F5B940254BAB
:1023D000C5F80C3D244950304CF02AFD234BC5F87C
:1023E000D03C20460123C5F8306D85F8386D85F85E
:1023F000B8361FB0BDEC028BBDE8F08FA51B0108FD
:102400000000B442A91B0108AD1B0108B11B010863
:102410000000FFFF30890020386D0D08DC9200209D
:10242000E8C40D08B51B0108B91B0108BD1B010854
:10243000C11B0108C51B0108C91B0108EC850C085C
:10244000C4850C08F889002040D10C08F6890020CA
:10245000B4890020A8DB0C082C860C08ECDB0C08E7
:10246000E40C0D083C0D0D08C4BD0D08BC0E0D0894
:1024700010B58BF095FE064C064B18602046FFF712
:102480008DFC2046044A0549BDE81040AEF07EBFF1
:10249000702B00206C2B00204CEA0020CD1B010883
:1024A0000069C0F3401070470F299DBF302303FB24
:1024B0000100503000207047014B93F9D103704761
:1024C000704B0020014BD3F8DC0D7047704B00209F
:1024D00008B503689B68984730B9044B93F8E2004D
:1024E000B0FA80F0400908BD0020FCE7707B0020B6
:1024F00008B504480EF0B2FC10B9034B93F8DC00A9
:1025000008BD00BF702B0020707B0020022A10B590
:102510000C4605D1BDE810400948352210F0D0BB6B
:10252000084BD3F8C80003685B689847A04205D100
:1025300060F002FABDE8104060F088B910BD00BF3D
:10254000702B0020707B0020012910B50C4610D0A4
:10255000022904D061B95EF043FF084A02E05EF050
:102560003FFF074A062158F0B3F8064BC3F8704AFC
:1025700010BD5EF035FF044AF4E700BF2CDD0C0807
:1025800004DD0C08707B00201BDD0C08012910B550
:102590000C4614D0022907D0D1B90E4BC3F8301D18
:1025A0005EF01EFF0C4A05E00A4BC3F8301D5EF0DA
:1025B00017FF0A4ABDE81040062158F089B85EF0BE
:1025C0000FFF074A062158F083F8024BC3F8304D3D
:1025D00010BD00BF707B00206BDD0C0840DD0C08D7
:1025E00054DD0C08012903D0022914BF0021022167
:1025F000014BC3F87C1D7047704B0020012902D0AD
:10260000022900D011B9024BC3F8341D704700BF36
:10261000707B00206C2910B400F3A6803F290FDCEA
:10262000162900F39980032940F39A807E4B0124F8
:102630008C402340002B00F093805DF8044B7047E2
:10264000A1F140032C2B00F28B8001A454F823F05D
:10265000092801086127010861270108612701088D
:102660006127010861270108612701086127010826
:102670003B2601086127010861270108612701083D
:10268000612701083B26010861270108612701082D
:102690006127010861270108FF2701086127010858
:1026A000FF27010861270108FF270108FF2701080C
:1026B000FF2701083B26010861270108FF270108C1
:1026C0003B26010861270108612701083B26010814
:1026D0003B260108612701083B2601086127010804
:1026E00061270108612701086127010861270108A6
:1026F0006127010861270108612701083B260108BD
:102700003B260108112B2BD801A454F823F000BF5D
:102710003B2601086127010861270108612701089C
:102720003B2601086127010861270108612701088C
:102730006127010861270108612701086127010855
:102740003B2601083B260108612701086127010893
:102750003B2601083B260108A1F12703112BD1D903
:102760005DF8044B60F0FABEA0291FDC9529F7DD67
:10277000A1F196030A2BF3D801A454F823F000BF6B
:102780003B2601086127010861270108612701082C
:102790003B2601083B260108612701083B2601086A
:1027A0006127010861270108FF270108B52921DCFD
:1027B000A929D5DDA1F1AA030B2BD1D801A454F886
:1027C00023F000BF3B2601086127010861270108AB
:1027D0003B26010861270108612701083B26010803
:1027E00061270108612701086127010861270108A5
:1027F0003B260108A1F1D003022BB1D81DE75DF8FB
:10280000044B002360F07CBE084B012283F82C2D82
:10281000A3F54053D3F8D80D00283FF40EAF5DF870
:10282000044B642160F0CEB810004100707B0020A2
:102830006C2938B50346154600F3A2803F2912DC07
:1028400038290ADC26296FDC102900F005811629B9
:1028500000F08881042900F016812A461846BDE858
:10286000384060F043BCA1F140022C2AF5D801A009
:1028700050F822F0312A01085B2801085B28010882
:102880005B2801085B2801085B2801085B28010818
:102890005B280108612A01085B2801085B28010800
:1028A0005B2801085B2801088B2A01085B280108C6
:1028B0005B2801085B2801085B280108D32A01086E
:1028C0005B280108232B01085B280108DD2A010889
:1028D000192B0108C92A01085B2B01085B28010894
:1028E000432B0108912A01085B2801085B28010895
:1028F0001F2A0108732B01085B2801086F2A0108B1
:102900005B2801085B2801085B2801085B28010897
:102910005B2801085B2801085B2801085B28010887
:10292000FB2B0108972A0108A1F12702112A94D84C
:1029300001A050F822F000BF1F2A01085B280108FF
:102940005B2801085B280108232A01085B2801088D
:102950005B2801085B2801085B2801085B28010847
:102960005B2801085B280108812A0108692A0108FF
:102970005B2801085B2801087B2A0108752A0108E9
:10298000A02921DC95297FF768AFA1F196020A2AD8
:102990003FF663AF01A050F822F000BF7D2B010885
:1029A0005B2801085B2801085B280108832B0108CC
:1029B000D52B01085B280108E32B01085B280108DF
:1029C0005B280108A32B0108B52923DCA9297FF77F
:1029D00044AFA1F1AA020B2A3FF63FAF01A050F885
:1029E00022F000BF9D2A01085B2801085B2801082E
:1029F000C32B01085B2801085B280108A32A0108F2
:102A00005B2801085B2801085B2801085B28010896
:102A10001B2C0108A1F1D002022A3FF61EAF0124AF
:102A20008DE0A91E854B4D424D4183F8D550F6E708
:102A3000AA1E5542814C554184F82B5D5EF0D0FCB6
:102A40007F4A94F82B1D7F4B002908BF13467E4A0E
:102A5000062157F03DFEE2E70A21FFF757FDDEE7CA
:102A60002A4601211846F8E72A460421FAE72A46B1
:102A70000321F7E72A460C21F4E72A460F21F1E764
:102A80002A460021EEE70B21E7E72A460D21E9E778
:102A90002A460521E6E72A461521E3E72A461121C1
:102AA000E0E7AB1E5A425A41644B93F8D01A914268
:102AB000B5D083F8D02A5EF093FC644A644B022DB3
:102AC00008BF1346634AC3E729461846FFF78AFD45
:102AD000A5E729461846FFF737FDA0E7574CC5B1D3
:102AE000022D0BD1012384F8283DD4F8C8000368D7
:102AF0005B6A984710B1584800F066FB5EF070FCC6
:102B0000524A94F8281D524B002908BF1346534AD5
:102B10009EE784F8285DE8E729461846FFF736FD6A
:102B20007DE7012445B1022D09D1444BC3F8284A61
:102B3000002283F8182B02E0404BC3F8285A2046A5
:102B400038BD01242DB1022DF9D1454B83F8E44164
:102B5000F5E7434B83F8E451F1E729461846FFF7C0
:102B60004DFD5CE7022A7FF45AAF3B4808F040FA7B
:102B700055E75FF0E1FE5FF069FE50E72A46072166
:102B800070E71846294660F0E1F936487AF0D8F83F
:102B9000044600283FF443AF284B0122C3F8282AFB
:102BA000C6E7264BD3F8E83A002B3FF438AF0124B0
:102BB00025B1022DC3D183F82C40C0E783F82C50F7
:102BC000BDE7022D7FF42BAF9FED270A2248FBF7CC
:102BD00055FC24E7022D7FF422AF1F480EF04CF87D
:102BE0001DE701242DB1022DA9D1144B83F82A4DE4
:102BF000A5E7124B83F82A5DA1E7022D12D10F4DF4
:102C0000D5F8C8000368DB6B9847044678B101210A
:102C1000A5F5A04002F08CFE91E7144829468AF001
:102C2000EBF9FCE60C48002102F082FEF7E65EF0CC
:102C3000D7FB0F4A042157F04BFDF0E6707B0020D4
:102C400080DD0C08CBC50C0888DD0C08D4AF0C085F
:102C500044EE0C0898DD0C08702B0020A4DD0C0855
:102C6000704B00200085002000000000787B0020D1
:102C7000B7DD0C0810B599B104681168416004B95A
:102C80000160126801681B68521A9A4202D800213A
:102C9000084610BD017A012381F001010372F7E7B4
:102CA000037A3BB144682CB11368029A12681B1B6B
:102CB0009342ECD90023C0E90033EFE70023C0E9D9
:102CC0000533C0E908338385037780F828307047DF
:102CD000F0B52DED028B044687B09F48B0EE408AD8
:102CE0000F467AF037F840B1236933B1206B00F515
:102CF0000E7010F0E5FA054638B12046FFF7DEFF0A
:102D0000002007B0BDEC028BF0BD236B934E93F90E
:102D10003C22002A1DDD93F8A032D3B1D6F8342D21
:102D2000002AEAD12369D4ED007A991E4842F5EED3
:102D3000C07A4841F1EE10FA84F82C0024D8C4E996
:102D40000822C4E9052284F82D2084F8282022775F
:102D5000D7E7D6F8C80003689B6B984718B196F878
:102D60000037002BDAD07E4800210EF005FBDFEDA6
:102D70007D7AB4EEE70AF1EE10FACFDA784803F084
:102D800093FB0028CAD1B8E76FB1F4EEC87AF1EE30
:102D900010FA3BDD236BD3F8C432DB0403D5724851
:102DA00015F052F8074684F82D708BF0C9FDD4ED6C
:102DB000027A9FED6E7A039067EE877AFCEEE77AEF
:102DC00017EE903A5B000593B4F90630CDED047A26
:102DD000002B1DDC0023C4E9083384F8283094F963
:102DE0000430002B40DC0023C4E90533237794F83A
:102DF0002C00002885D194F82D00002881D194F86A
:102E0000280000287FF47DAF207F7AE71746CAE7C5
:102E10000421534800F0A4FCB4F9063007EE903AC0
:102E2000F8EEE77A05ABF4EEC07AF1EE10FA009313
:102E3000CCBF0121002104AB03AA04F12000B0EEB5
:102E4000408AFFF717FF0028C9D05EF0C9FA07468D
:102E500018EE100AF9F750FB454ACDE900010421AC
:102E6000384657F035FCBAE7424F9FED437AD7F822
:102E70005026DFED426A07F58051D1EDDB7A82EA18
:102E8000E270B0EE476AA0EBE270A7EEA66A07EE2A
:102E9000900AF8EEE77AF4EEC67AF1EE10FA56D818
:102EA000D7F8540691EDDC6A07EE900AA6EE267A72
:102EB000F8EEE77AF4EEC77AF1EE10FA47D591ED25
:102EC000DD6A9FED2F7AA6EE267AF4EEC77AF1EE50
:102ED00010FACCBF4FF0010C4FF0000C642113FB33
:102EE00001F1D6F81837D21A002AB8BF52428A42E6
:102EF00030DAD7F85426D6F81C37D31A002BB8BFCF
:102F00005B428B42ACBF0023012304F11400BCF1EF
:102F1000000F01D183F0010505AB009303AA04ABB8
:102F20002946FFF7A7FE00283FF461AF5EF058FA8C
:102F3000D7F85016D7F85426642392FBF3F291FB8E
:102F4000F3F3009204210F4A57F0C2FB4FE74FF012
:102F5000000CC3E70023D8E700850020707B002029
:102F6000702B002000000034C83F002000007A448D
:102F7000B0DF0C08703B00200000FA430000C8429C
:102F80000000FAC3C1DF0C0873B58289036BD20756
:102F900004466CD493F93C22002A03DD93F8A02266
:102FA000002A64D1524DD5F8C810A5F1880291428B
:102FB0005DD0A5F58045B3F90860D5F8503607EE29
:102FC000903AD5F85436B8EEE77A07EE903AF8EE34
:102FD000E77A6846CDED017A8DED007A30F0D0F9D0
:102FE000730007EE903AF8EEE77AB0EEC00AF4EE1E
:102FF000C07AF1EE10FA42D4236B93F8F1223AB37F
:1030000007EE906AF8EEE77AF4EEC07AF1EE10FA85
:103010001EDB002183F8F112236B586B82F0C0FB9A
:10302000236B9FED347ADA6BD2ED067A05F65C02FB
:1030300067EE877A92ED007AF4EEC77AF1EE10FA35
:1030400006D5986B84F00CFE236B986B84F0A2FB82
:10305000A389226B13F0020302D192F8F11299B9FD
:10306000002382F8F232236B93F8F10205E000208E
:1030700083F8F102236B83F8F20202B070BD236B78
:10308000012283F8F122B7E705F27471D1ED007ADD
:103090009FED197AF0EEE76AF4EEC76AF1EE10FAE6
:1030A000DFDD05F26C71D1ED006A9FED146AB0EEC0
:1030B000E67AB4EEC67AF1EE10FAD2DD05F5EE61ED
:1030C00091ED007AB0EEC77AB4EEC67AF1EE10FA5E
:1030D000C7DD67EEA67AF5EEC07AF1EE10FAC0D53C
:1030E000D5F8543606498B42ACBF00230123B8E71C
:1030F000707B00200AD7233CC2B8323E920A063FBA
:103100006CEEFFFF08B5036B93F8F2223AB1DA6A6E
:1031100092F8A020022A03D0002283F8F22208BDF0
:103120000B4B9FED0C0AD3ED007AF5EEC07ADFED84
:103130000A7AF1EE10FAD8BFB0EE670A152060F0F7
:103140000DFFBDE808409FED050A132060F006BFA3
:10315000E442002000A08CC500A08C4500000000C7
:1031600000F5A040D0F8C80003681B6C18470000A9
:1031700000F5005393EDFC7A00F5A040B5EEC07A5F
:10318000F1EE10FA5DBFD0F8FC38DFED086AD3ED40
:10319000017AD0F814095FBFF8EEE77AE7EE267AF5
:1031A000FDEEE77A17EE900A704700BF0000C842B4
:1031B00000F5005090F8280428B141F001010842C0
:1031C00014BF01200020704700F5A040D0F814394A
:1031D000C0F830390023C0F83439704700F5A040FA
:1031E0004A68C0F830290B78DB0741BFD0F8FC38BB
:1031F0005B689B18C0F830397047000000F5A040AC
:10320000D0F830391944C0F83019704710B54B6800
:10321000516800F5A0448B42D8BF0A46D4F8300963
:10322000CCBF1A4619462DF06FF9C4F8300910BD0D
:1032300010B50446414869F059FA10F0080217BF6A
:103240003F4BDFED407A93ED977AD3ED997A1FBF2C
:1032500077EE877A9FED3C7A012267EE877A10F04D
:10326000010317BF364B9FED377AD3ED996A93ED83
:10327000967A1CBF37EE667ADFED336A04F50051AB
:1032800018BF27EE267AD1EDFE6AF5EEC06A18BFA8
:103290000123F1EE10FA4BDD294A9FED2B6AD2EDA6
:1032A000FE6A66EE866AF4EE676AF1EE10FA58BFBF
:1032B000F0EE667AF3B11A4604F5A043D3F8FC1891
:1032C000D1ED016AD3F83019F8EEE66A76EE876A36
:1032D00007EE101AB8EEC77AF4EEC76AF1EE10FAEC
:1032E000D8BFB0EE667ABDEEC77A17EE101AC3F8F3
:1032F00030190AB304F5A044D4F8FC3893ED017AF0
:10330000D4F83039B8EEC77A77EE277A07EE103A5C
:10331000B8EEC77AF4EEC77AF1EE10FA58BFB0EE05
:10332000677ABDEEC77A17EE103AC4F8303903E079
:10333000002ABFD1002BBFD110BD00BFC04D00205F
:10334000704B0020000000000000C84200F5A040C3
:103350000023C0F83439704713B5002304461046E3
:1033600001AA01931BF0FCFD034648B1DDED017A93
:103370009FED177A67EE877AFDEEE77A17EE903ABF
:1033800004F5A041D1F80427C1F83439042A1DD02E
:1033900004F50054B4F92224002A14DD83EAE37012
:1033A000A0EBE37007EE900A9FED0A7AF8EEE77A59
:1033B00067EE877A07EE102AB8EEC77AF4EEC77A7E
:1033C000F1EE10FA02D50023C1F8343902B010BD75
:1033D0000000C8420AD7233C0B78D1ED017A00F5F2
:1033E000A04013F0010F1CBFD0F8FC3893ED017A18
:1033F000F8EEE77A18BFB8EEC77A00F6141318BFD4
:1034000077EE877A93ED007AB8EEC77AB4EEE77A72
:10341000F1EE10FACCBF0120002070477047000089
:1034200000F50053B3F9DA3300EE103A00F5A0438B
:1034300000F59C40D3F8C82028308242B8EEC00A7C
:103440000CD1D3F80427042A02D093F8B9262AB164
:1034500003F50463D3ED007A30EE270A70470000CD
:10346000014608B501F5A041FFF7DAFF01F6141394
:10347000D3ED007A9FED057AF8EEE77AE0EE477A31
:10348000FDEEE77A17EE900A08BD00BF0000C842C3
:1034900010B5044604F5A044FFF7E2FFD4F8303934
:1034A000181A10BD70B504462DED028B04F5A04529
:1034B000FFF794FEDFED340A40F24310B7EE001A36
:1034C0000E462CF081FFD5F83429534207EE903A8E
:1034D000F8EEE77AD5F8303967EE807AB0EE408AB8
:1034E000FDEEE77A17EE901A1944C5F8301904F585
:1034F0001053D3ED096AF5EEC06AF1EE10FA3FDD24
:10350000002A3DDD2046FFF7C3FF9FED207A07EE3E
:10351000900A66EE876AF8EEE77AF4EEE67AF1EE64
:1035200010FA2DD531462046FFF758FE04F5B2417A
:10353000324610312046FFF70FFFD5F834295342A9
:1035400007EE903AF8EEE77AD5F8303967EE887AE8
:10355000B5EEC08AFDEEE77AF1EE10FA17EE901A9A
:103560001944C5F830190BDD07EE902AF8EEE77A1A
:1035700087EE887ABDEEC77A17EE103AC5F834396F
:10358000BDEC028B70BD00BF000000000000C8C28F
:10359000014608B5FFF744FF01F5B240D0ED107ABF
:1035A00037EEC00ADFED047A20EE270AFDEEC07A7E
:1035B00017EE900A08BD00BF0000C8422DE9F04197
:1035C00000F5B24800F5B24508F110082035044670
:1035D000294640461BF038FF04F5A04606F5D463A3
:1035E00004F5B2472A46394683ED000A40461BF0EF
:1035F00061FE06F2A463DFED210A83ED000AB7EE57
:10360000001A76202CF0E0FE04F53A5383ED710A9F
:103610002046FAF7C5FED6F8C80003685B689847ED
:103620000B280BD006D80A280FD00023C6F834394F
:10363000BDE8F0810E38C0B20128F6D829462046F0
:10364000FFF7CAFE0028F0D011E029462046FFF718
:10365000C3FE30B90A484FF48041FBF7CDF900288A
:10366000E3D12046FFF794FFB0F5FA6FE6DD2A4676
:1036700039462046BDE8F041FFF76EBE000000006D
:10368000702B002010B500F5A04300F58054D3F84E
:10369000242993F820399FED146A13F0010F07EEE7
:1036A000902A08BFD4F8C836F8EEE76A08BF07EEDC
:1036B000903A66EE866A04BFF8EEE77AE7EEC66AED
:1036C000FFF7CEFE04F5D96393ED000A07EE900AEA
:1036D000B8EEC00AF8EEE77A26EE400AA7EE860AB0
:1036E00030EE660A10BD00BF0AD7233C38B5044649
:1036F000FFF75EFD78B904F5B345583528460AF062
:1037000095F928B3284609F03DFD08BB2046BDE8E1
:103710003840FFF7B7BF04F5005595F8F83DDB07D3
:1037200004D505F6146595ED000A38BD04F5B340DF
:1037300058300AF09DF90028DDD095F8C21D04F537
:1037400070604CF081FE0228D5D19FED040AECE7B1
:1037500004F5B24494ED100AE7E700BF0000000052
:103760000022FFF7C3BF000010B504468BF0E8F855
:1037700004F50053D3F80C3EC01A41F28833984246
:103780000FD802212046FFF713FD50B104F5A043E6
:10379000D3F80437042B04D104F5385494ED000A0F
:1037A00010BD9FED010AFBE70000000008B52DEDFC
:1037B000028B00F5A0430146D3F8FC28D3F830393A
:1037C0005268DFED0D8A9B1A08EE103AFFF728FECB
:1037D000B8EEC88A0846A0EE288AFFF7C5FFBDEEFE
:1037E000C88AB8EEC88AA0EE288AFDEEC87ABDEC79
:1037F000028B17EE900A08BD0000C842F0B52DED0F
:10380000048B00F5005489B000F5706694F8C21D71
:103810000391054630464CF017FE039907463046A3
:103820004CF024FE042F0399B0EE408A21D10023EE
:1038300005A88DED050A0693079330F021F805F5EC
:10384000BB5005A918302DF0E9FEDFED987A8DED1B
:10385000050AB4EEE71AF1EE10FACDED060A8DED89
:10386000071A06DB05F5805393F8D47617F00107A5
:103870000CD194F8F83D002262F3000384F8102E76
:1038800084F8F83D09B0BDEC048BF0BD94F8F83D28
:103890009A075FBF43F0020384F8F83D04F6FC5337
:1038A00083ED008A04F6146383ED001A94F8103E49
:1038B000092B79D804F61863D3ED000A9FED7C9AA2
:1038C000B0EE480A2CF06EFC00BB04F6FC5394F8F2
:1038D000C21DD3ED008A30464CF0E6FD07EE900A9B
:1038E0009FED747AF8EEE77A78EEC88A67EE877A09
:1038F000F0EEE88A67EE897AF4EEE78AF1EE10FAE4
:10390000C2BF94F8103E013384F8103E04F61863E9
:1039100094F8C21DD3ED008A30464CF0C5FD07EE89
:10392000900AF8EEE77A9FED647A67EE897A78EE8E
:10393000C88A67EE877AF0EEE88AF4EEE78AF1EE5D
:1039400010FA02DD002384F8103E04F6186383EDBC
:10395000008A94F8F83DDA0794D52846FFF792FEDE
:1039600004F6146696ED008A30EE488A8AF0E8FF85
:10397000D4F80C2E41F28831821A8A42034605F5AA
:10398000385204F6046158D982ED008A284681ED48
:10399000008A0221FFF70CFC18B105F5B045EA6C6E
:1039A000AA64C4F80C3E6DE794F8F83D43F00103B7
:1039B00084F8F83D05F5A043D3F80467D3F8C82090
:1039C000301F05F59E43464203F13C0346419A42AF
:1039D00012D005F59E4358339A420DD005F59C430D
:1039E00028339A4209D1354B05F5B340B3F8661731
:1039F000583009F0E3FB00B13E4694F8F83D590712
:103A0000A3D4002EA1D002212846FFF7D1FB002825
:103A10009BD043F0040384F8F83D04F6146305F5E5
:103A200056561868F8F768FD1036CDE90001244AAB
:103A30000621304656F04CFE87E79FED1F0A92EDB7
:103A4000007ADFED207A28EE008AA7EE278A82ED41
:103A5000008AC4F80C0ED1ED007A38EE678AF3EED6
:103A60000E7AB0EEC88AB4EEE78AF1EE10FA7FF76C
:103A700009AF94F8F83D5B070CD53068F8F73CFDCA
:103A800005F556541034CDE900010F4A06212046B1
:103A900056F01EFE05F5375024220021383009B0BB
:103AA000BDEC048BBDE8F040B0F0B2B900000034CA
:103AB0000AD7233CCDCC4C3DCDCC4C3E707B002076
:103AC000D8DF0C08CDCC4C3FF5DF0C0838B52DED18
:103AD000028B0D460446FFF7D5FD002320462B70D0
:103AE000B0EE408AFFF740FE0221204638EE400A41
:103AF000FFF75EFB28B104F5005494F8F80D00F0D0
:103B00000100BDEC028B287038BD000070B50B7849
:103B100003F00503042B05460C46164615D105F5A2
:103B2000A04553F03FF9B2B24FF4801153F0F2F8D0
:103B3000D5F8FC28636852689B1A13F5FA7FC8BF52
:103B40006360237843F00103237070BDF8B500F57E
:103B5000805300F5A047D3F8C866D7F8C856B542D9
:103B6000044618D00D4A1268D26A92F89C2092B18D
:103B700000F5B241751B25222031FFF7C7FF07EE84
:103B8000905AB8EEE70ADFED067A04F53A5020EED7
:103B9000270A7DF0C7FFC7F8C866F8BD6C2B002068
:103BA0000AD7233CF8B500F5A044064694F8BB7646
:103BB0008C4600F5B245002F4FD004F512630FCBB1
:103BC00085E80F00012384F8BC369CE80F0004F55B
:103BD000126787E80F00D4F8283906F5B247203776
:103BE00093B9D4F82C397BB9D4F81839D4F82429EE
:103BF000C4F82839D4F81C39C4F82C3922B9D4F8BF
:103C0000141938461BF0F6F8394628223046FFF7DB
:103C10007DFF94F8201911F0040102D138461BF001
:103C20007BF906F5B2403A46294610301BF078FB86
:103C300028B104F5116494E80F0085E80F003046C0
:103C400006F064FC3046FFF7B9FC304607F044F854
:103C50003046BDE8F840FFF783BA04F511630FCB97
:103C600085E80F00012384F8BB3684F8BC76ACE706
:103C7000F8B500F500530446B3F98233002B0E4625
:103C800034DB0B7813F0020F14BF4FF0FF33012326
:103C900004F5A04504F5B24785F8D83805F5116359
:103CA0000FCB87E80F0096E80F0005F5126787E84D
:103CB0000F0004F5B241572220312046FFF726FFBE
:103CC0002046FFF781FA20460026FFF777FC2046C2
:103CD00007F002F885F8BC66C5F8DC6885F8C166AF
:103CE000204606F013FC85F81A6BF8BD4FF0FF3341
:103CF000CEE700002DE9F043364B1B6885B0054642
:103D0000D86AF9F709FC002861D105F5005393F949
:103D1000903D5A1C54D0002B05F5866711DD95F8AF
:103D20004124242107EE903A01FB027292ED0B7AB6
:103D3000F8EEE77AB0EEC77AB4EEE77AF1EE10FA71
:103D40003EDC05F5805305F5A25693F8D43613F002
:103D5000010406F1180629D0C3F340089B0732D4AA
:103D600095F8E41395F828444FF0B00909FB015188
:103D700091F8C1314CBB022B18D968461BF034F8BE
:103D80006946304615F00CF8044678B195F8E433EE
:103D900009FB03534246D3F8D01168461BF02AF8BA
:103DA00015F0D4FA694614F0E9FE0446384617F0D7
:103DB000C7FD304614F000FE2846FAF7EFFD204616
:103DC00005B0BDE8F0830024F0E74446EEE70020AC
:103DD000F6E700BF6C2B002038B50C4B1B6805467E
:103DE000D86A0C46F9F798FB10B10024204638BD7C
:103DF00015F0ACFA214614F0C1FE04460028F4D0B8
:103E000005F5AE40283030F055FBEFE76C2B002075
:103E1000F0B500F5A045002385F8BB3685F8BC3623
:103E200005F51163044600F5B24600EE101A0FCBFB
:103E300087B086E80F0002AE04F5B242B8EEC00AC1
:103E40003046174910324CF073F896E80F0005F52C
:103E5000126787E80F0004F5B24140F25712203193
:103E600020460191FFF752FE01992046FFF7D6FA4E
:103E700001992046FFF7B2F904F500532046B3F943
:103E80008233002BB4BF4FF0FF33012385F8D838BD
:103E9000FFF794FB204607B0BDE8F04006F01CBFDA
:103EA000A063002010B5034904464CF041F82046B9
:103EB00010BD00BFA0630020F8B500F5A04404F5D4
:103EC000116305460E4600F5B2470FCB87E80F0099
:103ED00006F108012846FFF765FEB388D4F82429C7
:103EE00003EB830303EB83039B001BB2002BD8BFC0
:103EF0004FF4C873A4F8B636D4F8FC385968521A8F
:103F0000C4F888269A680A32C4F82829DB680A337C
:103F1000C4F82C390023C4F89C3684F8B83684F8E9
:103F2000CC36C4F88C3605F5AD4300221A604FF04C
:103F3000FF33C4F8783695F8412405F586632421CB
:103F400001FB023304F5D664DB6A2360F8BD000090
:103F500070B50E4608310546FFF724FEB38805F517
:103F6000A04443B3642213FB02F3C4F88836B4F9C7
:103F7000B636002BD8BF4FF47A7305F53750D8BF4B
:103F8000A4F8B636242200213830AFF041FF04F502
:103F9000146305F5B04093ED000A3146403087F0D8
:103FA000A3F8D4F80437072B0CD128460421BDE828
:103FB0007040FAF7C3B9D4F88836002BD7DC40F646
:103FC000B833D2E770BD000030B5083104460FC9E0
:103FD00085B06D4685E80F0004F5B24110312846E2
:103FE0001BF03AF820462946FFF7DCFD04F5A04413
:103FF0000123C4F8F03005B030BD00000B7A00F5A5
:10400000A04013F0020F14BF4FF0FF33012380F8DC
:10401000D83870477FB501F1080305460E460FCB2F
:104020006C4684E80F0005F5B241103120461BF0C4
:1040300013F821462846FFF7B5FD31462846FFF71D
:10404000DDFF04B070BD00007FB501F10803044638
:104050000E460FCB6D4685E80F0004F5B2411031D6
:1040600028461AF0F9FF29462046FFF79BFD204617
:104070003146FFF7C3FF337907EE903A337E9B0753
:1040800048BF9FED0C7AF8EE677A04F5A04448BF6C
:1040900067EE877A9FED087A67EE877AFCEEE77A1B
:1040A00017EE903AC4F8D0380123C4F8F03804B0C1
:1040B00070BD00BF0000803B00A00C477FB501F140
:1040C000080304460E460FCB6D4685E80F0004F545
:1040D000B241103128461AF0BFFF29462046FFF7AB
:1040E00061FD20463146FFF789FFB38804F5A044FF
:1040F0004FF47A725343C4F8E8380123C4F8F03817
:1041000004B070BD2DE9F34100F5B24520350446F9
:104110000E4600F5B24029461AF05EFF04F5A047AE
:10412000C0B94FF0FF33C7F8783606F108084046AB
:104130001AF08AFE032802463AD1F16828461AF09E
:1041400059FEB388C7F8F038204602B0BDE8F04108
:10415000FFF7FCB824F090FBF9F752FE012812D9C2
:104160004FF0FF33C7F8783624F086FB90F8C4325E
:10417000DFED140AB02202FB030090ED300A28465E
:104180001BF008FAD1E704F58058D8F858062CF04F
:10419000EFF808F5CB63C7F87806D3ED007A9FED0A
:1041A0000A0ADFED080AF8EEE77A27EE800AE6E76A
:1041B00001AA002140461AF053FE0028C1D00199FF
:1041C0000022BBE700007A440AD7233C7FB501F107
:1041D000080304460E460FCB6D4685E80F0004F534
:1041E000B241103128461AF037FF29462046FFF722
:1041F000D9FC20463146FFF701FF04F5A044002317
:10420000C4F8F03804B070BD37B504460D468AF0E6
:1042100097FB2062D5ED027AF5EEC07AF1EE10FA46
:1042200015DD9FED127A67EE877AFCEEE77AC4ED32
:10423000077A5DF0D5F8E2694FF47A73B2FBF3F3D5
:104240000B4A062103B0BDE8304056F041BA68F091
:104250009BF80023009395F90D2095F90E3095F900
:104260000C1068F02DF8E061E3E700BF00007A442D
:1042700018E00C082DE9F0432DED028B85B00446C3
:1042800015F064F814F04AF904F5805304F5A046DB
:1042900093F850390BB9002877D0D6F87836013327
:1042A00073D1D6F89C36002B4BD08AF049FBD6F858
:1042B0009C36C01AB0F5FA6F67D394F8E423DFEDAB
:1042C0005F7A9FED5F8A4FF0B00808FB024292EDE3
:1042D000780A20EE270A2CF063F804F5AD49D9EDF1
:1042E000007A30EE670A2CF05BF8DFED567A20EEAC
:1042F000080A04F5565720EE270A2BF0F9FFFDEEC9
:10430000C07A103717EE905AC6F87856D9ED007A71
:1043100067EE887A17EE900AF8F7EEF8CDE9020119
:1043200094F8E43308FB0343D3F8DC01F8F7E4F82E
:10433000454ACDE900012B460621384656F0C8F91A
:1043400023E004F59070F9F75BFD02281DD994F87D
:10435000E433B02202FB034393ED777AF1EE047A63
:10436000B4EEE77AF1EE10FA0FDD384B1B68D86A2D
:104370000368DB699847012803D08AF0E1FAC6F8A0
:104380009C06D6F89C36002B8FD104F54053D6F806
:104390007816D3F8AC074A1C036846D01B6B9847C5
:1043A0002B4810F061FC20B104F5AE40283032F00B
:1043B000C5FA2046FFF7ECF8D6F888368342054662
:1043C00036DA07EE905A9FED237AF8EEE77A04F595
:1043D000565767EE877A103717EE900AF8F78CF881
:1043E0001D4ACDE900013846062156F071F9012534
:1043F0004FF0FF33C6F8783686F8B85606F51163E5
:104400000FCB04F5B24406F5126784E80F0087E885
:104410000F00124868F034F9002386F8BB362846AE
:1044200005B0BDEC028BBDE8F0835B6B9847B7E746
:10443000074810F0F9FB0028C3D1F1E735FA8E3CAC
:10444000E02E65420000C84228E00C086C2B0020DA
:10445000702B00200AD7233C4CE00C08C04D0020F4
:104460002DE9F04100F5B2473D4620350446294686
:1044700038461AF0B1FD04F5A04604F5405830B3B3
:10448000D6F878164B1C22D0D8F8AC0703681B6B03
:104490009847D6F8F038012B47D0D6F8F038022BE1
:1044A00006D12046FEF7DCFFD6F82439984243DDDA
:1044B0002046FEF7D5FFD6F82439C01A0028B8BF29
:1044C0004042B0F5FA7FCCBF0020012035E004F572
:1044D000B240294610301AF0B7FFDFED197AB4EE7A
:1044E000E70AF1EE10FA16D5384629461AF07CFE96
:1044F0009FED147ADFED140AF6EE007AE0EE077A0B
:1045000028469FED120AFDEEE77AF8EEE77A27EEED
:10451000800A1BF03FF8D8F8AC079FED0D0A03683E
:104520002A469B6A39469847B3E72046FEF798FF2C
:10453000D6F824399842B0DB0120BDE8F08100BFF5
:1045400000004843A00CB345000096430AD7233C23
:104550000000000073B5394CD1ED026AD4F814396B
:104560009FED377A07EE903AF8EEE77A0546D7EEF8
:10457000876A0E46F5EEC06AF1EE10FA08DD5CF0CF
:104580002FFF304A062156F0A3F8012002B070BD7B
:10459000D1ED037AF5EEC07A04F5D364F1EE10FAAA
:1045A00094ED006A12DDF4EEC67AF1EE10FA0DD544
:1045B0005CF016FF05462068F7F79EFF224ACDE91A
:1045C00000010621284656F083F8DEE7DFED1F7A6A
:1045D000337CB4EEE76AF1EE10FA54BFB0EE677ABE
:1045E000B0EE467A0BB90020D0E7B5EEC06AF1EE26
:1045F00010FA0CDC86EE876A03EB830307EE903A31
:10460000F8EEE77AF4EEC67AF1EE10FAEBD595F80B
:104610002440002CE7D18AF093F9AB6AC01A337CAE
:104620004FF47A7253439842DDD9012385F8243040
:104630008AF086F9A8622046A8E700BF707B0020B8
:104640000AD7233C68E00C0879E00C080AD723BCA1
:1046500038B5054679F0AAFD78F07CFB044640B9F0
:104660008AF06EF92B6AC01AEB69984284BFEC613C
:104670000124204638BD000038B504460D468AF0B6
:104680005FF904F5A0439FED077AC3F8F408D5ED70
:10469000027A67EE877AFDEEE77A17EE902AC3F882
:1046A000F02838BD00007A4410B504468AF048F975
:1046B00004F5A043D3F8F428801AD3F8F0289042E8
:1046C0004FF0000084BFC3F8F008012010BD0000C7
:1046D00000F5A04303F5D461D3F8F02891ED007AFA
:1046E00022EAE27207EE902AF8EEE77A0020B4EEB2
:1046F000E77AF1EE10FA44BFC3F8F00801207047E2
:1047000010B500F5005300F5A040B3F98233002B3B
:10471000B4BF4FF0FF33012380F8D83800F512649E
:1047200000F511600FC884E80F0010BD38B50446CD
:104730002DED028BF0EE408AB0EE608A09B30129BC
:104740005CD0B5EEC08AF1EE10FA67DDDFED347AA9
:10475000B4EEE78AF1EE10FA60D8FCEEC87A04F500
:10476000565017EE903A2F4A0621103055F0B0FF00
:10477000FDEEC87A04F5005417EE903A84F84F33F2
:104780003AE0F8EE000A2BF00DFD40B104F5A0442C
:104790004FF0FF33C4F80031BDEC028B38BD04F597
:1047A0000053B3F9582307EE902AF8EEE77AF4EEB7
:1047B000E87AF1EE10FAC4D8B3F95A3307EE903A1A
:1047C000F8EEE77AF4EEE87AF1EE10FAB9DBDFED15
:1047D000147A154A68EEA77A04F5A043FDEEE77A4D
:1047E00004F55650C3ED407AFCEEE87A062117EE48
:1047F000903A103055F06CFF0120CDE7FCEEC07A06
:1048000000F5565017EE903A084A0621103004F58C
:10481000005455F05DFFC4EDD98AEDE70020BBE7F9
:104820000000C842BFE00C0898E00C08ACE00C089F
:10483000D1F80D3000EE903AD1F80930097A00EE47
:10484000103AFFF773BF000070B58B88012B044648
:104850000D4611D100F590763046F9F7D1FA0228CD
:104860000AD994F8E413B02303FB01612046AC316C
:10487000BDE87040FFF7B0BA14F068FD05F108011B
:10488000BDE8704014F07AB9F0B500F5A0470024F7
:1048900089B0054687F8C14608460E462FF01CFC35
:1048A000A0B3012387F8B83605F54053D3F8AC0719
:1048B0000368DB6B984787F8BF46C7F8DC4803A856
:1048C0001AF092FAB7F864174FF6FF73994208BFCF
:1048D0002146013105F5AE4001AA89B2283031F0F8
:1048E000AFFBF0B1BDF80630A3F1150253425341BE
:1048F00087F8B93650B105F5B340BDF80610583009
:1049000008F05CFC10B1002387F8B93673885E2B81
:104910004ED8522B07D8103B9AB20F2A22D9002426
:10492000D5E00346E4E7533B0B2BF8D801A252F83D
:1049300023F000BFC94A0108D54A0108E54A010829
:104940001F4901081F4901081F4901081F490108A3
:104950001F4901081F4901081F490108314B01087F
:10496000E54A01080F2BDAD801A252F823F000BF64
:104970004D4A0108874A0108914A01089B4A0108EB
:10498000AF4A0108594A01081F4A01081F49010896
:104990001F4901081F4901081F4901081F49010853
:1049A0001F4901081F490108BF4A0108A54A01081B
:1049B000BD2B1AD8BB2B47D8B22B00F0A7800DD83F
:1049C000702B00F09E80722BA9D1D6ED027AFDEEFD
:1049D000E77A17EE903AC7F8F03835E0B32B9ED15E
:1049E00031462846FFF730FF2EE0D42B00F09380AD
:1049F00040F6B832934200F09680D22B8FD1B38824
:104A0000012B21D803F0010387F8BA3605F556507B
:104A1000B3884B4A0621103055F05AFE14E00023AB
:104A200005F5B34487F8F13658347188204607F00D
:104A30006DFE314628B1204609B0BDE8F04008F0CF
:104A400067B82846FFF738FA012440E006F108016C
:104A50002846FFF7A7F8F7E705F5B34458341521C2
:104A6000204608F0ABFB48B1002387F8F136314609
:104A7000204609B0BDE8F04007F04EBF3146284659
:104A8000FFF766FAE0E731462846FFF7C3FADBE7AF
:104A900031462846FFF7D8FAD6E731462846FFF7D1
:104AA0000DFBD1E731462846FFF790FBCCE705F533
:104AB0009C412922543128460EF032F8C4E7314691
:104AC0002846FFF71FFBBFE7012487F8BF462046B3
:104AD00009B0F0BD002305F5B34087F8F136314643
:104AE0005830A9E705F5B3475837384608F04AFB70
:104AF0003146044618B12846FFF766FAE7E738461C
:104B0000B7E731462846FFF7B7FD9DE7314628460F
:104B1000FFF78EFE98E7B188003918BF01212846BB
:104B200000F006FF90E7317A064807F0EDF98BE7D1
:104B300005F59C4031462830FFF766FB84E700BF4F
:104B4000D0E00C084885002000F5A04200F59C4309
:104B5000D2F8C82028339A4201D1FFF795BE012030
:104B60007047000010B500F5A04200F59C43D2F854
:104B7000C82028339A4204460ED100F59C410822F1
:104B800054310DF0CDFF04F55650044ABDE81040F5
:104B90000621103055F09CBD10BD00BFE0E00C08B0
:104BA0002DE9F04F2DED048B00F5A04505F65823B7
:104BB00093ED008ADFEDD47AB0EEC87AB4EEE77AEE
:104BC000F1EE10FA48BF00F50053DFEDD07A42BF96
:104BD000B3F9823308EE103AB8EEC88AD5F8F0304F
:104BE000B4EEE78AF1EE10FA94BF4FF0FF370127D9
:104BF00099B004460E46F0EEC88A85F8D878052BA1
:104C000016D8DFE813F006002C0067008600C1000C
:104C1000580100F540543A46D4F8AC070368B0EEAA
:104C2000680ADB6A08319847B94806F08FF808B976
:104C3000002041E1B74CD4F8FC38B4F9981A5B680D
:104C4000642201FB0231A4F5A040FFF7E1F8A4F5CE
:104C5000A04005F05BFC0123C5F8F030E8E700F563
:104C600040533A46D3F8AC070368B0EE680ADB6AF3
:104C700008319847D5F8D438002BB8BF5B42012BD8
:104C8000D6DD95F8D9381BB995F8DA38002BCFD096
:104C900004F5BE53D3ED000A93ED010AF1EE600A6C
:104CA000B1EE400AACF0BAFEDFED9B7A20EE270AA7
:104CB00004F5565410EE100A85ED3D0AF7F71CFC7A
:104CC0001034CDE90001954A0621204655F000FD3B
:104CD0000223C1E700F5B24801F1080908F1100804
:104CE000414648461AF0B0FB30EE680AF1EE047A0D
:104CF000B0EEC00AB4EEE70AF1EE10FA00F3E1807C
:104D0000D5F8D4380133022B40F2E5800323C5F8EF
:104D1000F03004F5405306F10808D3F8AC070368F7
:104D20003A46DB6AB0EE480A41469847DFED7C6AB6
:104D30009FED7C7AD5ED3D7A012F18BFB0EE667AF3
:104D400004F5A25377EE877A93ED890A9FED767A80
:104D5000A7EEC70A2BF024FBDFED747AB0EEC00A91
:104D6000B4EEE70AF1EE10FA7FF562AF04F55650A3
:104D7000062110306E4A55F0ABFC0423C5F8F03024
:104D800041462046FEF70EFF06F1080595E80F00A4
:104D900004F5A0489FED679A98ED3D0ADFED660A9D
:104DA0009FED668A08AF0DF1300987E80F0089E8AA
:104DB0000F0030EE090A38461AF0ECFBDFED5E0A10
:104DC00098ED3D0A48461AF0E5FB04F540534A4683
:104DD000D3F8AC07036839469B6AB0EE480A984797
:104DE00095E80F0004F5B34A0DF1400B0AF1580A9B
:104DF0008BE80F00D8ED3D9A504607F0ADFC79EEF8
:104E0000899A04F5B249F0EE400A5846B0EE690AB4
:104E100009F110091AF0BEFB5A46394648461AF005
:104E20007FFA834695E80F0098ED3D0A14AF87E8B6
:104E30000F00F0EE680A30EE090A38461AF0AAFBB5
:104E4000394648462A461AF035FA04F5A25005A913
:104E50001830F0EE408A8DED058A8DED068A8DEDD5
:104E6000078A14F071F8002849D0294648461AF0FC
:104E7000F7F903A905A8CDED040A8DED030A2EF07C
:104E800093FADFED257A20EE270A2BF01DFAB0EE1B
:104E9000C00ABBF1000F3FF4CBAEF3EE0E7AB4EED6
:104EA000E70AF1EE10FA22D50523C8F8F0303146B2
:104EB000504607F031FD012019B0BDEC048BBDE870
:104EC000F08F414648461AF0BFFAB4EEE80AF1EE18
:104ED00010FA7FF515AF04F540543A46D4F8AC0704
:104EE0000368B0EE680ADB6A49469847A0E6F6EE2A
:104EF000007AF4EEE78AF1EE10FAD5DC98E6BBF121
:104F0000000F3FF495AECFE700000034000000B47E
:104F1000702B0020707B0020E02E654208E10C0819
:104F20000000B4420000874335FA8E3CC2B8B23D5F
:104F30002AE10C080000344300007A44000000001D
:104F40002DE9F041074600F5B3408EB05830884651
:104F500008F058F9044650BB09AE07F5A0453046A5
:104F600019F042FFB5F864374FF6FF72934208BF5D
:104F70000023013307F5AE4007AA99B2283031F07B
:104F80005FF8C0B1B8F1000F01D0C5F8D44896E879
:104F90000F0001AC84E80F00D5F82C39009305F51B
:104FA000126595E80E00054803F086F90446204690
:104FB0000EB0BDE8F0810124F9E700BFE0790020E0
:104FC00070B5064606F5A045002105F08BFFD5F823
:104FD000DC487CB9304605F0B9FE10B90024204603
:104FE00070BDD5F8D438012BF8DD89F0A9FCC5F8DF
:104FF000DC08F4E7D5F8F01861B189F0A1FCD5F828
:10500000DC38C01AD5F8E8389842E7D90023C5F84B
:10501000F03801213046FFF793FF04460028DDD029
:1050200006F55650044A0621103055F051FB002376
:1050300085F8C136D3E700BF4CE10C0870B50A46CD
:105040008B88190A137E0546DB0748BF01EB8101F7
:1050500005F5A04448BF4900002605F043FF84F849
:10506000C166284605F072FE10B90024204670BDC6
:10507000D4F8F01851B1D4F8D438D4F8D0289342E9
:10508000F3DD012BF1DDC4F8F06801212846FFF7BC
:1050900057FF04460028E8D005F55650024A06217D
:1050A000103055F015FBE1E764E10C0838B5054612
:1050B00005F5A044898805F015FFD4F8F03883BBC6
:1050C000D4F8D438002BB8BF5B42012B02DC00249B
:1050D000204638BD94F8D92894F8DA3872B9002BF4
:1050E000F5D005F55650D4F814296423062192FB17
:1050F000F3F310300C4A55F0EBFA01E0002BF0D13D
:105100000121C4F8F0182846FFF71AFF04460028CA
:10511000DDD005F55650054A0621103055F0D8FA75
:10512000D6E70021EFE700BF7CE10C089AE10C080C
:1051300010B504460B4808F03FFE48B10A4BDFEDBE
:105140000B7AD3F8143A93ED090A20EE270A10BD22
:1051500004F50054B4F9B03300EE103AB8EEC00ACA
:10516000F5E700BF48850020707B00200AD7233C6C
:1051700038B52DED028B00F5005300F5A045B3F9CD
:10518000B4130029ACBF01234FF0FF330029B8BF8F
:10519000494285F8D838044689B205F0A3FE05F5E2
:1051A000D465204695ED008AFFF7C2FFB5EEC00A30
:1051B000F1EE10FAD8BF9FED0E0ABCEEC00AB8EEB1
:1051C000400AB4EEC08AF1EE10FA0AD804F556503F
:1051D0001030084A062155F07BFA0120BDEC028B05
:1051E00038BD204605F0B2FD0028EFD1F6E700BF3C
:1051F00000000000B4E10C082DE9F04700F5A048DC
:105200002DED028B4FF0FF33C8F8783608F51263A6
:105210000E4604460FCBB588367988B004AF2D0A08
:1052200087E80F001ED004F5B240394603901AF00B
:105230000BF903983946B0EE408A19F0D5FFDFED3F
:10524000547AB4EEE78AF1EE10FA0BDBEBB200EE23
:10525000903ADFED507AF8EE600A20EE270A3846E1
:105260001AF098F904F5405A98F8BC26DAF8AC0719
:105270009FED490A036804F5B2499B6A09F11009D8
:105280002AB33A4604F5B241984704F50053B3F9FE
:10529000B233002B1EDD07EE903A08F5D462F8EE2B
:1052A000E77A92ED007AB4EEE77AF1EE10FA11DDCA
:1052B00004F5B2443A46214648461AF031F8E0B9BE
:1052C0000025284608B0BDEC028BBDE8F0873A46C1
:1052D0004946D9E7D6B9002D3AD1DAF8AC572B6850
:1052E00020461E6AFFF724FF08F29463D3ED000AFC
:1052F0002846B047B0EE408A0CE0002DE0D108F51A
:10530000116898E80F0084E80F00DAE707EE906A6A
:10531000B8EE678A394648461AF096F8B4EEC08A65
:10532000F1EE10FA17DBB8F86437039339464846B4
:105330001AF08AF8BCEEC00A04F55650039B174ACF
:105340008DED000A0621103055F0C2F90125B8E7AD
:105350009FED118ADEE73A4604F5B241484619F05E
:10536000DFFF05460028ABD0B8F864370393394611
:1053700048461AF069F8BCEEC00A04F55650039B83
:10538000074A8DED000A0621103055F0A1F998E783
:1053900000000034E02E654200000000CCE10C0863
:1053A000EAE10C082DE9F0474B881F2B8AB0044630
:1053B0000D466BD80F2B41D804F55650BC4A04213A
:1053C000103055F085F99BE0A3F1BC02182AF3D800
:1053D00001A151F822F000BF015501080155010853
:1053E000B9530108B9530108B9530108B953010869
:1053F000B953010801550108B953010801550108C5
:10540000B9530108B9530108B953010801550108FE
:10541000B9530108B9530108B953010801550108EE
:105420000155010801550108B9530108B953010894
:1054300001550108B953010801550108A3F11002F3
:105440000F2AB9D801A151F822F000BF3D5501083B
:1054500017560108215601082D5601084356010828
:105460004955010813550108B9530108B9530108FA
:10547000B9530108B9530108B9530108B9530108D8
:10548000B95301084D560108375601085E2B21D843
:10549000522B91D9A3F153020B2A8DD801A151F8B7
:1054A00022F000BF575601086956010873560108DB
:1054B000B9530108B9530108B9530108B953010898
:1054C000B9530108B9530108B95301089D560108A1
:1054D00073560108722B00F0DC8007D8702B7FF424
:1054E0006BAF0AB0BDE8F047FFF7DEB8D42B09D8A0
:1054F000BB2B3FF669AFA3F1B202012A3FF65CAFC6
:1055000001204CE0DF2BFBD040F6B8329342F7D0BD
:1055100052E700F5B34658361621304607F0F6F844
:1055200030B1294630460AB0BDE8F04707F0E2BB8B
:1055300020460AB0BDE8F047FEF79CBE29460AB0F7
:10554000BDE8F047FFF758BE00F5B34558351521C3
:10555000284607F033FE28B128460AB0BDE8F047D8
:105560000BF02EB904F5A04504F5B249D5F804377F
:1055700004F5B0464F46072B06F1400607F1200719
:1055800009F110080ED104F5AE440194D5F888361F
:1055900000933A4643464946304685F069FE0AB0D4
:1055A000BDE8F0870DF127018DF827004148FEF78F
:1055B0008DFA05F2C463D3ED007AD5F8A8A605F5F7
:1055C000D363D3ED000A05F2A46330EE670A93EDCE
:1055D000001A8DED070A04F5B3401030CDED060A30
:1055E0008DED051A77F0ACFB0546204600F05CFF18
:1055F0009DF827309DED051ADDED060A9DED070AA1
:10560000CDE90203CDE900A543463A464946304676
:1056100085F084FDC3E7A98805F064FC0020BEE79F
:1056200029460AB0BDE8F047FFF708BD0AB0BDE85B
:10563000F047FFF7C5BC29460AB0BDE8F047FFF7C1
:1056400035BD0AB0BDE8F047FFF792BD0AB0BDE82E
:10565000F047FEF705BF04F59C40294628300AB004
:10566000BDE8F047FEF776BF04F5B3402946583051
:1056700059E704F5B3465836304607F083FD08B9BC
:1056800030466AE729462046FFF78AFA0028F7D114
:1056900085E70AB0BDE8F047FFF71AB804F59C406B
:1056A000294628300AB0BDE8F047FEF7D1BF00BF59
:1056B00008E20C08702B002070B500F5A04200F540
:1056C0009C43D2F8C82028339A4205460E4602D0A1
:1056D0000024204670BDFFF765FE04460028F7D081
:1056E00005F556503188103059F03EF9F1E70000C9
:1056F00021F04003152B04D0A1F15E03584258411C
:10570000704701207047000000F5A04200F59C435F
:10571000D2F8C8002833984205D1B2F866375B1A30
:10572000584258417047002070470000192962D83C
:10573000DFE801F00D1115191D2125282C613034E9
:1057400037553A3A3D404346494D6151595D00F560
:105750009D404830704700F59A401C30704700F576
:105760009A403830704700F59A405430704700F541
:105770009A407030704700F59B402C30704700F520
:105780009B40E6E700F59B406430704700F59C4085
:105790000C30704700F59C402830704700F59C4065
:1057A000E3E700F59C40E4E700F59D40F0E700F5F5
:1057B0009D40E2E700F59D40E6E700F59E4070471A
:1057C00000F59E40C9E700F59E403C30704700F56B
:1057D0009E405830704700F59E407830704700F585
:1057E0009F403030704700F59F406C30704700F5A7
:1057F0009F401430704700207047000000290DDBE7
:10580000074890F8F42DCBB29A4207D3D0F8F03D78
:105810000122595CA0F500500DF052BA704700BF4C
:10582000704B00202DE9F34100F5005300F556556B
:1058300093F8C03D03F0010603F0020803F00407EB
:105840005B07044605F1100535D01F4A062128469E
:1058500054F03EFF26B104F54450043079F0B4FA18
:10586000B8F1000F04D004F549501C3079F028F845
:1058700027B104F54E50343079F0D0FE04F5A04441
:10588000012384F8293D114A114B1249B8F1000F48
:1058900008BF1A46002F08BF1946CDE900210E4A5D
:1058A0000621002E18BF134628460C4A54F010FF5C
:1058B00002B0BDE8F0810A4A0621284602B0BDE8E0
:1058C000F04154F005BF00BF35E20C082AE20C0895
:1058D000F8CB0D0831E20C0824E20C0846E20C0873
:1058E00058E20C0810B5044600F54450043079F035
:1058F00097FA04F549501C3079F00EF804F54E5033
:10590000343079F0C5FE04F5A04393F8292D5AB13F
:10591000002283F8292D04F55650044ABDE81040B2
:105920000621103054F0D4BE10BD00BF78E20C0840
:1059300009B1FFF777BFFFF7D5BF000000F5A04220
:105940000346D2F8C810084881420AD092F8D50020
:1059500040B903F59C432833994203D192F8BA0623
:1059600070470020704700BF387A002010B5044609
:1059700088F0E6FF054BD3F8E830C01A642804D855
:105980002046BDE810405CF051BF10BD707B002088
:1059900010B500F53654D4ED0C7AF5EEC07AF1EE80
:1059A00010FA8AB04FF0000304F1300445D9079390
:1059B0000893099306AB019300F5A25007AB00933F
:1059C00003AA05AB04A9183013F05EF930B3DDED7E
:1059D000080A9DED070AABF085FEDDED090AABF084
:1059E00081FED4ED007A9DED047A77EEA76AB4EEDD
:1059F000E70AF1EE10FAF4EEC76AACBF012000200E
:105A0000F1EE10FA0CD802309DED037AF4EEC77A6D
:105A1000F1EE10FA0CD8003818BF01200AB010BD02
:105A2000F4EEC77AF1EE10FA9CBF0130C0B2EBE79A
:105A3000012894BF00200120F0E70020EEE70000DD
:105A400038B5104B1A7A0446DAB901251D7252F0A6
:105A50001FFE2A4604F5B3451121583552F074FD56
:105A6000284607F00FFC60B1284607F0CBFB062262
:105A700004F59E4100B13C31BDE8384002480DF0CC
:105A80004FB838BDB0880020702B002010B5074BF0
:105A90001A7A4AB100241C7252F0FAFD22461121F2
:105AA000BDE8104052F050BD10BD00BFB0880020CE
:105AB0002DE9FF41054605F5A258684608F118088A
:105AC00019F092F96946404613F032FA0646E8B1F9
:105AD000374877F035F950B105F53653D3ED0C7AE8
:105AE000F5EEC07AF1EE10FA94BF0126002605F516
:105AF000B340583007F0C6FB2E4C2F4F00B146B1D3
:105B0000002328462380FB73FFF7C0FF04B0BDE8E5
:105B1000F0812846FFF73CFFA0B363787BBB237876
:105B20000133DBB2082B237002D1404613F018F981
:105B30002378092B02D1404613F00AF92378092B68
:105B40001DD94FF48573238052F0A2FD022210214B
:105B500052F0FAFC88F0F4FE6368C01A47F2305342
:105B6000984209D905F55650144A0221103054F0D4
:105B7000AFFD88F0E5FE60602846FFF761FF6378BF
:105B8000FB73C3E72378002BF9D0013B6278DBB2CB
:105B90002370002AF3D0002BF1D1667052F078FD0B
:105BA0003246102152F0D0FC2846FFF76FFFE6E79F
:105BB00000850020B08800205D8900208CE20C0860
:105BC00010B500F5A044D4F80437042B01D101200E
:105BD00010BD00F5B340583008F0D4F80028F6D1D5
:105BE00094F83007F4E7000073B500F5A045019282
:105BF000A5F8E010044688F0A3FEC5F8E400D5F847
:105C0000C80003685B68984785F8DE00D5F8C800CF
:105C100003685B689847019A182818D8DFE800F0F5
:105C20000D170D0D0D0D0D0D0D175017571757575B
:105C300017414141171717415700324B93F82A3D3E
:105C400003B304F59B412C3120460CF069FFD5F8D5
:105C5000C80095F8DE6003685B68984704F5565401
:105C6000864204F1100445D0D5F8C80003689B684B
:105C70009847254A03460421204602B0BDE87040FB
:105C800054F026BD04F5005393F9C433022BD8D049
:105C9000042B0BBF04F59B4104F59A4148311C319C
:105CA000D2E7D5F89C3CD90203D504F59C41543188
:105CB000CAE704F59E419B064CBF58313C31C3E70F
:105CC00020460192FFF77CFF019A0028BFD104F51E
:105CD0000056019296F9C433002BB8D0D5F8C8000D
:105CE00003685B68984785F8DE0096F9C433019A2B
:105CF000022BCCE7054A0421204602B0BDE87040E3
:105D000054F0E6BC707B00209CE20C08BEE20C085C
:105D1000F0B5044604F5A04685B00F4615465CF084
:105D20000BFDD6F8C800A6F8E07003685B689847DA
:105D300018281ED8DFE800F00D0D0D0D0D0D0D0D0E
:105D40000D1D627F0D0D6E6E1D5252521D1D1D5296
:105D50000D003C4AD2F80417012921D104F5005363
:105D600093F8C533023B012B1AD904F5405383F84D
:105D70008C15D6F8C800344A344B052D18BF13468D
:105D8000026803939268904704F5565410340090CB
:105D9000039B2F4A0421204654F09AFC05B0F0BD25
:105DA00092F82A3D3BB104F59B412A462C3120460E
:105DB0000CF0B6FEDDE704F5005393F9C533032B71
:105DC00003D1204605F0F4F8D3E7022BEBD0042BE7
:105DD0002CD104F59C412A462831E8E7D6F89C3CB2
:105DE000DA0223D49B0604D504F59E412A46583195
:105DF000DDE704F59E412A463C31D8E72046FFF70F
:105E0000DFFE0028B5D104F5B340583007F062FA40
:105E10000028EED104F5005393F9C533032BD0D0FD
:105E2000022BC0D0042BD4D0012BA2D104F59C416D
:105E30002A465431BBE704F5005393F9C533042BCC
:105E400097D1C6E7707B0020D4E20C0850C70C083D
:105E5000DCE20C0870B500F5565504461035124AC0
:105E60000421284604F5A04654F032FC0023A6F88D
:105E7000E03004F5005393F80C33032B12D196F85D
:105E8000DE10302220460CF01BFFD6F8C800036855
:105E90009B689847054A034606212846BDE870409E
:105EA00054F016BC70BD00BFF0E20C0807E30C080C
:105EB00000F5405310B500220529044600F5565060
:105EC00083F88C2500F110000CBF054A054A042117
:105ED00004F5A04454F0FCFB0023A4F8E03010BD0E
:105EE00020E30C0831E30C08013A38B50446052AD2
:105EF0003DD8DFE802F04B1B86118F0300F5A0436D
:105F000093F8EC3A43B100F59F4104221431434821
:105F1000BDE838400CF004BE04F5A04393F8EC3A19
:105F200023B104F59E4104223C31F0E704F5A04280
:105F300004F59E43D2F8C8103C33994226D004F5AC
:105F40009F431433994221D0D2F80437042B1DD03B
:105F5000334D95F8F930CBB105F5116105F5E560E4
:105F600030F040FC20B12E4B012283F8302738BDA1
:105F700005F5116105F5E56030F034FF30B104F549
:105F80009C4104222831A5F5A040C1E704F5A042B8
:105F900004F59E43D2F8C8103C339942E7D004F58B
:105FA0009F4314339942E2D004F5B3405830D2F8FD
:105FB000045707F0E7FE0028D9D1042DD7D004F507
:105FC000005393F98F33022B0DD004F59C412046EA
:105FD000042254310CF0A4FD04F50D500F30BDE83F
:105FE000384048F0FBBF0E4890F8F930002BECD059
:105FF00000F5116100F5E56030F0F4FB0028B2D146
:10600000E3E700F5B340BDE8384001221421103029
:10601000F7F7AEBDBDE8384004F0CABF702B0020D2
:10602000707B002070B52DED068B044688F07CFC5B
:10603000414BB4F8BE101A88404E8A420546404A89
:1060400006D01980002330601370BDEC068B70BD44
:1060500033683C49C31A8B4265D9012313705CF045
:106060006BFC5CF023FB35605CF066FC5CF01EFBB7
:106070005CF044FB0428E8D95CF05EFB204600217C
:106080000AF0ACFF20460021B0EE40AA0AF0B0FFB3
:1060900020460121F0EE409A0BF06EF900212046D7
:1060A000B0EE408A0AF0AEFF04F5B3401030F0EED7
:1060B000408A76F04FFE9FED249A0028B0EE4A0AFF
:1060C0004FF0040008BFB0EE498A5DF047FFB0EE24
:1060D000690A13205DF042FFB0EE680A15205DF0FA
:1060E0003DFFB0EE680A1A205DF038FFB0EE480AB6
:1060F00046205DF033FF012108465EF03BFAB0EE2A
:10610000490A02205DF02AFFB0EE490A03205DF043
:1061100025FF20460BF052FBBDEC068B2046BDE868
:1061200070400CF091BA1278002A8ED044F62062AA
:1061300093428AD993E700BFBC880020C088002022
:10614000BE880020400D03000000000000F5A043C1
:1061500000F59C40D3F8C8202830824202D193F841
:106160003007E8B10F4B93F80C0303F54053A0F14F
:106170002702012A93F8383D0FD92C2809D00A2884
:1061800009D0A0F13102504250410A2B18BF002023
:1061900070470120F9E7012070470A3B58425841F7
:1061A000704700BF704B002008B500F5005393F80E
:1061B000502242B193F88C322BB1FFF7C7FF80F029
:1061C0000100C0B208BD0120FCE700002DE9F04746
:1061D00000F50055AE4E95F88CA2044600F5B3408C
:1061E0008AB0103076F0ACFDD6F80437042B814627
:1061F00042D1012104F5095808F11008404666F023
:10620000A5FD96F8383D0A2B074605D1B9F1000FD8
:1062100054D1002386F8383D95F85032002B58D1E0
:1062200095F956329B4D012B03D0063BDBB2012B77
:1062300011D895F80C330A2B0DD104F5A047D7F8E7
:10624000C80003681B6A984728B1D7F8CC102B22E6
:1062500020460CF065FC96F8383D0A2B04BF372326
:1062600086F8383D95F80C330A2B02D1372385F890
:106270000C330AB0BDE8F0870028BAD004F5A0437B
:10628000B6F86677D3F8C80003685B6898471428A7
:10629000AFD004F5B340583007F0C8FB0028A8D1B0
:1062A0003946A6F5A040FFF723FA01460028A1D001
:1062B00096F82C174B1E594259419BE740EA0A03B6
:1062C000DBB2002BA8D1744800F0EEF80028A0D073
:1062D000A2E7B9F1000FCCD004F5B040403084F013
:1062E00093FE0028C5D12046FFF730FF0028C0D11B
:1062F000002F00F0BC8069493A46404666F0FEF83F
:1063000095F95692B9F1010F06D040F38480A9F1B6
:106310000603DBB2012B7ED85FFA89F9B9F1010FD0
:106320004CD104F5A04204F59C43D2F8C8102833A0
:10633000994207D192F8303723B195F88F33013B5A
:10634000012B96D904F59C410A225431204606AE11
:106350000CF0E6FB304618F047FD95F9692292BB38
:10636000B9F1010F2FD004F5A049B5F96A32D9F877
:10637000FC18DFED4B5AD1ED017A002BF8EEE77AED
:1063800052DD07EE103AF8EEC76AE6EEA57A30461F
:10639000FDEEE77A17EE901A18F02CFD0023404628
:1063A000CDE9043366F06EFD04A967F0AFFA00286A
:1063B00057D0049B0893059B099317E004F59D4172
:1063C0000A220C31C2E72046FCF7D2FE07EE900A03
:1063D000E84604F5B242103221464046B8EEE70ADC
:1063E000FDF760FD98E80F0086E80F0095F956323A
:1063F000012B10D031462046FDF710F831462046DB
:10640000FDF736FC95F95632072B04D104F54054BC
:10641000012384F88A3552F03BF93A4609210AB043
:10642000BDE8F04752F090B8D5ED966A95ED995ACF
:1064300095ED977A35EE076A36EEC57AB4EEC67AF0
:10644000F1EE10FA89BF37EE067A95EDFC7A27EE69
:10645000257AF6EE006A94BFE7EE257AE7EE267A13
:1064600095E7D9F8FC389A680892DB68A4E7BAF196
:10647000000F3FF4FEAE95F88C32002B7FF4F9AE9E
:1064800004F55650074A0521103054F021F9C2E7AF
:10649000707B0020704B0020702B00204CE30C0818
:1064A0000000C84255E30C0810B5044600F5B3409F
:1064B000103076F04FFC98B104F5B340583008F036
:1064C00047F960B904F5AE4494ED027ADFED087A3D
:1064D000B4EEE77AF1EE10FAACBF0120002010BD57
:1064E00004F5AE4494ED027ADFED027AF0E700BFE6
:1064F000CDCCCC3D6666663F38B500F5A04500F5CD
:106500009F43D5F8C82030339A42044602D195F80B
:106510000007D8B904F5B340B5F86617583006F04F
:10652000F5F8A0B9D5F8C83004F59C442834A34246
:106530000CD195F800374BB1D5F80437032B05D1B2
:10654000B5F86607A0F116035842584138BD00203F
:10655000FCE700002DE9F74F00F5A04A00F59C424A
:10656000DAF8C81028329142044604D100F50059E7
:1065700099F968233AB90022CAF8F4268AF8F12674
:1065800003B0BDE8F08F88F0DBF9DAF8AC5680464E
:1065900035B1451B40F6C312954294BF0025012535
:1065A0002046FFF781FF834620B100278AF8F07666
:1065B000002642E004F5B340103076F0C1FB0190B4
:1065C0000028F2D004F5B0464036304684F01CFD79
:1065D0000746002842D09AF8F066002E39D145B31C
:1065E00004F5805041F27071D0F85026002AB8BFEF
:1065F00052428A4206DCD0F85426002AB8BF5242E2
:106600008A4229DD04F5AE4104F5B2406C31103008
:1066100018F01AFFDFED457ACAF8F486B4EEE70AFF
:10662000F1EE10FA4FF000024CBF01260026CAF826
:10663000F82601228AF8F0262F4604F59070F7F725
:10664000DFFB022832D9002F42D10022CAF8F426FB
:1066500096E75D465E46ECE73546EAE7304684F06D
:10666000BBFC064640B1002DA2D04FF4FA72019F48
:10667000CAF8F8260026E0E7DAF80427012A07D04E
:10668000032ADAD12046FFF737FF002890D1EAE746
:1066900009F58162D2ED007AF5EEC07AF1EE10FADA
:1066A00086DD9AF80027002A82D1DEE704F502553C
:1066B000183599F8E611284610F0F2FA0028C4D0EF
:1066C00099F8E611284610F0E3FB0028BBD1BCE79F
:1066D000DAF8F40610B9CAF8F48651E7DAF8F826C1
:1066E000A8EB00089045FFF44BAF9AF8F126002A7A
:1066F0007FF446AF01228AF8F12699F86833DB0768
:1067000005D504F5B3400C211030F7F731FA04F544
:106710005650103036B1064A022103B0BDE8F04FA2
:1067200053F0D6BF034A3146F7E700BF0000964258
:106730006CE30C0882E30C082DE9F04F2DED028B81
:10674000064685B0002306F50059039388F0F8F853
:10675000D9EDD97AF5EEC07AF1EE10FAC4BF9FED0B
:10676000C67A67EE877A06F5907BC8BFFCEEE77ABB
:1067700080465846CCBF17EE907A9627F7F740FB35
:10678000022840F2088196F8E4339FEDBC7AB022EB
:1067900002FB0363D3ED777A67EE877AFCEEE77A44
:1067A00017EE903A9F428CBF00270127B9F9583362
:1067B000022BB8BF022307EE903A06F5A250B8EEBE
:1067C000E78A03A9F6EE087A183028EE278A12F035
:1067D0008DFB054640B1DDED037AF4EEC87AF1EEAB
:1067E00010FAACBF012500255846F7F709FB012830
:1067F00006F5A0441AD806F5B340103076F0A0FA9A
:10680000A0B19DB904F5E16393ED007ADFED9C7AC8
:10681000B4EEE77AF1EE10FA08DDDDED037AF4EE7E
:10682000C87AF1EE10FAACBF0125002506F5B34099
:10683000583005F0C5F98246002840F0FD8006F585
:10684000B340103076F07CFA002800F0038196F80F
:10685000E43306EB0313D3F890317BB15846019330
:10686000F7F7CEFA012800F29880019BA8EB03000D
:1068700041F2873398428CBF00230123D4F8A82625
:1068800002B11BB9002D40F08A803D46D4F8C820E3
:1068900006F59C4328339A421AD199F99033002B7C
:1068A00040F08580002384F8F236D4F80437042BB6
:1068B00000F0AE80072B00F0C180032B08D13046DA
:1068C000FFF71AFE20B1002584F8F156C4F8AC5643
:1068D00094F8F23603B18DB907EE905A9FED697ABC
:1068E000F8EE677A04F5E16367EE877AD3ED006A24
:1068F0009FED657AE6EE877AC3ED007A3046FFF7C2
:10690000D3FD054698B194F80C27C4F8A8860AB9B7
:10691000C4F81087D4F8C81006F59C432833994270
:1069200005D1D4F8AC3603B10AB9C4F8AC8694F8F2
:10693000343884F80C5765F3C30384F834386FF0A7
:106940008FF929466FF068F9504B30465D71FFF7BB
:1069500001FE3046FAF7C2FD35B199F80E331BB986
:1069600087F0EEFFC9F8100389F80E533046FFF7A1
:106970009BFD002840F08E8006F5B340103076F085
:10698000E9F980F00100C0B284F8140705B0BDEC4D
:10699000028BBDE8F08F002708E753466EE728F02A
:1069A00091FF27F085FF00287FF46FAF6EE75B4211
:1069B00007EE903A06F6E853F8EEE77A93ED007AA0
:1069C000F4EEC77AF1EE10FA13DD012384F8F23603
:1069D000C4F8FC8604F5E163DFED2D7A93ED007ACF
:1069E000B4EEE77AF1EE10FA7FF75FAFC3ED007A0D
:1069F0005BE794F8F236002B3FF457AFD4F8FC363F
:106A000040F6B832A8EB030393423FF64BAF4CE796
:106A100006F5B040403084F0DFFA00283FF458AF6C
:106A200004F5D36393ED007ADFED197AB4EEE77ADB
:106A3000F1EE10FA7FF74CAF012549E704F5D36377
:106A400093ED007AFEEE007AB4EEE77AF1EE10FAFA
:106A5000F2D43DE7D4F80437002D18BF3D46012B92
:106A600001D1002534E706F5B040403084F0AAFAA1
:106A70000028F6D12CE700BF0000B4420000C84255
:106A80009A99993E9A99193E9A99593F5D890020A1
:106A9000CDCC4C3E002077E70020704700207047A7
:106AA00001207047034BD3F80407431E5842584156
:106AB000704700BF707B002030B587B002A818F087
:106AC00093F9374884F07EFA20B136493648FCF70E
:106AD00085FB1FE0324884F07FFAE8B1334C04F1C3
:106AE0002405234604F11002A4F11001A4F1D00002
:106AF000009584F097FACDE90045A4F51C7292ED5B
:106B0000000A2B4904F11003A4F11002A4F1D000F3
:106B100084F04AFA07B030BD214802A984F09AFAFD
:106B200008B102A9D2E7234CD4F8783D002B0CDD44
:106B300094F8183D4BB1A4F500501C49FCF74EFBEE
:106B4000A4F50050FCF702FCE4E7174804F0FEF857
:106B50000028BAD1184CD4F83439002BB5D004F53C
:106B6000126204F5106104F5116018F0D9FB0028D9
:106B7000ABD104F2A465D5ED007AB7EE000A04F5B6
:106B80001261A4F5A04030EE670AFCF78BFC04F517
:106B9000106204F51261A4F5A040FCF737FBB9E7D9
:106BA000B083002090840020702B0020808400207F
:106BB00068590020704B0020707B002008B50A48FF
:106BC00090F80134013B012B03D8A0F50050F8F7F1
:106BD00095FB0648F8F760FA0448F8F74FFBBDE864
:106BE00008400248F8F7A8BE704B0020702B002028
:106BF00010B5044607480CF087FE50B1064B93F8D9
:106C0000190B30B1236820469B6B984780F0010038
:106C1000C0B210BD80870020707B0020124B9842CC
:106C200010B5044601D1002010BD03F11C029042B2
:106C3000F9D003F138029042F5D003F1740290428A
:106C4000F1D0D4339842EED003681B6A984720B144
:106C5000064B93F88A35002BE5D1206907F0ACF894
:106C600080F00100C0B2DFE7A8780020705B002050
:106C7000174B984210B504460ED003F11C02904207
:106C80000AD003F13802904206D003F17402904218
:106C900002D0D433984206D10E4B93F9B903B0FA1F
:106CA00080F0400910BD03681B6A984718B10A4B71
:106CB00093F88A3543B9206907F07EF830B120692E
:106CC000BDE8104009F034BC0020EBE70120E9E703
:106CD000A8780020704B0020705B002073B50F4E29
:106CE0000D46114696F9A42A1AB90124204602B08D
:106CF00070BD036801915B69984704460028F4D190
:106D0000D6F89C3C019913F4802FEED00448054B33
:106D100000682A46C06A25F0B1FCE7E7707B0020D6
:106D20006C2B002094E30C08084A0260084A426079
:106D3000111F816002F10801C160A2F1380102F562
:106D40009C724261034A016182617047E0E30C0872
:106D500080850020C83F002008B503681B6E984757
:106D60000648D0F8C820A0F5FA739A4205D0BDE8CD
:106D70000840A0F5A040FEF7B5BD08BD707B00201F
:106D80002DE9F341594C04F5D06300221A60A4F5B3
:106D9000EC73C11A4B42A4F500584B4188F82038D7
:106DA00004F5D263002684F86466A4F8BA6684F811
:106DB000BE6684F87C6684F8F16684F8F266C4F8EE
:106DC000E466C4F8E066C4F8DC66C4F8EC661A60F1
:106DD0008369D3F8FC31A4F8B43604F51163054691
:106DE0000FCB04F5106787E80F0084F8BD6684F8C0
:106DF000CC66C4F8DC6887F0A3FDC4F8D0002B682B
:106E000028465B6998474FF0FF3384F8C166C4F8A1
:106E1000003188F88C6584F8C006286906F06AF9A4
:106E200084F8BF662B682846DB6D98470646002825
:106E300058D02B6828469B6B984784F80007D8F8F1
:106E4000AC070368DB6B984708F5A56078F024F978
:106E5000A4F5A0400AF016F8A8F55B6065F0DCFF29
:106E600094F83037CBB1A4F5A040FFF71DFBA0B9D3
:106E700004F5196075F06EFF78B9D4F8C80003689E
:106E80005B6B984748B95AF0ABFA194A062153F0A0
:106E90001FFC04F5E5602FF051FD1648F7F780FA66
:106EA0002B6993F9CC206AB1586801A912F01EF839
:106EB0002F699DED010A014607F18800FBF708FFE5
:106EC00087F841012B6828465B69984750B12B69C8
:106ED00093F93C22002A02DD93F8A03213B9002373
:106EE00084F8D530304602B0BDE8F081707B0020D8
:106EF000A0E30C08702B002070B503685B6E0E4693
:106F000015469847044650B995F900303BB90548F5
:106F1000054B00683246C06A294625F0AFFB204683
:106F200070BD00BF6C2B0020C4E30C0810B50E4CE4
:106F3000204677F0ADFE04F5AC7077F025FC04F543
:106F40002C7078F053FB094B03F5A042002182F826
:106F50007C1603F5AD42002103F540531160012278
:106F600083F8502010BD00BF745C0020702B0020FF
:106F700008B52DED028B1520B0EE408A5CF0EEFFD7
:106F8000B0EE480ABDEC028B1A20BDE808405CF068
:106F9000E5BF000008B5084890F9B9330121A0F514
:106FA000005033B10AF0E8F9BDE8084046205CF033
:106FB000D5BF0AF009FAF7E7704B002001207047AF
:106FC0000120704701207047012070470120704761
:106FD000192070470048704748E40C080048704783
:106FE00058E40C0884B010B503AC84E80E000369C3
:106FF000B3F9C010642359432046012217F0FAFE6A
:1070000004482146FCF734FEBDE81040012004B0DE
:10701000704700BF702B002013B50F4901AAA1F1E2
:10702000100017F09DFF40B1DFED0C7A9DED017A65
:10703000B4EEE77AF1EE10FA0CD8094CD4F8AC07AC
:1070400003689B6B984728B106492E22A4F540504F
:107050000BF066FD02B010BD90840020000000B46B
:10706000705B0020AC7A002070B51E4C0546D4F849
:10707000CC00036886B05B69984738B11A491B4851
:107080002F220BF04DFD012006B070BD04F6D81084
:1070900006F092FE0028F1D1A4F50056D6F8AC0710
:1070A00003689B6B984728B1D6F8AC0703681B6C44
:1070B000984798B10E4B0FCB02AC84E80F002846DE
:1070C00001F05AF82868059B009394E80E00446C80
:1070D0002846A0472846FFF79FFFD4E704F5126330
:1070E000E9E700BF707B0020AC7A0020702B002005
:1070F0008084002010B50446FFF78EFF2046BDE8CF
:10710000104001F075B80000042070470048704737
:107110004DEA0C08004870474DEA0C08037F73B134
:10712000D0ED087AFDEEE77A17EE903A084AC2F8F9
:107130001837437F3BB1436AC2F81C3770478369F5
:10714000D3F8F831F2E78369D3F8FC31F4E700BFF4
:10715000707B002008B50023838300F1280180693B
:1071600011F0DAFE012008BDF8B56D4E2DED048B4F
:1071700004460121304606F5A04797ED469ADFED1B
:10718000699A09F02BFF0121B0EE408A304609F0E0
:107190002FFFC8EE297A06F50055A069B5F9DC3352
:1071A00004F1280108EE903AF8EEE88AB5F9DE33EA
:1071B00068EEA78AC0EE297A08EE103AB8EEC88ABF
:1071C00028EE278A11F0A8FE95F9E2335BB39FED14
:1071D000567AF0EEE87AF4EEC77AF1EE10FA22D59C
:1071E000227FA369002A54D1012222770022226241
:1071F00094ED087ADFED4D7AD3F8F8314C4867EE1C
:10720000C77A9FED4C7A67EE877A0122FDEEE77A26
:10721000B0EE490A17EE901A0B44C7F8183700234E
:1072200077F0C6FC08E0002341482377F0EE490AD6
:10723000B0EE680A77F0B8FC04205CF08FFE95F998
:10724000E23343B19FED387AF0EEC87AF4EEC77AB4
:10725000F1EE10FA28D4002337486377F0EE490A9C
:10726000B0EE480A77F0FAF813205CF077FEB5F933
:10727000E033002B03DD314E96F9CA335BBB28485F
:107280002021F7F7B9FB002842D1254809F0CAFCB4
:1072900041E0D3EDC56A96ED467AD4ED087AE6EE84
:1072A000877AC4ED087AA3E7637F2BB9012363775C
:1072B000A369D3F8FC316362616AC7F81C17A3693C
:1072C000D3F8FC010023091A1A461B48B0EE490AFC
:1072D00077F0AAF9C8E70121A6F5405009F092FE1F
:1072E00080EE297AB5F9E033002106F56D7007EEDE
:1072F000903AF8EEE77AF0EE490A27EE870A78F03E
:1073000075F8BDEC048B2046BDE8F840FFF730BEB1
:107310000348F8F781F907EE900AB8EEE70AF0E7BC
:10732000702B002000A08C4500000034E02E654248
:10733000745C00200000C842CC5D0020705B00201F
:107340002DE9F04F2DED0C8BDFF8A0A39FEDDCDADB
:107350009FEDDC9A97B000F128050AF5A04B044692
:10736000012150469BED46BA09F038FE01215046F6
:10737000F0EE408A09F03CFE01215046B0EE408A12
:1073800009F040FEDFEDD07A88EEA77A0AF50056C4
:1073900001A8B6F9DC330AEE903AF8EEEAAAB6F99B
:1073A000DE33DFEDCA8A6AEE87AA88EE277A0AEE14
:1073B000103AB8EECAAAB6F9E0339FEDC58A2AEEB4
:1073C00007AA80EE277A09EE903AF8EEE99A6AEE7B
:1073D0008D7A69EE879AF0EEEACAF4EEC8CACDED6E
:1073E000017AB0EECACA6AEE0D7AF1EE10FAF0EE4A
:1073F000E9BAB4EEC8CACDED027A58BF4FF0010920
:1074000069EE8D7A48BF4FF00009F1EE10FAF4EE04
:10741000C8BA9AED460ACDED037A54BF4FF0010881
:107420004FF00008F1EE10FA54BF012700272CF0AE
:107430002DF901A928462BF0D3FB28462BF0CAFCD6
:1074400028462BF039FC20EE090A284620EE280AAF
:10745000BDEEC00A10EE103ACBF818372BF046FC00
:1074600020EE090A20EE280ADFED9A8ABDEEC00A56
:10747000CDED0D8A10EE103ACBF81C370DF1280B2C
:107480004FF07E535946A0690A93CDED0C8ACDED9D
:107490000B8A11F041FD0021504609F06DFFB0EE5E
:1074A000C00AB4EEC80AF1EE10FA16D55046FEF73F
:1074B000FBFF90B9F4EEC8CAF1EE10FA0DD5B4EEA8
:1074C000C8CAF1EE10FA08D5F4EEC8BAF1EE10FA17
:1074D00044BF9BE80F0085E80F000AA82BF0DEFCF4
:1074E000294612A88DED141A8DED120ACDED130A5E
:1074F000CDED151A2BF0E4FC0DF1100A51460EA843
:107500008DED101ACDED048ACDED058ACDED068AFC
:107510008DED0E0ACDED0F0ACDED111A2BF09AFA72
:10752000B6F9DC33DFED6C7A01EE103AB6F9DE33F2
:1075300009EE103AB6F9E03308EE903AB8EEC11A07
:10754000B8EEC99AF8EEE88A21EE271A29EE279AB2
:1075500068EEA78AF4EEC8CAF1EE10FA21EE0D1A11
:1075600029EE0D9A68EE8D8A07D594F83830DFED54
:10757000597A002B18BFB0EE671AB4EEC8CAF1EE04
:1075800010FA07D594F83930DFED527A002B18BF86
:10759000B0EE679AF4EEC8BAF1EE10FA07D594F897
:1075A0003A30DFED4C7A002B18BFF0EE678A9AE88C
:1075B000070007AE86E80700F1EE410AC2209DED04
:1075C000070A28F001FFC3208DED070AB0EE491A23
:1075D000F1EE490A9DED080A28F0F6FEB0EE681AB1
:1075E000F1EE680A8DED080AC4209DED090A28F025
:1075F000EBFE514630468DED090A2BF0DDFF12A956
:1076000028468DED120ACDED130A8DED141A2BF0DC
:10761000E7FA28462BF0DEFB304BDDED076A93EDF1
:10762000427A9FED280AC6EE877A3046DDED086A79
:10763000CDED077AD3ED987A86EEA77ADDED096A6B
:107640008DED087A86EEA77A8DED097A2CF01EF87A
:10765000B9F1000F01D0CDED07AAB8F1000F01D0AC
:107660008DED08AA0FB1CDED099AF0EE4B0A9DED14
:10767000070A1B4877F098FA04205CF06FFCF0EEE4
:107680004B0A9DED080A174876F0E8FE13205CF0DF
:1076900065FC0021F0EE4B0A9DED090A124877F0D7
:1076A000A5FE2046FFF764FC84F8389084F8398002
:1076B00084F83A7017B0BDEC0C8BBDE8F08F00BFBA
:1076C00035FA8E3CE02E654200A08C450000C84291
:1076D0000000003400000000CDCC4C3E705B002068
:1076E000745C0020CC5D0020245F0020702B002003
:1076F00010B50446FFF74EFC0B4B93F9E223022A28
:107700000DD1B3F9E023002A09DD03F5805393F985
:10771000CA3323B12046BDE81040FFF711BE204612
:10772000BDE81040FFF720BD704B00200A207047D5
:10773000004870475A0A0D08004870475A0A0D0859
:1077400001207047012070470120704701207047D9
:10775000034BD3F80407031F58425841704700BF3A
:10776000707B002070B52D4CD4F8CC20A4F5BA73F2
:107770009A42064615D1036993F844318BB104F55A
:10778000E5602EF0A5FC054658B959F029FE244ABB
:10779000032152F09DFF3369012283F843212846DB
:1077A00070BD94F8EC3A23B194F9A43A9A1E53426E
:1077B000534184F8C03604F511630FCB194D04F51D
:1077C000126484E80F0085E80F00A5F5EC702FF037
:1077D000F5FA154B1C68E66A336830465B689847D3
:1077E000B0B196F84D309BB1E36A9B8F83B159F0ED
:1077F000F7FDE36A0D4A9B8F062152F069FFE36AA9
:10780000A5F5EC70998F2FF0C5F8E36A00229A87EE
:10781000074884F059FB0125C1E700BF707B0020B9
:1078200040E50C08708400206C2B00205AE50C0801
:107830000057002038B50D4C94F82C37012B11D18E
:1078400004F5E5602CF0BCFBB4F8665704F6D810DC
:10785000294605F0B3FC28B9152D03D104F50460C1
:1078600083F090FC0023C4F8AC3638BD707B002058
:1078700008B511F06BFD90F87C32DB0704D5BDE84C
:10788000084002482FF036B908BD00BF988200209A
:1078900038B5354C94F82C37012B0ED0A4F5D671A1
:1078A0000822A4F5A0400BF03BF959F099FDBDE882
:1078B00038402E4A062152F00BBF04F6D810B4F817
:1078C000665705F09FFC28B104F6D810BDE8384093
:1078D00008F0D8BD162D05D0152D36D1D4F80437B3
:1078E000072B0AD122480CF031FF21480DF07CF81B
:1078F000BDE838401E480CF08DBFA4F5A040F8F755
:10790000A9F9A4F5A040F8F787F8A4F54053D4F8F6
:10791000181793F9202464235A4304F5046083F074
:107920008DFBC4F8180704F5046083F0C9FC30B17E
:10793000BDE838409FED0F0A46205CF00FBBA4F570
:10794000A040BDE83840F7F74FBE1E2D18BF4FF0DE
:10795000FF33074818BFC4F87836F8F77BF90448B6
:10796000F8F75AF80248ECE7707B002074E50C0841
:10797000702B00200000000070B5134890F9A43A65
:107980000E46154613B90124204670BDD0F89C3C24
:107990005B0310D5B0F8661700F6D81004F0B6FEF9
:1079A000044640B9094B0A48006832462946C06A75
:1079B00024F064FEE8E707482EF08AFB044600281E
:1079C000E1D1054BEFE700BF707B0020A0E50C087C
:1079D0006C2B002098820020B4E50C0810B5144BE5
:1079E000B3F86637532B04461ED10AF0BDF89FED5D
:1079F000110A46205CF0B2FA9FED0E0A49205CF0B5
:107A0000ADFA9FED0C0A4A205CF0A8FA46205CF023
:107A100085FB49205CF082FB4A205CF07FFB20461E
:107A2000BDE81040FFF782BABDE81040FFF7C6B8C6
:107A3000707B00200000000008207047004870475D
:107A400040E60C08004870474CE60C0801207047DF
:107A500008B50248FDF7E6FE012008BD702B0020A6
:107A6000014800F061B900BF1C79002010B5044640
:107A7000FFF7A4F82046BDE81040FFF78BBA0000DE
:107A80000120704700487047C4E60C080048704762
:107A9000CCE60C08012070470120704710B5054B5B
:107AA00003F5126403F511630FCB84E80F00012086
:107AB00010BD00BF707B002008B50B4800F5A04248
:107AC00000F500530321D3F8E83D93FBF1F3C2F82E
:107AD0001837F8F705F80448F7F79EFFBDE80840A7
:107AE0000148F7F781BD00BF702B002007207047C9
:107AF000004870470DC90C080048704744E70C085F
:107B00000120704701207047012070477047000036
:107B100008B5002303774362034884F0D5F903488E
:107B2000FBF752FB012008BD00570020702B0020FE
:107B300010B5194CD4F8D03DB3F9083023B9D4F8B6
:107B4000DC3DB3F90830F3B1002303774362D4F886
:107B5000D00D5AF0E1FF04F6E853D3ED007A0F4858
:107B6000F8EEE77A27EE800ABDEEC00A10EE103A72
:107B7000C0F81837A0F5A040F7F7B2FFBDE81040F5
:107B8000074802F0D9BF037F002BE0D0A4F50050D6
:107B9000F8F760F8F2E700BF704B0020707B002020
:107BA000702B002070B54F4DDFED4F7A95F8E43320
:107BB0009FED4E7A2DED048BB02606FB035393ED1B
:107BC000788A9FED4B9A28EE278A05F5B353BDEED0
:107BD000C88A93ED010AF8EEC87A044667EE897AFE
:107BE00097EE870A28F0DCFB237FF0EE408A002B1B
:107BF00063D105F50053D3F8D03DB3F90830002B1D
:107C00005BD1284609F00EF8002856D195F8E433E8
:107C100095F8281406FB035393F8C12100294CD191
:107C2000012A4AD993ED777AF0EE087AB4EEE77A32
:107C3000F1EE10FA41DBDFED2F7AB0EEE80AB4EE98
:107C4000E70AF1EE10FA38D5636A9BB386F078FE46
:107C5000636AC01AB0F5FA7F33D8237F002B3DD07A
:107C6000254DA5F1200696E80F0085E80F0094ED5C
:107C7000088AA5F110013046B8EEC88A17F0E4FB77
:107C800028EE098ADFED1D0A284670EE200AB0EEC4
:107C9000480A17F07FFCA6F52453BDEC048BD3F8FB
:107CA000AC079FED170A03682A4631469B6ABDE878
:107CB0007040184786F044FE6062636A002BCCD0A7
:107CC000C4E7104D84ED088A012323770023636203
:107CD00005F110030FCB85E80F00BEE7BDEC048B68
:107CE00070BD00BF702B00200000C84235FA8E3CEA
:107CF0000AD7233CDB0FC93F9084002000007A4460
:107D00000000000070840020036A0B60007F704751
:107D10000520704700487047BCE70C0800487047D2
:107D2000CCE70C080120704738B52DED028B4B4C89
:107D30009FED4B8AD4F8D00D5AF0EEFED4F8E83D12
:107D400007EE903AF8EEE77A04F5405527EE800A00
:107D5000A4F50050BDEEC00A10EE103AC5F8183771
:107D6000F7F7BEFED4F8D40D5AF0D6FEB5EEC00A31
:107D7000F1EE10FADABF04F6EC53D3ED007AD4ED4D
:107D8000DC7A3848CBBF20EE270A20EE270A20EE07
:107D9000080A28EE400ABDEEC00A10EE103AC5F8F7
:107DA0001C37F7F769FE94EDDC7AD5F81C0704F66A
:107DB000EC5327EE087AD3ED007A27EE888AFDEEA1
:107DC000C77A17EE902AFDEEC87A17EE901A28F0BF
:107DD0009BFBC5F81C072348FDF7B0FD20B1D5F883
:107DE0001C375B42C5F81C3795F8DC3063B194F959
:107DF000C433022B08D1002301214620C5F81837CF
:107E0000C5F81C375CF00EFC5AF096FD5F215BF064
:107E100057FDF8B15BF024FD02281BD195F8BD3663
:107E2000C3B905F5D26304F5826493ED007AD4ED0D
:107E3000007AB4EEE77AF1EE10FA0BD5012385F85B
:107E4000BD36BDEC028B084A0848BDE83840042125
:107E500052F03EBCBDEC028B38BD00BF704B002021
:107E60000000C842702B0020D4E70C0800610020FD
:107E700010B50446FEF7A2FE2046BDE81040FFF70D
:107E800089B80000062070470048704754E80C0885
:107E90000048704764E80C080120704701207047D3
:107EA00001207047012070477047000008B5044862
:107EB00084F00AF80348FBF787F9012008BD00BFEA
:107EC00000570020702B002038B50F4C04F50055EA
:107ED000D5F8D00D5AF020FE05F6E852D2ED007A22
:107EE000F8EEE77A04F5A04327EE800A2046BDEEBF
:107EF000C00A10EE102AC3F81827F7F7F1FD204644
:107F0000BDE8384002F018BE702B00200F207047EB
:107F100000487047DCE80C0800487047E4E80C08AB
:107F200001207047012070470120704701207047F1
:107F3000012070470120704730B5184B2DED028BA2
:107F4000002283F88A2503F52453103305460FCB0E
:107F500085B06C4684E80F00114804F099FB90B19D
:107F6000A86900F57F702BF0C1F90D48B0EE408A8A
:107F700004F0F2FBF0EE400A9FED0A0A204628EEDC
:107F8000000A17F007FB00230748EB612146FBF7C7
:107F90006FFE012005B0BDEC028B30BD705B002090
:107FA00048850020E02E6542702B002038B5424CF9
:107FB00094F8C13643B194F8EC3A2BB104F6D810DA
:107FC000BDE8384008F030BAD4F8DC36002B18DCB5
:107FD0003A48F7F73FFED4F8E036002B29DC374863
:107FE000F7F71AFD364890F88A35002B46D0012164
:107FF000A0F5405009F0C0F9BDE8384046205BF0DC
:10800000ADBF86F09DFCD4F8DC36C01A40F6B7331D
:108010009842DDD82B4DD4F8D006D5F8E82D514242
:1080200028F072FAC4F81807A5F50050F7F758FDC4
:10803000D1E786F085FCD4F8E036C01A40F6B733B5
:108040009842CCD81F4BDFED206A93EDDC7AD4F850
:10805000D40603F6EC53D3ED007A27EE267A67EECA
:10806000A67ABDEEC77AFDEEE77A17EE102A17EE74
:10807000901A28F049FAC4F81C07B3E7A0F580501D
:1080800090F94F33012B04DCBDE838400B48F7F77B
:10809000ABBAD4F8EC36002BF6D086F051FCD4F80D
:1080A000EC36C01A40F6B7339842EDD804F5DD64DB
:1080B00094ED000AA0E700BF707B0020702B002029
:1080C000705B0020704B00200000C842D0ED077AA2
:1080D0000348FCEEE77A17EE903A99B202F002BF3D
:1080E000702B002084B010B503AC84E80E000B4860
:1080F00021466F22FBF70AFD9DF80C1011F00401D8
:1081000002D1204616F008FF04482146FBF7B0FDD7
:10811000BDE81040012004B0704700BF702B002064
:10812000B0EEC00AFDEEC07A38B54FF6FF720546D4
:108130000C4617EE900A002128F0E6F907EE900AA7
:10814000002CF8EEE77A054BC5ED077A14BF4FF027
:10815000FF32012283F8D82838BD00BF707B002091
:10816000FEF7AABC0C20704700487047BDEB0C0816
:1081700000487047CE500E0808B50C48FCF7C0FA0E
:108180000A480B49FBF74AF90848F6F7B1FE40B137
:1081900006484FF48051F6F72FFC10B10348FBF767
:1081A00013F8024802F0B2F9012008BD702B00203C
:1081B0009084002008B50D48F7F74CFD0B48F6F702
:1081C00097FE50B109484FF48051F6F715FC20B1E5
:1081D000BDE80840054802F0AFBC0448F7F71CFCB6
:1081E000BDE808400148F7F7FFB900BF702B002039
:1081F00008B50A484FF48051F6F7FEFB38B108483D
:108200000022D0F8301900F5126016F0F3FDBDE839
:1082100008400248002102F065BE00BF702B00201C
:10822000707B0020881A10B528F096F8104BD3F810
:10823000D4280028B8BF4042002AB8BF524248F6AE
:10824000A041B2FBF1F24FF47A7102FB01118842B6
:108250000CDC93F82029D20606D503F5126403F549
:1082600011630FCB84E80F00012000E0002010BD57
:10827000707B002013B504468069019100F57F7082
:108280002BF034F8DFED0A7A20EE270A28F006F802
:10829000DFED087A019920EE270A2046FDEEC07A2C
:1082A00017EE902A02B0BDE81040FFF7BBBF00BF39
:1082B000E02E65420000C84284B070B52DED048BFD
:1082C00086B00FAD85E80E004E4CDFED4F8A0646B6
:1082D000D4F8AC0704F5005404F6EC0393ED000A5F
:1082E0000368B0EEC00A5B6A9847B4EEE80AF1EEA4
:1082F00010FAB0EE408A07DA012006B0BDEC048B1C
:10830000BDE8704004B070474049284616F0A8FF09
:1083100002A8CDED030A8DED020A2BF0B7F804A8F0
:108320008DED040AB0EE480ACDED050A2AF06AFF89
:1083300013A928468DED000ACDED010A16F090FF35
:1083400002A88DED020ACDED030A2BF019F8B4EE68
:10835000E80AF1EE10FACFDBB4EEC08AF1EE10FAC3
:108360009FED2B9ADFED2B8ADFED2B9A2BD802A8FD
:1083700069462AF037FF04A88DED040ACDED050A01
:108380002AF0B4FF684620EE098A2AF0AFFF94F97C
:10839000D83807EE903AF8EEE77A28EE288AA7EE6A
:1083A000A90A27F0FDFF20EE090ABDEEC88A20EEDB
:1083B000280A18EE101AFDEEC07A304617EE902A01
:1083C000FFF730FF99E738EE400A38EE088A80EE72
:1083D000080AA9F0EFFA02A8B0EE408A2AF086FF58
:1083E00094F9D838F0EE007AB0EE697AA8EE677AA0
:1083F00007EE903AF8EEE77AA7EE270A27F0D0FFCB
:10840000C0E700BF705B00200000003480840020C3
:10841000E02E65420000C842DB0FC93F10B504469C
:108420000848F6F765FD20B92046BDE81040FEF784
:1084300043BB04484FF48051F6F7DEFA0028F3D02E
:1084400010BD00BF702B002000207047004870470F
:10845000CCE90C0800487047D4E90C0800207047AC
:10846000036993F8140118B1D3F8C402C0F3801063
:108470007047000038B5154C05460021204608F02D
:10848000ADFD04205BF06AFD0021204608F0B0FD40
:1084900013205BF063FD0021204608F0B3FD284661
:1084A000FEF766FD2046012108F066FF46205BF0DE
:1084B00055FDAB6904F5A044D3F8F831C4F818377A
:1084C000AB69D3F8FC31C4F81C3738BD702B0020E1
:1084D000FEF72CBD17207047004870474CEA0C0887
:1084E0000048704754EA0C0801207047012070478B
:1084F0000120704710B50369002283F84021036909
:108500000446D3F83C0103689B689847A368186841
:108510007DF09EF8206904F02FFE0349A06910F059
:10852000FBFC012010BD00BF087900201FB50B4CDB
:108530009FED0B0AD4F80C0A6C302BF053F8FDEECB
:10854000E00ABDEEC00A10EE903AC4F81C3710EEF7
:10855000103AC4F8183704B010BD00BF707B00207B
:108560009F0CB34530B52DED028B83B0044686F0E9
:10857000E7F90146206900F50E700BF00FF938B1EC
:10858000204603B0BDEC028BBDE83040FEF716BBC1
:10859000206990F84031BBB1012104F073FDA3685C
:1085A000DFED400A1868036801215B6EB0EE600AD7
:1085B0009847206903F0C8F93B4803B0BDEC028B33
:1085C000BDE83040FFF794B8384DDFED398A02211D
:1085D00004F058FDD5F8D40D5AF09EFA2369D3ED76
:1085E000390A93F93C2220EE200A002A60EE280A7C
:1085F0003FDD93F8A032002B3BD0D5F8DC0DCDED5C
:10860000000A5AF089FA2369D5F8D00D93ED3A8A19
:1086100020EE080A20EE288A5AF07EFA236993EDAC
:10862000381A20EE410A20EE281ADDED000A2069F2
:10863000CDED010A8DED001A03F0C2F9A36895F99A
:10864000E22318689DED001ADDED010A0368F0EEE3
:10865000408A2AB31B6CB0EE480A9847A368186892
:108660000368F2EE040A5B6E0021B0EE680A9847D8
:10867000A2E7D5F8D00DCDED000A5AF04DFA2369E6
:10868000D5F8DC0D93ED388A20EE080A20EE288A12
:108690005AF042FA236993ED3A1A20EE010AC2E732
:1086A000DB6BD8E700000000E0780020704B002072
:1086B0000000C8421220704700487047CCEA0C08FE
:1086C00000487047D4EA0C08012070470120704729
:1086D0000120704738B52DED028B43689FED1C8A51
:1086E0001D680446006904F06DF9236993ED131ABF
:1086F000D3ED110A434200EE103A21EE081A60EE63
:10870000880AB8EEC00A28467EF05CF963682069E2
:108710001D6804F057F9236993ED131AD3ED110A7C
:10872000434200EE103A21EE081A60EE880AB8EED5
:10873000C00A28467EF0C0F99FED060A206903F0C2
:108740002FF9206905F0BCFEBDEC028B012038BD7D
:108750000000C84200000000014800F051BE00BF08
:10876000547A002013B5044600698830FAF70CFCEF
:1087700086F0E6F80146206900F50E700BF00EF861
:1087800028B1204602B0BDE81040FEF717BA2069B4
:1087900090F840313BB3012104F074FCA368DFED95
:1087A000170A18680368B0EE600A5B6E01219847EB
:1087B000206903F0C9F863689FED100A18687FF01C
:1087C0002BFB0F48F6F768FC0D48F6F757FD2046DF
:1087D0009FED0A0AFEF7CCFB2069883002B0BDE8A5
:1087E0001040FAF78FBC074804F0A8FD20690190FB
:1087F00004F04EF9019806F069FAE2E70000000083
:10880000702B0020488500201420704700487047D6
:1088100052E40C0800487047E1500E0801207047F0
:108820000020704770B504460E4800F03BF82369FD
:10883000002583F84051206904F05CFF6069052140
:1088400003F020FD084826690221FAF789FF86ED2A
:10885000B70A2369C3F848512369C3F84C51012072
:1088600070BD00BF8C7A0020702B0020014800F002
:10887000C7BD00BF547A0020014800F069B800BFAE
:108880008C7A00201320704700487047BCEB0C081E
:1088900000487047C4EB0C08012070470120704766
:1088A0000120704738B52DED028BDFED240AC36837
:1088B0009FED238A0446B0EE600A18687AF04AFAFF
:1088C000E36818687AF024FB636820691D6804F087
:1088D00079F8236993ED131AD3ED110A434200EEA0
:1088E000103A21EE081A60EE880AB8EEC00A28464F
:1088F0007EF068F8636820691D6804F063F82369F6
:1089000093ED131AD3ED110A434200EE103A21EE13
:10891000081A60EE880AB8EEC00A28467EF0CCF845
:10892000206905F0CDFD256986F00AF8C5F86C01CF
:10893000BDEC028B00230120E36138BD0000000084
:108940000000C842014800F05BBD00BF547A00201F
:1089500030B52DED048B0446006985B08830FAF7F8
:1089600013FB38B1B54805B0BDEC048BBDE8304011
:10897000FFF7F8BE85F0E4FF05462069294600F5BB
:108980000E700AF00BFF38B1204605B0BDEC048B29
:10899000BDE83040FEF712B9206990F8403163B36A
:1089A000012104F06FFBA368DFEDA50A18680368D6
:1089B0000121B0EE600A5B6E9847206902F0C4FFA7
:1089C00063689FED9F0A18687FF026FADFED9C0A26
:1089D000E368B0EE600A18687AF0BCF9E3681868DA
:1089E0007AF096FA9748F6F757FB964805B0BDEC33
:1089F000048BBDE83040F6F741BCC36A93F8CB3036
:108A000013B99148FFF74EFF206903F003F918B13D
:108A1000E36818687AF09AF92369D3F86C31EB1A95
:108A2000B3F5FA7F0BD9E368DFED850A1868B0EE7D
:108A3000600A7AF08FF9E36818687AF069FA2369B6
:108A40009FED828AC3F86C510221206904F01AFB61
:108A5000636820691D6803F0B5FF236993ED131A5D
:108A6000D3ED110A434200EE103A21EE081A60EEEF
:108A7000880A2846B8EEC00A7DF0A4FFD4E9033581
:108A800018687AF0D1F9A368186803689B6EF0EE55
:108A9000408A984703AAF0EE400A02A9B0EE680A9D
:108AA000284602F0D1FFE368DDED030A18689DED6A
:108AB000020A7AF04FF9636818687DF075FF18B9FB
:108AC000636818687EF066FEE368614D18680121EE
:108AD0007AF08AFBE3681B689B68D3EDCF7AFDEEE2
:108AE000E77A05F6D81017EE903AC5F81837E3681C
:108AF0001B689B68D3EDD07AFDEEE77A17EE903ACB
:108B0000C5F81C3704F01AFC2369D3F83C0103684C
:108B100005F21C725B6B05F5E361984748B1636829
:108B20001B68D3F88823C3F89423D3F88C23C3F8A5
:108B300098232069DFED479A04F018FBD5F8183721
:108B4000206907EE903AD5F81C37F8EEE78A07EE71
:108B5000903A0121B8EEE79A06F052F8A368186837
:108B600020EE290A036868EEA98A29EE299ADB6AB1
:108B700020EE081A69EE080A28EE880A9847D5F808
:108B8000C820354B9A4248D1636993F86430062B6C
:108B90000AD8206903F08CFC30B16069072103F02A
:108BA00071FB206904F0A6FD26480221FAF7D8FDE2
:108BB000206903F05BF8636993F86430072BB0EE2B
:108BC000408A08D12369D3F8C4329B0403D4A06936
:108BD000012110F067FE6368B5EEC08AF1EE10FA6D
:108BE0001868CCBF01210021B1EE480A7DF070FF6A
:108BF000206907F0A7FD206903F002FF1148F6F78E
:108C00004BFA1048F6F73AFB9FED0D0A2046FEF7A7
:108C1000AFF905B0BDEC048B30BDB03B9A42206982
:108C200007D190F8423123B19FED050A02F0B8FE5A
:108C3000E1E7019003F02CFF0198F7E7707A00203C
:108C400000000000702B00208C7A00200000C84239
:108C5000707B00200AD7233CAC7A00201520704797
:108C6000004870473CEC0C08004870473CEC0C088E
:108C7000012070470120704700207047C369012B15
:108C800006D1044B93F8AC0B431E58425841704731
:108C900000207047707B00200E4BB3F98223B3F99C
:108CA000B43307EE102A07EE903AB8EEC77AF8EE22
:108CB000E77AB0EEC77AF0EEE77AB4EE677AF1EED3
:108CC00010FAC8BFF0EE477AB7EE080A27EE800A1E
:108CD000704700BF704B00202DE9F041774C2DED1F
:108CE000048B94F81C8B8AB00546B8F1000F0CD0A9
:108CF0003122A4F1C401A4F5A04009F011FF012024
:108D00000AB0BDEC048BBDE8F0810123C36104F51A
:108D1000116696E80F0004F5106787E80F002B69CD
:108D2000D4F8FC28B3F8C070DB6A526893F8A0301E
:108D30006421022B17FB012740F0988007EE907A00
:108D40003246B8EEE70AA4F5A04106A8FBF7AAF858
:108D500006A9304616F078FB2846F0EE408AFFF769
:108D60009BFF2B69B3F9C020D3ED310A01EE102A25
:108D7000B3F9C220B0EE409A00EE102AB8EEC11A44
:108D80001A20B8EEC00A27F01FFB2B69B3F9C030D8
:108D9000F4EEC98A07EE903AF1EE10FA54BFF0EE05
:108DA000686AF0EE496AB8EEE77AC8EEA67A4246FB
:108DB0000821A4F5A040B0EE408A67EE877AB4EEB1
:108DC000670AF1EE10FA48BFB0EE678AFAF78EFC38
:108DD000DFED3B7A38EE408AB4EEE78AF1EE10FA26
:108DE0001DDBC5F81C8096E80F0004F5126585E8C8
:108DF0000F0004F61413D3ED008ADFED327AF8EE9B
:108E0000E88A3046E8EE278A16F01EF8FDEEE87A8A
:108E1000024617EE901A284615F0ECFF6FE7F4EEC5
:108E2000C98AF1EE10FA21D505AA4146304616F05E
:108E300017F818B1059B9F42A8BF1F4658F0D0FAFB
:108E4000064619EE100AF3F757FBCDE9020118EEBA
:108E5000900AF3F751FB1C4ACDE900010621304688
:108E600051F036FC6869032103F00CFA39461748C3
:108E7000FAF7CEFF286903F08FFC154805AA0021F8
:108E800015F0EEFF98B1134806AA002115F0E8FF8F
:108E900068B1DDE905316A698B4292F82010D4BFD0
:108EA0000023012363F3000182F8201027E76A6999
:108EB000D4F81439D4F82419EEE700BF707B0020F1
:108EC000000000340000C84244EC0C08702B002065
:108ED0008084002090840020014800F091BA00BFF7
:108EE000547A0020F0B52DED028B99B0044685F040
:108EF00027FD0146206900F50E700AF04FFC05467B
:108F000038B1204619B0BDEC028BBDE8F040FDF74A
:108F100055BEE36983B1012B00F02181A248F6F729
:108F2000BBF8A148F6F7AAF99F4819B0BDEC028B2F
:108F3000BDE8F040F6F700BD9FED9C8A60688DEDBE
:108F4000098A8DED0A8A8DED0B8A8DED0C8A0BAAAC
:108F500009A901230068964D7DF04AFC2069B0EE16
:108F6000480A03F0D9F863681B68D3EDCF7AFDEEA9
:108F7000E77A05F6D81017EE903AC5F81837636807
:108F80001B68D3EDD07AFDEEE77A17EE903AC5F87C
:108F90001C3704F0D3F92369D3F83C01036805F2C8
:108FA0001C725B6B05F5E361984748B163681B6809
:108FB000D3F88823C3F89423D3F88C23C3F89823D9
:108FC000206904F0D9F8A36820691E683368DF6A55
:108FD000D5F8183707EE903AD5F81C37F8EEE78A3F
:108FE00007EE903AF8EEE70ACDED050A05F08AF8AB
:108FF000DDED050AB0EE401A3046B0EE680AB8471B
:109000002069C36B93ED070A02F0CAFC206903F0E4
:10901000F7FC63688DED0D8A8DED0E8A8DED0F8A5C
:1090200018680FA97DF036FF0D9B14930E9B1593C6
:1090300002220F9B169314A910A816F07BFA5D4923
:1090400007AA10A815F08CFF48B1DFED5B7A9DED03
:10905000077AB4EEE77AF1EE10FAFFF65FAF01237C
:10906000E36105F511630FCB544E86E80F00D5F888
:10907000FC3822695B68B2F8C070642217FB0237C3
:1090800007EE907A06F11002B8EEE70AA6F5B241B3
:1090900014A8FAF707FF06F1100014A916F0D4F986
:1090A0002046B0EE408AFFF7F7FDB4EEC08AF1EE3D
:1090B00010FAF0EE408A22D508AA002106F120001D
:1090C00015F0CEFE18B1089B9F42A8BF1F4658F06E
:1090D00087F9064618EE900AF3F70EFACDE9020179
:1090E00018EE100AF3F708FA354ACDE90001062117
:1090F000304651F0EDFA6069032103F0C3F83946B8
:109100002948FAF785FE206903F046FB294907AA9A
:10911000A1F1100015F024FF636988B19DED077A75
:10912000DFED257A93F82020B4EEE77AF1EE10FA1D
:10913000ACBF0121002161F3000283F82020EDE69D
:10914000D5F81429D5F824198A4293F82010D4BFF1
:109150000022012262F3000183F82010DEE620697C
:1091600006F020F8636993F86430042B08D910489E
:10917000D0F8FC382A46596800F5126015F03AFE1E
:10918000636993F86430032B02D9206907F018FB58
:10919000236993F8D431013B012B3FF6BFAE02485F
:1091A000F6F7ACF8BAE600BF702B00200000000014
:1091B000707B002090840020000000347084002028
:1091C00044EC0C0830B5C369012B85B004D1414C87
:1091D00094F8AC3B012B04D005B0BDE83040FDF75E
:1091E0006BBCA4F54053DFED3C6AB3F982239FEDDD
:1091F0003B0A07EE102AB3F9B42307EE902AB8EE23
:10920000C77AF8EEE77AB4F9982AB0EEC77AF0EEAA
:10921000E77AB4EE677A00EE902AF1EE10FAC8BF52
:10922000F0EE477AB8EEE07AD3EDFC0A03F56B6214
:1092300070EEC70A92ED007A27EE267AF5EEC00AA4
:10924000F7EE006AF1EE10FAB4EEE67A48BFDFED11
:10925000230AF1EE10FAD8BFB0EE667AF3EE046A94
:1092600077EEA71A67EEA67AC0EE876A04F5D46295
:1092700004F512646D4693EDD77A92ED001AB0EEC4
:10928000612AA6EE872AF4EE427AF1EE10FA48BF80
:10929000B0EE672AF4EE421AF1EE10FAC8BFB0EE53
:1092A000612A26F0C3FF94E80F0007EE901A9FEDA5
:1092B0000C7AF8EEE77A85E80F00E0EE077A0948C5
:1092C0002946FDEEE77ACDED017AF9F787FF05B083
:1092D00030BD00BF707B00209A99193F000000004C
:1092E0000000C842702B00201120704700487047D2
:1092F000D4EC0C0800487047E0EC0C0801207047E3
:109300000120704701207047012070470369002247
:1093100083F8402101207047164B03F5446292ED1B
:10932000007AB3F9E029D3F8140BB5EEC07AF1EE68
:1093300010FA07EE902AC8BFDFED0F6AF8EEE77A61
:10934000CABF27EE267A20EE270A27EE000A67EE2C
:10935000A07ABDEEC00AFDEEE77A10EE102AC3F83F
:10936000182717EE902AC3F81C270368034A5B6B83
:10937000111F1847707B00200000C8428C8200201B
:109380001D49DFED1E6AB1F9E029A1F54050F5EE67
:10939000C00AD0F8E83D9342A8BF134607EE903AC2
:1093A000F1EE10FAF8EEE77AD6BF00F6EC5090ED49
:1093B000DC7A90ED007A27EE800A07EE902ACCBF87
:1093C00027EE267A27EE667AF8EEE77ABDEEC00A37
:1093D000B4EEE77AF1EE10FA58BFB0EE677A60EEBD
:1093E000870A10EE103AFDEEE00AC1F8183710EEC9
:1093F000903AC1F81C377047707B00200000C842CB
:1094000037B52B4CD4F8D03DB3F908201B8B07EEB1
:10941000102A07EE903AD4F8D43DB8EEC77AB3F9E3
:1094200008201B8BF8EEE77A054687EE270A2148CD
:1094300007EE102A07EE903AB8EEC77AF8EEE77A10
:109440008DED010AC7EE270ACDED000A09F056FF9F
:10945000DDED000A9DED010A28B1284603B0BDE804
:109460003040FFF759BF04F54053D3F89C2C520409
:1094700005D4284603B0BDE83040FFF781BFB3F9FB
:10948000E02907EE902AF8EEE77A27EE800A67EEE9
:10949000A00ABDEEC00AFDEEE00A10EE102AC3F8E5
:1094A000182710EE902AC3F81C2703B030BD00BF68
:1094B000704B00208087002010B5044685F040FAEC
:1094C0000146206900F50E700AF068F920B12046C7
:1094D000BDE81040FDF772BB114803F02FFF206973
:1094E00090F9D0304BB102F0F5F90E48F5F7D4FD04
:1094F000BDE810400B48F5F7C1BE02F061FA2069E3
:1095000005F09EFB0748F5F7C7FD0648F5F7B6FEE0
:1095100020469FED050ABDE81040FDF729BD00BFBC
:1095200048850020702B0020000000000B207047B1
:1095300000487047FAEF0C080048704758ED0C08D7
:1095400001207047012070470120704700207047BC
:1095500038B53048F6F77EFB2E48F6F75DFA2D4811
:10956000F6F742F82B481021F5F746FAE0B12A4AFF
:10957000D2F81439D2F824299342D4BF002301230E
:10958000254C94F8882972B973B304F511630FCB95
:1095900004F5106585E80F00A4F5A040FAF70EF871
:1095A000012384F8883938BD1C4AB2F9B41D00295A
:1095B000F9DD02F540529FED1A7AD2F81439D2F84B
:1095C00004299B1A07EE903AF8EEE77A67EE877A5D
:1095D00007EE101AB8EEC77AF4EEC77AF1EE10FA79
:1095E000CCBF01230023CBE7A4F54053642193F9BA
:1095F0002024D4F8180712FB01F2D3F8E81D8A42A0
:10960000A8BF0A465142C3F8E82D26F07DFFC4F8F2
:109610001807C8E7702B0020707B0020704B0020DB
:109620000AD7233CF0B52F4C2DED028B04F51165C4
:10963000074695E80F0004F5106686E80F0083B032
:10964000A4F5A040F9F794FD0146A4F5A040FAF76F
:10965000DFFB002384F88839C4F8F03094F8EC3A42
:10966000D3B394F81C3B3BB13122A4F1C401A4F55F
:10967000A04009F055FA2FE094F9A63A032B03D144
:109680002C22A4F1A801F2E7013BDBB2012B23D885
:109690003B69DB6A93F8A030022B1DD104F51261FF
:1096A000284615F0D1FEA4F1A800B0EE408AFFF7DD
:1096B000F3FAB4EEC08AF1EE10FA0DD501AA012139
:1096C000284615F0CDFB38B1B4F8983A642213FB64
:1096D00002F3019A9342D3DC012003B0BDEC028B6C
:1096E000F0BD00BF707B002070B52DED028B244DC6
:1096F00095F9A63A012B03D00020BDEC028B70BD7A
:10970000A5F54053B3F9B443002CB8BF6442A4B2EA
:109710002CB9B3F98243002CB8BF6442A4B2194EED
:10972000D6F8AC0703689B6B984730B116491748C9
:10973000272209F0F5F90120DFE706F52451144A44
:1097400001F1100015F0ECFD0028EFD1114805F5EE
:10975000D46595ED008A02F0FFFF07EE904AF8EE1F
:10976000E77AB4EEE70AF1EE10FA44BF07EE904A4A
:10977000B8EE670AB4EEC08AF1EE10FABCD5D5E7B0
:10978000707B0020705B0020C87A0020702B0020C6
:10979000908400204885002030B5424C94F8EC3A83
:1097A00089B0054663BB404DB5F9B43383EAE37134
:1097B000A1EBE37189B200294FD13C4801F092FB43
:1097C00094F8BE36CBBB95F98F33022B4DD194F86C
:1097D000F9308BB13649A1F5F4702DF003FB58B187
:1097E00001233449314884F86137282209F098F977
:1097F00018BB002384F86137012384F8BE361CE0CF
:1098000094F9A63A022B1AD103AD284615F0ECFACA
:1098100004F512630FCB85E80F0001A9A4F5A04061
:10982000FBF7BEF9D4F8F030052B06D12722A4F1BE
:10983000A801A4F5A04009F073F909B030BD85F086
:109840007FF8D4F8D030C01AB0F57A7FABD928466B
:10985000FFF74AFF0028A6D0EFE7002BB4BF4FF078
:10986000FF33012384F8D838A7E7012B0CD10F4828
:1098700001F06CFA40B10D48F9F70AFE0028B8BFB4
:109880004042B0F57A7FA2DB95F98F33042BD4D117
:1098900094F8F930002BAFD00549A1F5F4702DF004
:1098A0001DFB9CE7707B0020704B0020702B00207C
:1098B000808400209879002002207047004870477B
:1098C000D5EC0C0800487047C8500E08034B002226
:1098D000C3F81827C3F81C27704700BF707B00200F
:1098E00038B5094D04462846F5F7D6FB2846F5F766
:1098F000C5FC2046F5F7DAFC2846F6F71DF82046A9
:10990000BDE83840FDF746BB702B00200D207047A6
:109910000048704740EE0C080048704748EE0C08BD
:10992000012070470120704701207047002380F814
:10993000273080F8383001207047000001480021AE
:1099400001F0D0BA702B00202DE9F041BB4CD4F8C7
:109950001C29D4F818392DED088B1343D4F8142999
:10996000134388B005460FD1B548F6F773F9B448EC
:10997000F6F752F89FEDB30A462008B0BDEC088B0D
:10998000BDE8F0415AF0EABA0FF0E0FC90F87C3202
:10999000DB07E9D5B5F91C3095F8271009EE103A28
:1099A000B5F9243008EE903AB8EEC99AF8EEE88A94
:1099B000002940F0E0809FEDA4AA29EE0ABA012216
:1099C000FDEECB7AA4F5A04017EE903AC4F88836A5
:1099D000F9F78CFEA86900F57F700790B0EE408A19
:1099E00029F084FCDFED997A20EE270A26F056FC58
:1099F0000798F0EE409A29F0C3FCA4F5A040F0EEE1
:109A000040AAFCF751FD00287FD104F5116696E8C5
:109A10000F0005F1280787E80F0096E80F0004F50E
:109A2000126C8CE80F008A4F87E80F00D4F82439B5
:109A300007EE903AF8EEE77AF0EE680A77EE8B7A66
:109A4000B0EE690AFDEEE77A07F1200017EE903AD2
:109A5000C4F8243915F09EFD002384F8F13695F9F9
:109A6000263003EB830303EB83039B000121A7F55F
:109A7000B240A4F8B636F4F761FC94F80087B8F168
:109A8000000F78D1A7F564579FED727AB7F9583374
:109A900007EE903AF8EEE77A67EE877AF4EEE7AAF7
:109AA000F1EE10FA67DD57F09BFC064619EE900ABE
:109AB000F2F722FDCDE9040118EE900AF2F71CFD41
:109AC000CDE9020119EE100AF2F716FD624ACDE95E
:109AD00000010621304650F0FBFD84F031FFC4F850
:109AE0007486C4F8600684F02BFF0123C4F8700666
:109AF00029EE8A0A85F8273026F0FAFBBDEEC00A67
:109B000010EE103AC4F8783635E084F019FFD4F836
:109B10001037C01A42F2107398427FF676AFF0EE1B
:109B2000087AF4EEE7AAF1EE10FA7FF76EAFBCEE1A
:109B3000C88A04F5126718EE103A9BB208EE103A84
:109B4000B8EEC88A04F51166B4EEC89AF1EE10FAC0
:109B500048D857F045FC414A062150F0B9FD96E837
:109B60000F0087E80F00012385F827300321A4F5B3
:109B7000A040F4F7E3FB32480BF076F830B1304800
:109B80000321F4F7DBFB002385F82730D4F80437F2
:109B9000012B40F0B680D4F81439EA6A9FED2AAA66
:109BA0009B1A07EE903AD4F878360133F8EEE79A2C
:109BB0005CD0DFED2B7AE9EE0A7AF4EEE79AF1EE6B
:109BC00010FA0ADA274905F1280015F03DFCF4EEF9
:109BD000C08AF1EE10FA00F2948019480321F4F7DC
:109BE000ADFB8EE057F0FCFB1F4A062150F070FDE4
:109BF00096E80F0005F1280C8CE80F0096E80F009E
:109C000087E80F00D4F8243907EE903A39EE488AF5
:109C1000F8EEE77AF0EE680AE8EE0A7A3846B0EE37
:109C2000690AFDEEE77A17EE903AC4F8243915F088
:109C3000B1FC012185F8271099E700BF707B002057
:109C4000702B0020000000000000C842E02E65429A
:109C5000708400209A99993E91EE0C0850EE0C0801
:109C6000000048C3808400206CEE0C08B5F91E305B
:109C700007EE903AF8EEE77A05F1280667EE8A7A61
:109C8000F4EEE79AF1EE10FA55DB4449304615F050
:109C9000ABFADFED437AB6EE008AA0EE278A96E8AB
:109CA0000F00BDEEC88A9FED3F0AB8EEC88A04F5E2
:109CB000126728EE008A87E80F00F0EE680A3A483B
:109CC000B0EE480A15F066FCD4F8243907EE903A55
:109CD000F8EEE77A28EE0A0AE9EE0A7AFDEEE77A6C
:109CE00017EE903AC4F8243926F002FBBDEEC00A04
:109CF00010EE103AC4F87836D4F80437012B3FF44C
:109D000058AF2A480AF090FF18B128480321F4F709
:109D100015FBD4F80437012B17D124480AF016FD9F
:109D200022480AF061FE214808B0BDEC088BBDE86E
:109D3000F0410AF06FBD1949304615F085FBF4EE8D
:109D4000C08AF1EE10FAA0D9D6E795F838302BB9D1
:109D5000174862F095FC012385F838301348F5F771
:109D600079FF1248F5F758FE1048F5F73DFC114809
:109D700090F88C356BB1002380F88C3533220221AA
:109D8000A0F5405008B0BDEC088BBDE8F041FBF7F2
:109D9000BFBF08B0BDEC088BBDE8F0818084002017
:109DA000A00CB3450AD7233C90840020702B0020E0
:109DB000C04D0020705B002010B50446FCF7B4FFD6
:109DC0002046054B40F8283B15F00EF82046034985
:109DD00045F02EF8204610BD44EF0C08DCEE0C08D0
:109DE0001820704700487047ACEF0C0800487047D7
:109DF000B4EF0C0801207047012070470120704724
:109E000008B50548F5F726FF0348F5F705FEBDE858
:109E100008400148F5F7E8BB702B002008B506485C
:109E200082F0C0FABCEEC00A044810EE103A99B2B3
:109E3000BDE8084001F056B800570020702B002004
:109E400010B50D4CD4F8783D002B12DDA4F5005070
:109E5000FAF756FCA4F5005000F058FB04F5396001
:109E600082F0EAFB04F53960044981F083FF0120A8
:109E700010BD0020FCE700BF704B00209084002044
:109E800070B5214CD4F8CC0003688EB05B6898475D
:109E900007282CD00A2809D0062805D10FF056FA39
:109EA00090F87C32DB071BD4012017E004F26476C3
:109EB0000FCE07AD0FC596E8070085E8070009AB90
:109EC0000FCB01AD85E80F00D4F82C39009304F5D1
:109ED00012630ECBA4F5C870FEF7EEF90EB070BD9C
:109EE0000FF034FA00F51B700FC801ADEAE707A9BF
:109EF000A4F50770FDF708FF0028D5D00799A4F551
:109F0000C870FEF7B7F9E9E7707B0020F0B585B0BF
:109F10000E4E0391144657F063FA06F5A047054626
:109F2000D7F8CC00026892689047039B0090084ADB
:109F30002846062150F0CCFBD7F8CC1022463046FC
:109F400005B0BDE8F04008F0EBBD00BF702B00206D
:109F5000BCEF0C082DE9F0472DED028B96B00024E4
:109F600007466C4882F048FA0594069407940FF06F
:109F7000EDF905A90EF020FF70B3674B93ED007A61
:109F8000B5EEC07AA3F67459F1EE10FA09F540580F
:109F900027DBDDED067ADDED056A67EEA77A27EEB1
:109FA000077AE6EEA67AF4EEC77AF1EE10FA18DD3B
:109FB000D8F8CC0003685B6898470A2811D057F09E
:109FC0000FFA564A062150F083FB2622A8F5D671D7
:109FD000A8F5A04008F0A4FD16B0BDEC028BBDE8CA
:109FE000F087D8F8CCA04E4B01949A450294039484
:109FF000049417D108F264760FCE08AD0FC596E829
:10A00000070085E8070011A814F0EEFEB8F8BC17A9
:10A010000FAA0AF510602CF013F878BB0294019493
:10A02000049403949FED3F0A01A829F0F7F803A8D0
:10A030008DED080A9FED3B0ACDED090A29F0EEF8F7
:10A0400034488DED0F0AB0EE401AF0EE601ACDEDF7
:10A05000100A9DED080ADDED090A82F027F90628AD
:10A06000044618D10023C8F8D43884F069FC2E497E
:10A07000C8F8240D274881F07DFEADE701A911A89D
:10A0800015F05EF80028C9D003A90AA815F058F801
:10A090000028C3D0C6E709F54D6984F051FCDFED17
:10A0A000237A99ED008AD8F8246D28EE278ADFED0F
:10A0B000207AB4EEE78AF1EE10FA0546384658BF2A
:10A0C000B0EE678AFFF7DCFE48B9022C16D0BCEE72
:10A0D000C88AAD1B18EE103A9D42FFF47DAF013CDB
:10A0E000062C0ED8DFE804F0040A0D0D100D130045
:10A0F000104924223846FFF709FF6DE70E49252253
:10A10000F8E70E491622F5E70D492622F2E70D4938
:10A110000122EFE700570020E4580020D8EF0C0898
:10A12000987900200000C8429084002000007A4402
:10A1300000409C46FEEF0C0813F00C0828F00C08B9
:10A1400040F00C0857F00C08032070470048704797
:10A15000DCF00C0800487047E8F00C08F8B52A4D10
:10A1600006460027A5F54050A5F88875F5F7B8FC18
:10A17000B369A5F58052D3F8F811D2F8E83D9942B9
:10A1800005F5005421DBC4F81837B36992EDDC7A89
:10A19000D3ED7F6A9FED1D6AF8EEE66A27EE067A38
:10A1A000F4EEC76AF1EE10FA18DBBDEEC77A17EECF
:10A1B000103A1748C4F81C37FBF7C0FB20B1D4F89D
:10A1C0001C375B42C4F81C37F8BD5B429942DADDAC
:10A1D000012385F88835C4F81877D6E702F6EC52E3
:10A1E000D2ED007A67EE867AF4EEE76AF1EE10FAC5
:10A1F00093BFFDEEE77A012385F8893517EE903A93
:10A2000088BF0023D5E700BF705B00200000C84274
:10A21000702B002070B500212DED028B04463448D0
:10A22000344D06F0DBFE32480021F0EE408A06F0A5
:10A23000DFFE95F88835B0EE408AD3B1B0EE680AFB
:10A24000042059F08BFE95F8893593B3B0EE480A97
:10A25000132059F083FE2648002106F0D3FE204645
:10A26000FCF786FEBDEC028B2046BDE87040FCF793
:10A2700091BE05F50056A5F54050F4F70DFFD6F850
:10A280001837002B0CDCD6F81837002BDBDA04204B
:10A2900059F078FEB4EEE80AF1EE10FACED4D2E727
:10A2A000042059F06FFEB4EEE80AF1EE10FAEADD90
:10A2B000C4E7114D0E48F4F7E1FFD5F81C37002B29
:10A2C0000CDCD5F81C37002BC5DA132059F05AFEE8
:10A2D000B4EEC80AF1EE10FAB8D4BCE7132059F076
:10A2E00051FEB4EEC80AF1EE10FAEADDAEE700BFA7
:10A2F000702B0020705B0020707B0020F0B52DEDEE
:10A30000028B1E4690F814318FB004461746B0EE0B
:10A31000408A53B1C56A45B195F8CB1039B157F0B1
:10A320005FF8274A062150F0D3F9042044E02E229A
:10A3300002A80191A9F06CFD2B6801AA5B6832218B
:10A340002846984738B957F04BF81E4A01AB02210E
:10A3500050F0BEF9E9E794F8D83143B9012584F803
:10A36000D8512946204604F0C3F8174B5D7284F09B
:10A37000E7FA9FED160ADFED167ABDF85830A4F81B
:10A38000E63128EE000A9DF85C30C4F8DC01B4EE3A
:10A39000E70AF1EE10FA58BFB0EE670ABCEEC00A49
:10A3A000082BA8BF082384ED780A84F8E47184F8A8
:10A3B000E56184F8E83100200FB0BDEC028BF0BD00
:10A3C00060F10C0880F10C085D89002000007A44DF
:10A3D0000060EA4638B590F8D83104464BB1002504
:10A3E00080F8D851294604F083F8024BC4E9775528
:10A3F0005D7238BD5D89002070B590F8D831044693
:10A400006BB384F09DFAD4F8DC21D4F8E031821AE1
